:100000000000032089BE01006DBE010025BE010075
:1000100025BE010025BE010025BE010025BE010050
:1000200025BE010025BE010025BE01006DBE0100F8
:100030006DBE010025BE010041B30100B9B501004C
:100040006DBE01006DBE01006DBE01006DBE010000
:100050006DBE01006DBE01006DBE01006DBE0100F0
:100060006DBE01006DBE01006DBE01006DBE0100E0
:100070006DBE01006DBE01006DBE01006DBE0100D0
:100080006DBE01006DBE01006DBE01006DBE0100C0
:100090006DBE01006DBE01006DBE01006DBE0100B0
:1000A0009D7D0100F97E01006DBE01006DBE010065
:1000B0006DBE01006DBE01006DBE0100DDD001000E
:1000C0006DBE01003DF201006DBE010099F301001B
:1000D0006DBE0100C9F401006DBE01006DBE0100DE
:1000E0006DBE01006DBE01006DBE01006DBE010060
:1000F0006DBE01006DBE01006DBE01006DBE010050
:100100006DBE01006DBE01006DBE01006DBE01003F
:100110006DBE010011D401006DBE01006DBE010075
:100120006DBE01006DBE01006DBE01006DBE01001F
:100130006DBE01006DBE01006DBE01006DBE01000F
:100140008DB001006DBE0100F9F501006DBE01002A
:100150006DBE01006DBE01006DBE01006DBE0100EF
:100160006DBE01006DBE0100558001006DBE010035
:100170006DBE01006DBE01006DBE01006DBE0100CF
:100180006DBE0100CD4701006DBE01006DBE0100D6
:100190006DBE01006DBE010029F701006DBE0100BA
:1001A0006DBE01006DBE01006DBE01006DBE01009F
:1001B0006DBE01006DBE01006DBE01006DBE01008F
:1001C0006DBE01006DBE01006DBE01006DBE01007F
:1001D000FFFFFFFFFFFFFFFFFFFFFFFFFFFFFFFF2F
:10040000FFFFFFFFFFFFFFFFFFFFFFFFDEF9FFFF23
:1004100010B5054C237833B9044B13B10448AFF33E
:1004200000800123237010BD00F0002000000000B8
:10043000D4610200084B10B51BB108490848AFF35E
:1004400000800848036803B910BD074B002BFBD0A0
:10045000BDE81040184700BF0000000004F0002075
:10046000D4610200F4E9002000000000704700BFE2
:1004700010B54FF4097104461BF0CAFE204610BDAA
:1004800070B54FF06A522DED028B064644F2D82328
:1004900008EE902A40F6DB72C0F202034FF61A050E
:1004A00040F6DA70C4F24902C2F20005C3F64920F0
:1004B00008EE102A336000240FE007EE904AF8EEB1
:1004C000E77A77EE807A67EEA87A67EE887A27EE89
:1004D000800A1FF051FC10EE100A22F00FFC41ECD4
:1004E000100B1FF0B1FA00230022CCF2900351EC64
:1004F000100B22F057FC41EC100B1FF0B9FA51EC35
:10050000100B22F027FF0134B4F5806FB6EE000A1D
:1005100025F8020FD1D14FF06A534FF21A0508EEB9
:10052000103AC2F20005002407EE904AF8EEE77A8E
:10053000013467EE887A17EE900A22F0DFFB9FED18
:10054000140B41EC110B1FF017FD002351EC100BA5
:100550000022C3F6F07322F071FA00230022C4F2E5
:10056000B00322F01FFC22F015FF22F0C7FB41EC84
:10057000100B1FF07DFA51EC100B22F0EBFEB4F5DE
:10058000806F25F8020FCFD1BDEC028B304670BDD5
:100590000000000000000040704700BF10B54FF49D
:1005A000097104461BF034FE204610BD2DE9F04FC2
:1005B0004DF63456C2F200060A9D0B989DF8307035
:1005C000B6F800C044F2F024C0F20204C5EB000A01
:1005D000002F18BF0C466FEA0C0B0AF1200A4DF6EB
:1005E00034194DF63438043A271FA1F1040E0FFADE
:1005F0008BFB4FEAAA1AC2F20009C2F200080026D9
:1006000027E0B4F5007F02D08CB3C943C9B239F8F2
:1006100011104CEA010101EBC00080B20BEA0004AA
:10062000E143C9B2241238F8111001F58061490084
:10063000E14010EA0C0F18BFC94357F8044F09985E
:1006400009B2013604EB8131402E03444EF8041FF9
:1006500010D052F8041F1944891301F44074554412
:10066000B4F5807FC9B2A8B2CBD1C943C9B239F8B9
:100670001110D0E7BDE8F08F2DE9F04F4DF634555D
:10068000C2F2000509982E880A9D9DF82C7044F24C
:10069000F024C0F20204C0EB050E002F14BF0F4679
:1006A00027466FEA06090EF1200E4DF634184DF676
:1006B000343C3C1F0D1F0FFA89F9FC374FEAAE1E80
:1006C000C2F20008C2F2000C2AE0BBF5007F04D0A1
:1006D000BBF1000F30D0C943C9B238F81110314313
:1006E00001EBCA0A1FFA8AFA09EA0A0B6FEA0B0140
:1006F000C9B24FEA2B2B3CF8111001F5806149007B
:100700001AEA060F21FA0BF154F804AF18BFC943D7
:1007100009B20AEB8131BC421A4445F8041F0ED0DD
:10072000911301F4407B7044BBF5807F1FFA80FA7F
:10073000C9B2CAD1C943C9B238F81110D0E7BDE86F
:10074000F08F00BF2DE9F04F4DF6345083B0C2F268
:1007500000000D9EB0F800C00C9C9DF840A00F9FBB
:100760000E980E9D019344F2F02EC0F2020EC4EBDF
:10077000060B6FEA0C06BAF1000F14BF8A46F24668
:1007800033B20BF1200B4DF634194DF63438AAF183
:10079000040600686D680093A1F1040E0AF1FC0ADA
:1007A0004FEAAB1B0137C2F20009C2F2000829E090
:1007B000B0F5007F02D098B3DB43DBB239F81330D9
:1007C0004CEA030303EBC101009B89B203EA010079
:1007D000C343DBB2001238F8133003F580635B00CB
:1007E000C34011EA0C0F18BFDB4356F8041F0198F1
:1007F0001BB29B031944564502444EF8041F284679
:1008000011D01D4643193B4113449B1303F4407020
:100810005C44B0F5807FDBB2A1B2C9D1DB43DBB26F
:1008200039F81330CEE70E9A1560536003B0BDE877
:10083000F08F00BF2DE9F04F45F23C4403EB43033A
:10084000C0F2020404EBC3050646144689460FCDE8
:1008500091B00AAF0FC795E80300002387E80300B3
:10086000012704F160088DF8247007978DF8253072
:100870008DF826300AAD48E00AF1FF3101EB011195
:1008800006EB0111133121F00F0194E80140C0146F
:10089000C0F500706060BEF1000F3FD0BEF5FE7F76
:1008A0003EDA10AFBA441AF81CCCBCF1000F04D0E9
:1008B00012F1000C18BF4FF0010CC3F301123AB152
:1008C00010AF07EB020B1BF81CBCBBF1000F34D1BF
:1008D00003F0C003C02B02D11B9B0F2B41DDA3688B
:1008E000E2680190CDF808C0CDF800E03046FFF78F
:1008F000C3FE9DF81C300AF81C3CE368A26803EBB9
:100900008213E3601034A04514D055F8043B13F073
:10091000030A03F00402AFD14946B6E740F2FF1ED6
:10092000B0F5FE7FBDDB002AE7D110AB9A440AF890
:100930001C2CE2E711B0BDE8F08F013A02EB021285
:10094000E368CDF80CC006EB02120290CDF804E08B
:10095000A0680090133222F00F023046FFF726FE07
:10096000C7E71F46E268A36803971A9F0190CDF876
:1009700010C00297CDF800E03046FFF7E3FEB8E77D
:1009800000207047704700BF704700BF704700BF2E
:10099000704700BF704700BF10B504461AF0F8FA60
:1009A000204610BD10B5044623F0CAF90146204682
:1009B000BDE810401EF046BA44F2884008B5182140
:1009C000C0F202001EF03EFA41F69853C2F2010353
:1009D000FB21986C03681B68984744F2A4400F21E0
:1009E000C0F202001EF02EFA4FF60F301DF0A0FBF1
:1009F00044F2B440C0F202000F211EF023FA4EF27E
:100A0000C000C2F20000BDE808401AF0CBBE00BF33
:100A100044F2C44008B51421C0F202001EF012FADC
:100A200041F69853C2F20103FC21986C03681B68DD
:100A3000984744F2A4400F21C0F202001EF002FACF
:100A40004FF60F401DF074FB44F2B440C0F20200B8
:100A50000F211EF0F7F94EF2C000C2F20000BDE80F
:100A600008401AF09FBE00BF44F2DC4008B51D21CB
:100A7000C0F202001EF0E6F941F69853C2F20103FB
:100A8000FE21986C03681B68984744F2A4400F212C
:100A9000C0F202001EF0D6F94FF60F601DF048FBC1
:100AA00044F2B440C0F202000F211EF0CBF94EF226
:100AB000C000C2F20000BDE808401AF073BE00BFDB
:100AC00044F2FC4008B51621C0F202001EF0BAF94B
:100AD00041F2E040C2F201004FF20F6119F098F9C3
:100AE00044F214501421C0F202001EF0ABF94FF290
:100AF0000F601DF01DFB44F2B440C0F202000F2154
:100B00001EF0A0F94EF2C000C2F20000BDE808409D
:100B10001AF048BE44F22C5008B51521C0F202006C
:100B20001EF090F941F69853C2F20103FA21986C35
:100B300003681B68984744F2A4400F21C0F20200EA
:100B40001EF080F94FF60F201DF0F2FA44F2B44087
:100B5000C0F202000F211EF075F94EF2C000C2F281
:100B60000000BDE808401AF01DBE00BF38B544F2D1
:100B700044504EF2C00541F2D4441021C2F20104A7
:100B8000C2F20005C0F202001EF05CF928461AF01D
:100B900009FE20680EF02EFD20680EF037FC20685C
:100BA0000EF048FC44F258501B21C0F202001EF027
:100BB00049F941F69853C2F20103FF21986C03688A
:100BC0001B68984744F2A4400F21C0F202001EF0B7
:100BD00039F94FF60F701DF0ABFA44F2B440C0F291
:100BE00002000F211EF02EF92846BDE838401AF009
:100BF000D9BD00BF10B50446240444F2745004F477
:100C0000FE041521C0F2020044F473441EF01AF9E8
:100C100044F0020441F2E0402146C2F2010019F022
:100C2000F7F844F214501421C0F202001EF00AF941
:100C300020461DF07DFA44F2B440C0F202000F21BC
:100C40001EF000F94EF2C000C2F20000BDE81040F4
:100C50001AF0A8BD44F28C5008B51321C0F202006E
:100C60001EF0F0F841F2E040C2F201004FF60F3101
:100C700019F0CEF844F214501421C0F202001EF014
:100C8000E1F84FF60F301DF053FA44F2B440C0F2D1
:100C900002000F211EF0D6F84EF2C000C2F2000092
:100CA000BDE808401AF07EBD44F2A05008B50F21FF
:100CB000C0F202001EF0C6F841F2E040C2F20100AC
:100CC0004FF60F4119F0A4F844F214501421C0F269
:100CD00002001EF0B7F84FF60F401DF029FA44F25B
:100CE000B440C0F202000F211EF0ACF84EF2C0007A
:100CF000C2F20000BDE808401AF054BD44F2B05002
:100D000008B51821C0F202001EF09CF841F2E04044
:100D1000C2F201004FF60F6119F07AF844F2145054
:100D20001421C0F202001EF08DF84FF60F601DF086
:100D3000FFF944F2B440C0F202000F211EF082F825
:100D40004EF2C000C2F20000BDE808401AF02ABD11
:100D500044F2CC5008B51021C0F202001EF072F827
:100D600041F2E040C2F201004FF60F2119F050F8B5
:100D700044F214501421C0F202001EF063F84FF642
:100D80000F201DF0D5F944F2B440C0F202000F214B
:100D90001EF058F84EF2C000C2F20000BDE8084054
:100DA0001AF000BD38B505464EF2C00444F2E050DA
:100DB000C2F200041E21C0F202001EF043F82946D0
:100DC00000230A2220461AF0FFFC44F200600E21A4
:100DD000C0F202001EF036F84DF63853C2F200039E
:100DE0000A22197C204600231AF0EEFC44F210601F
:100DF0000121C0F202001EF025F820461AF0D2FCB4
:100E0000002038BD10B5044644F214601F21C0F222
:100E1000020004F00F041EF015F844F010044FF225
:100E2000021343EA044441F2E0402146C2F20100C9
:100E300018F0EEFF44F214501421C0F202001EF02C
:100E400001F820461DF074F944F2B440C0F20200EB
:100E50000F211DF0F7FF4EF2C000C2F20000BDE806
:100E600010401AF09FBC00BF44F2346008B5102156
:100E7000C0F202001DF0E6FF41F69853C2F20103F2
:100E8000FA21986C03681B68984744F2A4400F212C
:100E9000C0F202001DF0D6FF41F2E040C2F20100B4
:100EA0004FF60F2118F0B4FF44F21450C0F20200C4
:100EB00014211DF0C7FF4EF2C000C2F20000BDE8D1
:100EC00008401AF06FBC00BF44F2486008B5132117
:100ED000C0F202001DF0B6FF41F69853C2F20103C2
:100EE000FB21986C03681B68984744F2A4400F21CB
:100EF000C0F202001DF0A6FF41F2E040C2F2010084
:100F00004FF60F3118F084FF44F21450C0F2020083
:100F100014211DF097FF4EF2C000C2F20000BDE8A0
:100F200008401AF03FBC00BF44F25C6008B50F21D6
:100F3000C0F202001DF086FF41F69853C2F2010391
:100F4000FC21986C03681B68984744F2A4400F2169
:100F5000C0F202001DF076FF41F2E040C2F2010053
:100F60004FF60F4118F054FF44F21450C0F2020043
:100F700014211DF067FF4EF2C000C2F20000BDE870
:100F800008401AF00FBC00BF44F26C6008B518218D
:100F9000C0F202001DF056FF41F69853C2F2010361
:100FA000FE21986C03681B68984744F2A4400F2107
:100FB000C0F202001DF046FF41F2E040C2F2010023
:100FC0004FF60F6118F024FF44F21450C0F20200F3
:100FD00014211DF037FF4EF2C000C2F20000BDE840
:100FE00008401AF0DFBB00BF44F2886008B51B213F
:100FF000C0F202001DF026FF41F69853C2F2010331
:10100000F621986C0368DB6C984744F2A4400F21EA
:10101000C0F202001DF016FF4FF20F601DF088F8BD
:1010200044F2B440C0F202000F211DF00BFF4EF25B
:10103000C000C2F20000BDE808401AF0B3BB00BF18
:1010400038B544F244504EF2C00541F2D444102168
:10105000C2F20104C2F20005C0F202001DF0F2FE6D
:1010600028461AF09FFB20680EF0C4FA20680EF0A4
:10107000CDF920680EF0DEF944F2A4601621C0F22A
:1010800002001DF0DFFE41F2E040C2F201004FF627
:101090000F7118F0BDFE44F214501421C0F202008A
:1010A0001DF0D0FE4FF60F701DF042F844F2B44030
:1010B000C0F202000F211DF0C5FE2846BDE83840F1
:1010C0001AF070BB38B544F244504EF2C00541F2FC
:1010D000D4441021C2F20104C2F20005C0F20200A1
:1010E0001DF0B0FE28461AF05DFB20680EF082FA73
:1010F00020680EF08BF920680EF09CF944F2BC6079
:101100001621C0F202001DF09DFE41F69853C2F276
:101110000103FF21986C03681B68984744F2A440C0
:101120000F21C0F202001DF08DFE41F2E040C2F23C
:1011300001004FF60F7118F06BFE44F21450C0F22C
:10114000020014211DF07EFE2846BDE838401AF04A
:1011500029BB00BF44F2D46008B51621C0F20200DA
:101160001DF070FE41F69853C2F20103F621986C0F
:101170000368DB6C984744F2A4400F21C0F20200E0
:101180001DF060FE41F2E040C2F201004FF20F613B
:1011900018F03EFE44F21450C0F2020014211DF07B
:1011A00051FE4EF2C000C2F20000BDE808401AF045
:1011B000F9BA00BFF8B5064644F2EC600C46C0F23E
:1011C0000200122115461DF03DFE711EC9B20F2905
:1011D00015D841F69857C2F2010741F0A001B86C4A
:1011E00003681B689847B86C036804F07F011B68AC
:1011F0009847B86C036805F07F011B68984744F274
:1012000000700A21C0F202001DF01CFE6B1E1B02C2
:10121000240404F4FE0403F470632343310143F413
:10122000504343F00D03C9B241F2E0401943C2F20A
:10123000010018F0EDFD44F21450C0F20200142138
:101240001DF000FE4EF2C000C2F20000BDE8F84002
:101250001AF0A8BAF8B541F2D443C2F20103054628
:101260001B6801F5005644F20C700C46013D0D213F
:10127000C3F8C060C0F202001DF0E4FDE9B20F291E
:1012800015D841F69857C2F2010741F0E001B86C59
:1012900003681B689847B86C036806F07F011B68F9
:1012A0009847B86C0368C6F3C6111B68984744F2A8
:1012B000A44004F30D040F2104F50054C0F2020011
:1012C0001DF0C0FD2902230403F4FE0301F4706144
:1012D000194341F46041640404F0FE4441F00E01FE
:1012E00041F2E0402143C2F2010018F091FD44F2C6
:1012F0001450C0F2020014211DF0A4FD4EF2C000F3
:10130000C2F20000BDE8F8401AF04CBA1F2970B5CF
:101310000C46054608D84DF63853C2F2000318793A
:101320000FF050F90AF014FF44F21C700D21013D3A
:10133000C0F202001DF086FDE9B20F290FD841F678
:101340009856C2F2010641F0C001B06C03681B68F8
:101350009847B06C036804F07F011B68984744F21B
:10136000A4400F21C0F202001DF06CFD230403F421
:10137000FE03290243F4404343F00C0301F470617F
:1013800041F2E0401943C2F2010018F041FD44F27D
:101390001450C0F2020014211DF054FD4EF2C000A2
:1013A000C2F20000BDE870401AF0FCB9F0B54AF294
:1013B0003472C2F2010283B040F2206311680091DE
:1013C000C2F2010300991E681268019241F2AE4513
:1013D000C2F2010541F2AC42C2F20102891B44F2A1
:1013E0002C704EF2C004C2F20004019F2980002636
:1013F0000C21C0F2020016701F601DF023FD2B8827
:1014000020464EF6602191FBF3F11AF06DF944F29B
:101410003C700521C0F202001DF014FD2988204611
:101420001AF062F944F244700F21C0F202001DF07C
:1014300009FD20461AF0B6F903B0F0BD08B541F237
:10144000AC41C2F201014AF6AB230A780132D2B2B2
:10145000CAF6AA23A3FB02031B0903EB4303A2EB77
:10146000C30313F0FF0F0A7001D1FFF79FFF44F28F
:1014700054701021C0F202001DF0E4FC41F2E04083
:10148000C2F201004FF60F0118F0C2FC44F21450F2
:101490001421C0F202001DF0D5FC4FF60F001CF025
:1014A00047FE44F2B440C0F202000F211DF0CAFC16
:1014B0004EF2C000C2F20000BDE808401AF072B956
:1014C00008B541F2AC41C2F201014AF6AB230A78F9
:1014D0000132D2B2CAF6AA23A3FB02031B0903EB13
:1014E0004303A2EBC30313F0FF0F0A7001D1FFF710
:1014F0005DFF44F268701521C0F202001DF0A2FCED
:1015000041F69853C2F20103F821986C03681B68F6
:10151000984744F2A4400F21C0F202001DF092FC53
:101520004FF60F001CF004FE44F2B440C0F202007B
:101530000F211DF087FC4EF2C000C2F20000BDE892
:1015400008401AF02FB900BF08B541F2AC41C2F211
:1015500001014AF6AB230A780132D2B2CAF6AA23B5
:10156000A3FB02031B0903EB4303A2EBC30313F02A
:10157000FF0F0A7001D1FFF719FF44F280701021AC
:10158000C0F202001DF05EFC41F69853C2F2010366
:10159000F821986C03681B68984744F2A4400F2117
:1015A000C0F202001DF04EFC41F2E040C2F2010028
:1015B0004FF60F0118F02CFC44F21450C0F2020058
:1015C00014211DF03FFC4EF2C000C2F20000BDE845
:1015D00008401AF0E7B800BF1F2970B50C46054651
:1015E00008D84DF63853C2F2000318790EF0EAFF1E
:1015F0000AF0AEFD44F294701221013DC0F20200E7
:101600001DF020FCE9B20F290FD841F69856C2F21E
:10161000010641F0C001B06C03681B689847B06CCC
:10162000036804F07F011B68984744F2A4400F212F
:10163000C0F202001DF006FC230403F4FE0328029E
:1016400043F4404343F00C0300F4706018431CF073
:101650006FFD44F2B440C0F202000F211DF0F2FB16
:101660004EF2C000C2F20000BDE870401AF09AB815
:1016700070B5064644F2A8700C46C0F2020017216D
:1016800015461DF0DFFB711EC9B20F292BD841F69C
:101690009856C2F2010641F0A001B06C03681B68C5
:1016A0009847B06C036804F07F011B689847B06CE2
:1016B000036805F07F011B68984744F20070C0F290
:1016C00002000A211DF0BEFB44F2B440C0F2020049
:1016D0000F211DF0B7FB4EF2C000C2F20000BDE8C2
:1016E00070401AF05FB844F20070C0F202000A21A4
:1016F0001DF0A8FB002EE7D1681E0002240404F4AC
:10170000FE0400F47060204340F4504040F00D00AF
:101710001CF00EFDD8E700BF1F2938B50C46054662
:1017200008D84DF63853C2F2000318790EF04AFF7C
:101730000AF00EFD240404F4FE04013D44F2C070DE
:1017400044F440442D020D2105F47065C0F20200FE
:1017500044F00C041DF076FB2C4341F2E04021469E
:10176000C2F2010018F054FB44F214501421C0F2EC
:1017700002001DF067FB20461CF0DAFC44F2B44086
:10178000C0F202000F211DF05DFB4EF2C000C2F25C
:101790000000BDE838401AF005B800BF70B5064635
:1017A00044F2D07015460C46C0F2020012211DF022
:1017B00049FB6B1E1B02240404F4FE0403F4706353
:1017C000234343F45043340143F00D03E4B21C437C
:1017D00041F2E0402146C2F2010018F019FB44F248
:1017E0001450C0F2020014211DF02CFB16B9204643
:1017F0001CF09EFC44F2B440C0F202000F211DF028
:1018000021FB4EF2C000C2F20000BDE8704019F0AA
:10181000C9BF00BF38B541F698550446C2F201056C
:1018200044F2E4701A21C0F202001DF00BFBA86C18
:101830000368F3211B689847A86C036804F07F01D4
:10184000DB6C984744F2A4400F21C0F202001DF067
:10185000F9FA200400F4FE0040F4734040F0020066
:101860001CF066FC44F2B440C0F202000F211DF0EF
:10187000E9FA4EF2C000C2F20000BDE8384019F0AB
:1018800091BF00BF70B54DF63853C2F200030E464B
:101890001B7C1446054623B1984202D0FFF782FA1A
:1018A00038B141F2D443C2F20103314618680DF059
:1018B00077FC44F600001221C0F202001DF0C2FACB
:1018C000230603F0FE43340443F40043013D43F098
:1018D000080304F4FE042D021C4305F470652C4338
:1018E00041F2E0402146C2F2010018F091FA44F2C0
:1018F00014501421C0F202001DF0A4FA20461CF07E
:1019000017FC44F2B440C0F202000F211DF09AFA15
:101910004EF2C000C2F20000BDE8704019F042BFB4
:1019200070B54DF63853C2F200030E461B7C1446C8
:10193000054623B1984202D0FFF734FA40B141F294
:10194000D443C2F201032246186831460DF0E8F98B
:1019500044F614001121C0F202001DF073FA2306B0
:1019600003F0FE43340443F41043013D43F0090304
:1019700004F4FE042D021C4305F470652C4341F26F
:10198000E0402146C2F2010018F042FA44F214503D
:101990001421C0F202001DF055FA20461CF0C8FBCD
:1019A00044F2B440C0F202000F211DF04BFA4EF297
:1019B000C000C2F20000BDE8704019F0F3BE00BFE5
:1019C00038B541F698550446C2F2010544F62800A0
:1019D0001521C0F202001DF035FAA86C0368F3214E
:1019E0001B689847A86C036804F07F01DB6C98477C
:1019F00044F2A4400F21C0F202001DF023FA21049A
:101A000001F4FE0141F4734141F2E04041F0020172
:101A1000C2F2010018F0FCF944F21450C0F20200C6
:101A200014211DF00FFA4EF2C000C2F20000BDE812
:101A3000384019F0B7BE00BF38B541F69855044696
:101A4000C2F2010544F640002421C0F202001DF05C
:101A5000F9F9A86C0368F1211B689847A86C036822
:101A600021461B68984744F2A4400F21C0F20200AF
:101A700004F00F041DF0E6F944F010044FF20210D8
:101A800040EA04401CF054FB44F2B440C0F20200AF
:101A90000F211DF0D7F94EF2C000C2F20000BDE8E0
:101AA000384019F07FBE00BF38B541F6985504465E
:101AB000C2F2010544F668001F21C0F202001DF0C9
:101AC000C1F9A86C0368F1211B689847A86C0368EA
:101AD00021461B68984744F2A4400F21C0F202003F
:101AE00004F00F041DF0AEF944F010044FF202119F
:101AF00041F2E04041EA0441C2F2010018F088F9E5
:101B000044F21450C0F2020014211DF09BF94EF271
:101B1000C000C2F20000BDE8384019F043BE00BF6B
:101B200038B541F2D443C2F2010301F500521B68FB
:101B300005460C4644F68800C3F8C0200D2104F386
:101B40000D04C0F202001DF07DF904F500536C1E77
:101B50001A04240202F4FE0204F47064144344F4F0
:101B600060445B0403F0FE4344F00E041C4341F266
:101B7000E0402146C2F2010018F04AF944F2145044
:101B80001421C0F202001DF05DF920461CF0D0FACD
:101B900044F2B440C0F202000F211DF053F94EF29E
:101BA000C000C2F20000BDE8384019F0FBBD00BF24
:101BB000F8B541F2D443C2F2010305461B6801F5B2
:101BC000005644F698000C46013D1221C3F8C0604F
:101BD000C0F202001DF036F9E9B20F2915D841F61E
:101BE0009857C2F2010741F0E001B86C03681B6826
:101BF0009847B86C036806F07F011B689847B86C7B
:101C00000368C6F3C6111B68984744F2A44004F366
:101C10000D040F2104F50054C0F202001DF012F96A
:101C20002802230403F4FE0300F47060184340F418
:101C30006040640404F0FE4440F00E0020431CF0B9
:101C400077FA44F2B440C0F202000F211DF0FAF816
:101C50004EF2C000C2F20000BDE8F84019F0A2BD8B
:101C60004AF28853C2F2010310B41A68136850682C
:101C700019780478507A137A044201EA03011AD0E1
:101C8000937A03F0030309B143F0040343F008031C
:101C90009910082B91722AD8072B22D2032B2ED011
:101CA00011D9042B13D0062B14D1D3685DF8044B43
:101CB000023BD3607047937A03F003030029E7D017
:101CC00043F00403E4E7012B0BD0022B02D1D368CD
:101CD000013BD3605DF8044B70470D2BF7D00E2B02
:101CE000F8D1D3685DF8044B0133D36070470C2BF7
:101CF00005D0F2D8092BD8D00B2BE8D0EAE7D3686F
:101D00005DF8044B0233D360704700BF4AF288533A
:101D1000C2F2010310B49A68136850681978047805
:101D2000507A137A044201EA03011AD0937A03F03D
:101D3000030309B143F0040343F008039910082B8F
:101D400091722AD8072B22D2032B2ED011D9042B23
:101D500013D0062B14D1D3685DF8044B023BD3603B
:101D60007047937A03F003030029E7D043F004039C
:101D7000E4E7012B0BD0022B02D1D368013BD360E7
:101D80005DF8044B70470D2BF7D00E2BF8D1D368BC
:101D90005DF8044B0133D36070470C2B05D0F2D8AB
:101DA000092BD8D00B2BE8D0EAE7D3685DF8044BB9
:101DB0000233D360704700BF4AF28853C2F2010376
:101DC00010B4DA681368506819780478507A137A76
:101DD000044201EA03011AD0937A03F0030309B124
:101DE00043F0040343F008039910082B91722AD89A
:101DF000072B22D2032B2ED011D9042B13D0062B64
:101E000014D1D3685DF8044B023BD3607047937ADA
:101E100003F003030029E7D043F00403E4E7012BB8
:101E20000BD0022B02D1D368013BD3605DF8044B89
:101E300070470D2BF7D00E2BF8D1D3685DF8044B0B
:101E40000133D36070470C2B05D0F2D8092BD8D0C2
:101E50000B2BE8D0EAE7D3685DF8044B0233D3607C
:101E6000704700BF4AF28853C2F2010310B41A69E6
:101E70001368506819780478507A137A044201EA9A
:101E800003011AD0937A03F0030309B143F004036A
:101E900043F008039910082B91722AD8072B22D2FD
:101EA000032B2ED011D9042B13D0062B14D1D368B9
:101EB0005DF8044B023BD3607047937A03F0030351
:101EC0000029E7D043F00403E4E7012B0BD0022BF9
:101ED00002D1D368013BD3605DF8044B70470D2BF2
:101EE000F7D00E2BF8D1D3685DF8044B0133D360E3
:101EF00070470C2B05D0F2D8092BD8D00B2BE8D08B
:101F0000EAE7D3685DF8044B0233D360704700BF43
:101F10004AF28853C2F2010310B45A691368506838
:101F200019780478507A137A044201EA03011AD02E
:101F3000937A03F0030309B143F0040343F0080369
:101F40009910082B91722AD8072B22D2032B2ED05E
:101F500011D9042B13D0062B14D1D3685DF8044B90
:101F6000023BD3607047937A03F003030029E7D064
:101F700043F00403E4E7012B0BD0022B02D1D3681A
:101F8000013BD3605DF8044B70470D2BF7D00E2B4F
:101F9000F8D1D3685DF8044B0133D36070470C2B44
:101FA00005D0F2D8092BD8D00B2BE8D0EAE7D368BC
:101FB0005DF8044B0233D360704700BF4AF2885388
:101FC000C2F2010310B49A69136850681978047852
:101FD000507A137A044201EA03011AD0937A03F08B
:101FE000030309B143F0040343F008039910082BDD
:101FF00091722AD8072B22D2032B2ED011D9042B71
:1020000013D0062B14D1D3685DF8044B023BD36088
:102010007047937A03F003030029E7D043F00403E9
:10202000E4E7012B0BD0022B02D1D368013BD36034
:102030005DF8044B70470D2BF7D00E2BF8D1D36809
:102040005DF8044B0133D36070470C2B05D0F2D8F8
:10205000092BD8D00B2BE8D0EAE7D3685DF8044B06
:102060000233D360704700BF4AF28853C2F20103C3
:1020700010B4DA691368506819780478507A137AC2
:10208000044201EA03011AD0937A03F0030309B171
:1020900043F0040343F008039910082B91722AD8E7
:1020A000072B22D2032B2ED011D9042B13D0062BB1
:1020B00014D1D3685DF8044B023BD3607047937A28
:1020C00003F003030029E7D043F00403E4E7012B06
:1020D0000BD0022B02D1D368013BD3605DF8044BD7
:1020E00070470D2BF7D00E2BF8D1D3685DF8044B59
:1020F0000133D36070470C2B05D0F2D8092BD8D010
:102100000B2BE8D0EAE7D3685DF8044B0233D360C9
:10211000704700BF4AF28853C2F2010310B41A6A32
:102120001368506819780478507A137A044201EAE7
:1021300003011AD0937A03F0030309B143F00403B7
:1021400043F008039910082B91722AD8072B22D24A
:10215000032B2ED011D9042B13D0062B14D1D36806
:102160005DF8044B023BD3607047937A03F003039E
:102170000029E7D043F00403E4E7012B0BD0022B46
:1021800002D1D368013BD3605DF8044B70470D2B3F
:10219000F7D00E2BF8D1D3685DF8044B0133D36030
:1021A00070470C2B05D0F2D8092BD8D00B2BE8D0D8
:1021B000EAE7D3685DF8044B0233D360704700BF91
:1021C0004AF28853C2F2010310B45A6A1368506885
:1021D00019780478507A137A044201EA03011AD07C
:1021E000937A03F0030309B143F0040343F00803B7
:1021F0009910082B91722AD8072B22D2032B2ED0AC
:1022000011D9042B13D0062B14D1D3685DF8044BDD
:10221000023BD3607047937A03F003030029E7D0B1
:1022200043F00403E4E7012B0BD0022B02D1D36867
:10223000013BD3605DF8044B70470D2BF7D00E2B9C
:10224000F8D1D3685DF8044B0133D36070470C2B91
:1022500005D0F2D8092BD8D00B2BE8D0EAE7D36809
:102260005DF8044B0233D360704700BF4AF28853D5
:10227000C2F2010310B45A681368506819780478E0
:10228000507A137A044201EA03011AD0937A03F0D8
:10229000030309B143F0040343F008039910082B2A
:1022A00091722AD8072B22D2032B2ED011D9042BBE
:1022B00013D0062B14D1D3685DF8044B023BD360D6
:1022C0007047937A03F003030029E7D043F0040337
:1022D000E4E7012B0BD0022B02D1D368013BD36082
:1022E0005DF8044B70470D2BF7D00E2BF8D1D36857
:1022F0005DF8044B0133D36070470C2B05D0F2D846
:10230000092BD8D00B2BE8D0EAE7D3685DF8044B53
:102310000233D360704700BF4AF28853C2F2010310
:1023200010B4D3F8E8201368506819780478507A0C
:10233000137A044201EA03011AD0937A03F00303EB
:1023400009B143F0040343F008039910082B91727C
:102350002AD8072B22D2032B2ED011D9042B13D02D
:10236000062B14D1D3685DF8044B023BD360704751
:10237000937A03F003030029E7D043F00403E4E772
:10238000012B0BD0022B02D1D368013BD3605DF847
:10239000044B70470D2BF7D00E2BF8D1D3685DF8A6
:1023A000044B0133D36070470C2B05D0F2D8092BB6
:1023B000D8D00B2BE8D0EAE7D3685DF8044B0233A2
:1023C000D36070474AF28853C2F2010310B4D3F8C5
:1023D000EC201368506819780478507A137A044214
:1023E00001EA03011AD0937A03F0030309B143F021
:1023F000040343F008039910082B91722AD8072B85
:1024000022D2032B2ED011D9042B13D0062B14D19A
:10241000D3685DF8044B023BD3607047937A03F0B6
:1024200003030029E7D043F00403E4E7012B0BD0BA
:10243000022B02D1D368013BD3605DF8044B704797
:102440000D2BF7D00E2BF8D1D3685DF8044B013378
:10245000D36070470C2B05D0F2D8092BD8D00B2BAA
:10246000E8D0EAE7D3685DF8044B0233D3607047E5
:102470004AF28853C2F2010310B4D3F8A8201368BB
:10248000506819780478507A137A044201EA0301FB
:102490001AD0937A03F0030309B143F0040343F025
:1024A00008039910082B91722AD8072B22D2032BEC
:1024B0002ED011D9042B13D0062B14D1D3685DF87C
:1024C000044B023BD3607047937A03F00303002967
:1024D000E7D043F00403E4E7012B0BD0022B02D139
:1024E000D368013BD3605DF8044B70470D2BF7D0E8
:1024F0000E2BF8D1D3685DF8044B0133D3607047DD
:102500000C2B05D0F2D8092BD8D00B2BE8D0EAE75A
:10251000D3685DF8044B0233D36070474AF28853A6
:10252000C2F2010310B4D3F8AC20136850681978D4
:102530000478507A137A044201EA03011AD0937A9C
:1025400003F0030309B143F0040343F008039910B7
:10255000082B91722AD8072B22D2032B2ED011D907
:10256000042B13D0062B14D1D3685DF8044B023B27
:10257000D3607047937A03F003030029E7D043F058
:102580000403E4E7012B0BD0022B02D1D368013BFB
:10259000D3605DF8044B70470D2BF7D00E2BF8D1AC
:1025A000D3685DF8044B0133D36070470C2B05D022
:1025B000F2D8092BD8D00B2BE8D0EAE7D3685DF826
:1025C000044B0233D36070474AF28853C2F20103CE
:1025D00010B4D3F8B0201368506819780478507A92
:1025E000137A044201EA03011AD0937A03F0030339
:1025F00009B143F0040343F008039910082B9172CA
:102600002AD8072B22D2032B2ED011D9042B13D07A
:10261000062B14D1D3685DF8044B023BD36070479E
:10262000937A03F003030029E7D043F00403E4E7BF
:10263000012B0BD0022B02D1D368013BD3605DF894
:10264000044B70470D2BF7D00E2BF8D1D3685DF8F3
:10265000044B0133D36070470C2B05D0F2D8092B03
:10266000D8D00B2BE8D0EAE7D3685DF8044B0233EF
:10267000D36070474AF28853C2F2010310B4D3F812
:10268000B4201368506819780478507A137A044299
:1026900001EA03011AD0937A03F0030309B143F06E
:1026A000040343F008039910082B91722AD8072BD2
:1026B00022D2032B2ED011D9042B13D0062B14D1E8
:1026C000D3685DF8044B023BD3607047937A03F004
:1026D00003030029E7D043F00403E4E7012B0BD008
:1026E000022B02D1D368013BD3605DF8044B7047E5
:1026F0000D2BF7D00E2BF8D1D3685DF8044B0133C6
:10270000D36070470C2B05D0F2D8092BD8D00B2BF7
:10271000E8D0EAE7D3685DF8044B0233D360704732
:102720004AF28853C2F2010310B4D3F8B8201368F8
:10273000506819780478507A137A044201EA030148
:102740001AD0937A03F0030309B143F0040343F072
:1027500008039910082B91722AD8072B22D2032B39
:102760002ED011D9042B13D0062B14D1D3685DF8C9
:10277000044B023BD3607047937A03F003030029B4
:10278000E7D043F00403E4E7012B0BD0022B02D186
:10279000D368013BD3605DF8044B70470D2BF7D035
:1027A0000E2BF8D1D3685DF8044B0133D36070472A
:1027B0000C2B05D0F2D8092BD8D00B2BE8D0EAE7A8
:1027C000D3685DF8044B0233D36070474AF28853F4
:1027D000C2F2010310B4D3F8BC2013685068197812
:1027E0000478507A137A044201EA03011AD0937AEA
:1027F00003F0030309B143F0040343F00803991005
:10280000082B91722AD8072B22D2032B2ED011D954
:10281000042B13D0062B14D1D3685DF8044B023B74
:10282000D3607047937A03F003030029E7D043F0A5
:102830000403E4E7012B0BD0022B02D1D368013B48
:10284000D3605DF8044B70470D2BF7D00E2BF8D1F9
:10285000D3685DF8044B0133D36070470C2B05D06F
:10286000F2D8092BD8D00B2BE8D0EAE7D3685DF873
:10287000044B0233D36070474AF28853C2F201031B
:1028800010B4D3F8C0201368506819780478507ACF
:10289000137A044201EA03011AD0937A03F0030386
:1028A00009B143F0040343F008039910082B917217
:1028B0002AD8072B22D2032B2ED011D9042B13D0C8
:1028C000062B14D1D3685DF8044B023BD3607047EC
:1028D000937A03F003030029E7D043F00403E4E70D
:1028E000012B0BD0022B02D1D368013BD3605DF8E2
:1028F000044B70470D2BF7D00E2BF8D1D3685DF841
:10290000044B0133D36070470C2B05D0F2D8092B50
:10291000D8D00B2BE8D0EAE7D3685DF8044B02333C
:10292000D36070474AF28853C2F2010310B4D3F85F
:10293000C4201368506819780478507A137A0442D6
:1029400001EA03011AD0937A03F0030309B143F0BB
:10295000040343F008039910082B91722AD8072B1F
:1029600022D2032B2ED011D9042B13D0062B14D135
:10297000D3685DF8044B023BD3607047937A03F051
:1029800003030029E7D043F00403E4E7012B0BD055
:10299000022B02D1D368013BD3605DF8044B704732
:1029A0000D2BF7D00E2BF8D1D3685DF8044B013313
:1029B000D36070470C2B05D0F2D8092BD8D00B2B45
:1029C000E8D0EAE7D3685DF8044B0233D360704780
:1029D0004AF28853C2F2010310B4D3F8C820136836
:1029E000506819780478507A137A044201EA030196
:1029F0001AD0937A03F0030309B143F0040343F0C0
:102A000008039910082B91722AD8072B22D2032B86
:102A10002ED011D9042B13D0062B14D1D3685DF816
:102A2000044B023BD3607047937A03F00303002901
:102A3000E7D043F00403E4E7012B0BD0022B02D1D3
:102A4000D368013BD3605DF8044B70470D2BF7D082
:102A50000E2BF8D1D3685DF8044B0133D360704777
:102A60000C2B05D0F2D8092BD8D00B2BE8D0EAE7F5
:102A7000D3685DF8044B0233D36070474AF2885341
:102A8000C2F2010310B4D3F8CC201368506819784F
:102A90000478507A137A044201EA03011AD0937A37
:102AA00003F0030309B143F0040343F00803991052
:102AB000082B91722AD8072B22D2032B2ED011D9A2
:102AC000042B13D0062B14D1D3685DF8044B023BC2
:102AD000D3607047937A03F003030029E7D043F0F3
:102AE0000403E4E7012B0BD0022B02D1D368013B96
:102AF000D3605DF8044B70470D2BF7D00E2BF8D147
:102B0000D3685DF8044B0133D36070470C2B05D0BC
:102B1000F2D8092BD8D00B2BE8D0EAE7D3685DF8C0
:102B2000044B0233D36070474AF28853C2F2010368
:102B300010B4D3F8D0201368506819780478507A0C
:102B4000137A044201EA03011AD0937A03F00303D3
:102B500009B143F0040343F008039910082B917264
:102B60002AD8072B22D2032B2ED011D9042B13D015
:102B7000062B14D1D3685DF8044B023BD360704739
:102B8000937A03F003030029E7D043F00403E4E75A
:102B9000012B0BD0022B02D1D368013BD3605DF82F
:102BA000044B70470D2BF7D00E2BF8D1D3685DF88E
:102BB000044B0133D36070470C2B05D0F2D8092B9E
:102BC000D8D00B2BE8D0EAE7D3685DF8044B02338A
:102BD000D36070474AF28853C2F2010310B4D3F8AD
:102BE000D4201368506819780478507A137A044214
:102BF00001EA03011AD0937A03F0030309B143F009
:102C0000040343F008039910082B91722AD8072B6C
:102C100022D2032B2ED011D9042B13D0062B14D182
:102C2000D3685DF8044B023BD3607047937A03F09E
:102C300003030029E7D043F00403E4E7012B0BD0A2
:102C4000022B02D1D368013BD3605DF8044B70477F
:102C50000D2BF7D00E2BF8D1D3685DF8044B013360
:102C6000D36070470C2B05D0F2D8092BD8D00B2B92
:102C7000E8D0EAE7D3685DF8044B0233D3607047CD
:102C80004AF28853C2F2010310B4D3F8D820136873
:102C9000506819780478507A137A044201EA0301E3
:102CA0001AD0937A03F0030309B143F0040343F00D
:102CB00008039910082B91722AD8072B22D2032BD4
:102CC0002ED011D9042B13D0062B14D1D3685DF864
:102CD000044B023BD3607047937A03F0030300294F
:102CE000E7D043F00403E4E7012B0BD0022B02D121
:102CF000D368013BD3605DF8044B70470D2BF7D0D0
:102D00000E2BF8D1D3685DF8044B0133D3607047C4
:102D10000C2B05D0F2D8092BD8D00B2BE8D0EAE742
:102D2000D3685DF8044B0233D36070474AF288538E
:102D3000C2F2010310B4D3F8DC201368506819788C
:102D40000478507A137A044201EA03011AD0937A84
:102D500003F0030309B143F0040343F0080399109F
:102D6000082B91722AD8072B22D2032B2ED011D9EF
:102D7000042B13D0062B14D1D3685DF8044B023B0F
:102D8000D3607047937A03F003030029E7D043F040
:102D90000403E4E7012B0BD0022B02D1D368013BE3
:102DA000D3605DF8044B70470D2BF7D00E2BF8D194
:102DB000D3685DF8044B0133D36070470C2B05D00A
:102DC000F2D8092BD8D00B2BE8D0EAE7D3685DF80E
:102DD000044B0233D36070474AF28853C2F20103B6
:102DE00010B4D3F8E0201368506819780478507A4A
:102DF000137A044201EA03011AD0937A03F0030321
:102E000009B143F0040343F008039910082B9172B1
:102E10002AD8072B22D2032B2ED011D9042B13D062
:102E2000062B14D1D3685DF8044B023BD360704786
:102E3000937A03F003030029E7D043F00403E4E7A7
:102E4000012B0BD0022B02D1D368013BD3605DF87C
:102E5000044B70470D2BF7D00E2BF8D1D3685DF8DB
:102E6000044B0133D36070470C2B05D0F2D8092BEB
:102E7000D8D00B2BE8D0EAE7D3685DF8044B0233D7
:102E8000D36070474AF28853C2F2010310B4D3F8FA
:102E9000E4201368506819780478507A137A044251
:102EA00001EA03011AD0937A03F0030309B143F056
:102EB000040343F008039910082B91722AD8072BBA
:102EC00022D2032B2ED011D9042B13D0062B14D1D0
:102ED000D3685DF8044B023BD3607047937A03F0EC
:102EE00003030029E7D043F00403E4E7012B0BD0F0
:102EF000022B02D1D368013BD3605DF8044B7047CD
:102F00000D2BF7D00E2BF8D1D3685DF8044B0133AD
:102F1000D36070470C2B05D0F2D8092BD8D00B2BDF
:102F2000E8D0EAE7D3685DF8044B0233D36070471A
:102F30004AF28853C2F2010310B49A6A13685068C7
:102F400019780478507A137A044201EA03011AD0FE
:102F5000937A03F0030309B143F0040343F0080339
:102F60009910082B91722AD8072B22D2032B2ED02E
:102F700011D9042B13D0062B14D1D3685DF8044B60
:102F8000023BD3607047937A03F003030029E7D034
:102F900043F00403E4E7012B0BD0022B02D1D368EA
:102FA000013BD3605DF8044B70470D2BF7D00E2B1F
:102FB000F8D1D3685DF8044B0133D36070470C2B14
:102FC00005D0F2D8092BD8D00B2BE8D0EAE7D3688C
:102FD0005DF8044B0233D360704700BF4AF2885358
:102FE000C2F2010310B4DA6A1368506819780478E1
:102FF000507A137A044201EA03011AD0937A03F05B
:10300000030309B143F0040343F008039910082BAC
:1030100091722AD8072B22D2032B2ED011D9042B40
:1030200013D0062B14D1D3685DF8044B023BD36058
:103030007047937A03F003030029E7D043F00403B9
:10304000E4E7012B0BD0022B02D1D368013BD36004
:103050005DF8044B70470D2BF7D00E2BF8D1D368D9
:103060005DF8044B0133D36070470C2B05D0F2D8C8
:10307000092BD8D00B2BE8D0EAE7D3685DF8044BD6
:103080000233D360704700BF4AF28853C2F2010393
:1030900010B41A6B1368506819780478507A137A50
:1030A000044201EA03011AD0937A03F0030309B141
:1030B00043F0040343F008039910082B91722AD8B7
:1030C000072B22D2032B2ED011D9042B13D0062B81
:1030D00014D1D3685DF8044B023BD3607047937AF8
:1030E00003F003030029E7D043F00403E4E7012BD6
:1030F0000BD0022B02D1D368013BD3605DF8044BA7
:1031000070470D2BF7D00E2BF8D1D3685DF8044B28
:103110000133D36070470C2B05D0F2D8092BD8D0DF
:103120000B2BE8D0EAE7D3685DF8044B0233D36099
:10313000704700BF4AF28853C2F2010310B45A6BC1
:103140001368506819780478507A137A044201EAB7
:1031500003011AD0937A03F0030309B143F0040387
:1031600043F008039910082B91722AD8072B22D21A
:10317000032B2ED011D9042B13D0062B14D1D368D6
:103180005DF8044B023BD3607047937A03F003036E
:103190000029E7D043F00403E4E7012B0BD0022B16
:1031A00002D1D368013BD3605DF8044B70470D2B0F
:1031B000F7D00E2BF8D1D3685DF8044B0133D36000
:1031C00070470C2B05D0F2D8092BD8D00B2BE8D0A8
:1031D000EAE7D3685DF8044B0233D360704700BF61
:1031E0004AF28853C2F2010310B49A6B1368506814
:1031F00019780478507A137A044201EA03011AD04C
:10320000937A03F0030309B143F0040343F0080386
:103210009910082B91722AD8072B22D2032B2ED07B
:1032200011D9042B13D0062B14D1D3685DF8044BAD
:10323000023BD3607047937A03F003030029E7D081
:1032400043F00403E4E7012B0BD0022B02D1D36837
:10325000013BD3605DF8044B70470D2BF7D00E2B6C
:10326000F8D1D3685DF8044B0133D36070470C2B61
:1032700005D0F2D8092BD8D00B2BE8D0EAE7D368D9
:103280005DF8044B0233D360704700BF4AF28853A5
:10329000C2F2010310B4DA6B13685068197804782D
:1032A000507A137A044201EA03011AD0937A03F0A8
:1032B000030309B143F0040343F008039910082BFA
:1032C00091722AD8072B22D2032B2ED011D9042B8E
:1032D00013D0062B14D1D3685DF8044B023BD360A6
:1032E0007047937A03F003030029E7D043F0040307
:1032F000E4E7012B0BD0022B02D1D368013BD36052
:103300005DF8044B70470D2BF7D00E2BF8D1D36826
:103310005DF8044B0133D36070470C2B05D0F2D815
:10332000092BD8D00B2BE8D0EAE7D3685DF8044B23
:103330000233D360704700BF4AF28853C2F20103E0
:1033400010B41A6C1368506819780478507A137A9C
:10335000044201EA03011AD0937A03F0030309B18E
:1033600043F0040343F008039910082B91722AD804
:10337000072B22D2032B2ED011D9042B13D0062BCE
:1033800014D1D3685DF8044B023BD3607047937A45
:1033900003F003030029E7D043F00403E4E7012B23
:1033A0000BD0022B02D1D368013BD3605DF8044BF4
:1033B00070470D2BF7D00E2BF8D1D3685DF8044B76
:1033C0000133D36070470C2B05D0F2D8092BD8D02D
:1033D0000B2BE8D0EAE7D3685DF8044B0233D360E7
:1033E000704700BF4AF28853C2F2010310B45A6C0E
:1033F0001368506819780478507A137A044201EA05
:1034000003011AD0937A03F0030309B143F00403D4
:1034100043F008039910082B91722AD8072B22D267
:10342000032B2ED011D9042B13D0062B14D1D36823
:103430005DF8044B023BD3607047937A03F00303BB
:103440000029E7D043F00403E4E7012B0BD0022B63
:1034500002D1D368013BD3605DF8044B70470D2B5C
:10346000F7D00E2BF8D1D3685DF8044B0133D3604D
:1034700070470C2B05D0F2D8092BD8D00B2BE8D0F5
:10348000EAE7D3685DF8044B0233D360704700BFAE
:103490004AF28853C2F2010310B49A6C1368506860
:1034A00019780478507A137A044201EA03011AD099
:1034B000937A03F0030309B143F0040343F00803D4
:1034C0009910082B91722AD8072B22D2032B2ED0C9
:1034D00011D9042B13D0062B14D1D3685DF8044BFB
:1034E000023BD3607047937A03F003030029E7D0CF
:1034F00043F00403E4E7012B0BD0022B02D1D36885
:10350000013BD3605DF8044B70470D2BF7D00E2BB9
:10351000F8D1D3685DF8044B0133D36070470C2BAE
:1035200005D0F2D8092BD8D00B2BE8D0EAE7D36826
:103530005DF8044B0233D360704700BF4AF28853F2
:10354000C2F2010310B4DA6C136850681978047879
:10355000507A137A044201EA03011AD0937A03F0F5
:10356000030309B143F0040343F008039910082B47
:1035700091722AD8072B22D2032B2ED011D9042BDB
:1035800013D0062B14D1D3685DF8044B023BD360F3
:103590007047937A03F003030029E7D043F0040354
:1035A000E4E7012B0BD0022B02D1D368013BD3609F
:1035B0005DF8044B70470D2BF7D00E2BF8D1D36874
:1035C0005DF8044B0133D36070470C2B05D0F2D863
:1035D000092BD8D00B2BE8D0EAE7D3685DF8044B71
:1035E0000233D360704700BF4AF28853C2F201032E
:1035F00010B41A6D1368506819780478507A137AE9
:10360000044201EA03011AD0937A03F0030309B1DB
:1036100043F0040343F008039910082B91722AD851
:10362000072B22D2032B2ED011D9042B13D0062B1B
:1036300014D1D3685DF8044B023BD3607047937A92
:1036400003F003030029E7D043F00403E4E7012B70
:103650000BD0022B02D1D368013BD3605DF8044B41
:1036600070470D2BF7D00E2BF8D1D3685DF8044BC3
:103670000133D36070470C2B05D0F2D8092BD8D07A
:103680000B2BE8D0EAE7D3685DF8044B0233D36034
:10369000704700BF4AF28853C2F2010310B45A6D5A
:1036A0001368506819780478507A137A044201EA52
:1036B00003011AD0937A03F0030309B143F0040322
:1036C00043F008039910082B91722AD8072B22D2B5
:1036D000032B2ED011D9042B13D0062B14D1D36871
:1036E0005DF8044B023BD3607047937A03F0030309
:1036F0000029E7D043F00403E4E7012B0BD0022BB1
:1037000002D1D368013BD3605DF8044B70470D2BA9
:10371000F7D00E2BF8D1D3685DF8044B0133D3609A
:1037200070470C2B05D0F2D8092BD8D00B2BE8D042
:10373000EAE7D3685DF8044B0233D360704700BFFB
:103740004AF28853C2F2010310B49A6D13685068AC
:1037500019780478507A137A044201EA03011AD0E6
:10376000937A03F0030309B143F0040343F0080321
:103770009910082B91722AD8072B22D2032B2ED016
:1037800011D9042B13D0062B14D1D3685DF8044B48
:10379000023BD3607047937A03F003030029E7D01C
:1037A00043F00403E4E7012B0BD0022B02D1D368D2
:1037B000013BD3605DF8044B70470D2BF7D00E2B07
:1037C000F8D1D3685DF8044B0133D36070470C2BFC
:1037D00005D0F2D8092BD8D00B2BE8D0EAE7D36874
:1037E0005DF8044B0233D360704700BF4AF2885340
:1037F000C2F2010310B4DA6D1368506819780478C6
:10380000507A137A044201EA03011AD0937A03F042
:10381000030309B143F0040343F008039910082B94
:1038200091722AD8072B22D2032B2ED011D9042B28
:1038300013D0062B14D1D3685DF8044B023BD36040
:103840007047937A03F003030029E7D043F00403A1
:10385000E4E7012B0BD0022B02D1D368013BD360EC
:103860005DF8044B70470D2BF7D00E2BF8D1D368C1
:103870005DF8044B0133D36070470C2B05D0F2D8B0
:10388000092BD8D00B2BE8D0EAE7D3685DF8044BBE
:103890000233D360704700BF4AF28853C2F201037B
:1038A00010B41A6E1368506819780478507A137A35
:1038B000044201EA03011AD0937A03F0030309B129
:1038C00043F0040343F008039910082B91722AD89F
:1038D000072B22D2032B2ED011D9042B13D0062B69
:1038E00014D1D3685DF8044B023BD3607047937AE0
:1038F00003F003030029E7D043F00403E4E7012BBE
:103900000BD0022B02D1D368013BD3605DF8044B8E
:1039100070470D2BF7D00E2BF8D1D3685DF8044B10
:103920000133D36070470C2B05D0F2D8092BD8D0C7
:103930000B2BE8D0EAE7D3685DF8044B0233D36081
:10394000704700BF4AF28853C2F2010310B45A6EA6
:103950001368506819780478507A137A044201EA9F
:1039600003011AD0937A03F0030309B143F004036F
:1039700043F008039910082B91722AD8072B22D202
:10398000032B2ED011D9042B13D0062B14D1D368BE
:103990005DF8044B023BD3607047937A03F0030356
:1039A0000029E7D043F00403E4E7012B0BD0022BFE
:1039B00002D1D368013BD3605DF8044B70470D2BF7
:1039C000F7D00E2BF8D1D3685DF8044B0133D360E8
:1039D00070470C2B05D0F2D8092BD8D00B2BE8D090
:1039E000EAE7D3685DF8044B0233D360704700BF49
:1039F0004AF28853C2F2010310B49A6E13685068F9
:103A000019780478507A137A044201EA03011AD033
:103A1000937A03F0030309B143F0040343F008036E
:103A20009910082B91722AD8072B22D2032B2ED063
:103A300011D9042B13D0062B14D1D3685DF8044B95
:103A4000023BD3607047937A03F003030029E7D069
:103A500043F00403E4E7012B0BD0022B02D1D3681F
:103A6000013BD3605DF8044B70470D2BF7D00E2B54
:103A7000F8D1D3685DF8044B0133D36070470C2B49
:103A800005D0F2D8092BD8D00B2BE8D0EAE7D368C1
:103A90005DF8044B0233D360704700BF4AF288538D
:103AA000C2F2010310B4DA6E136850681978047812
:103AB000507A137A044201EA03011AD0937A03F090
:103AC000030309B143F0040343F008039910082BE2
:103AD00091722AD8072B22D2032B2ED011D9042B76
:103AE00013D0062B14D1D3685DF8044B023BD3608E
:103AF0007047937A03F003030029E7D043F00403EF
:103B0000E4E7012B0BD0022B02D1D368013BD36039
:103B10005DF8044B70470D2BF7D00E2BF8D1D3680E
:103B20005DF8044B0133D36070470C2B05D0F2D8FD
:103B3000092BD8D00B2BE8D0EAE7D3685DF8044B0B
:103B40000233D360704700BF4AF28853C2F20103C8
:103B500010B41A6F1368506819780478507A137A81
:103B6000044201EA03011AD0937A03F0030309B176
:103B700043F0040343F008039910082B91722AD8EC
:103B8000072B22D2032B2ED011D9042B13D0062BB6
:103B900014D1D3685DF8044B023BD3607047937A2D
:103BA00003F003030029E7D043F00403E4E7012B0B
:103BB0000BD0022B02D1D368013BD3605DF8044BDC
:103BC00070470D2BF7D00E2BF8D1D3685DF8044B5E
:103BD0000133D36070470C2B05D0F2D8092BD8D015
:103BE0000B2BE8D0EAE7D3685DF8044B0233D360CF
:103BF000704700BF4AF28853C2F2010310B45A6FF3
:103C00001368506819780478507A137A044201EAEC
:103C100003011AD0937A03F0030309B143F00403BC
:103C200043F008039910082B91722AD8072B22D24F
:103C3000032B2ED011D9042B13D0062B14D1D3680B
:103C40005DF8044B023BD3607047937A03F00303A3
:103C50000029E7D043F00403E4E7012B0BD0022B4B
:103C600002D1D368013BD3605DF8044B70470D2B44
:103C7000F7D00E2BF8D1D3685DF8044B0133D36035
:103C800070470C2B05D0F2D8092BD8D00B2BE8D0DD
:103C9000EAE7D3685DF8044B0233D360704700BF96
:103CA0004AF28853C2F2010310B49A6F1368506845
:103CB00019780478507A137A044201EA03011AD081
:103CC000937A03F0030309B143F0040343F00803BC
:103CD0009910082B91722AD8072B22D2032B2ED0B1
:103CE00011D9042B13D0062B14D1D3685DF8044BE3
:103CF000023BD3607047937A03F003030029E7D0B7
:103D000043F00403E4E7012B0BD0022B02D1D3686C
:103D1000013BD3605DF8044B70470D2BF7D00E2BA1
:103D2000F8D1D3685DF8044B0133D36070470C2B96
:103D300005D0F2D8092BD8D00B2BE8D0EAE7D3680E
:103D40005DF8044B0233D360704700BF4AF28853DA
:103D5000C2F2010310B4DA6F13685068197804785E
:103D6000507A137A044201EA03011AD0937A03F0DD
:103D7000030309B143F0040343F008039910082B2F
:103D800091722AD8072B22D2032B2ED011D9042BC3
:103D900013D0062B14D1D3685DF8044B023BD360DB
:103DA0007047937A03F003030029E7D043F004033C
:103DB000E4E7012B0BD0022B02D1D368013BD36087
:103DC0005DF8044B70470D2BF7D00E2BF8D1D3685C
:103DD0005DF8044B0133D36070470C2B05D0F2D84B
:103DE000092BD8D00B2BE8D0EAE7D3685DF8044B59
:103DF0000233D360704700BF4AF28853C2F2010316
:103E000010B4D3F880201368506819780478507A79
:103E1000137A044201EA03011AD0937A03F00303F0
:103E200009B143F0040343F008039910082B917281
:103E30002AD8072B22D2032B2ED011D9042B13D032
:103E4000062B14D1D3685DF8044B023BD360704756
:103E5000937A03F003030029E7D043F00403E4E777
:103E6000012B0BD0022B02D1D368013BD3605DF84C
:103E7000044B70470D2BF7D00E2BF8D1D3685DF8AB
:103E8000044B0133D36070470C2B05D0F2D8092BBB
:103E9000D8D00B2BE8D0EAE7D3685DF8044B0233A7
:103EA000D36070474AF28853C2F2010310B4D3F8CA
:103EB00084201368506819780478507A137A044281
:103EC00001EA03011AD0937A03F0030309B143F026
:103ED000040343F008039910082B91722AD8072B8A
:103EE00022D2032B2ED011D9042B13D0062B14D1A0
:103EF000D3685DF8044B023BD3607047937A03F0BC
:103F000003030029E7D043F00403E4E7012B0BD0BF
:103F1000022B02D1D368013BD3605DF8044B70479C
:103F20000D2BF7D00E2BF8D1D3685DF8044B01337D
:103F3000D36070470C2B05D0F2D8092BD8D00B2BAF
:103F4000E8D0EAE7D3685DF8044B0233D3607047EA
:103F50004AF28853C2F2010310B4D3F888201368E0
:103F6000506819780478507A137A044201EA030100
:103F70001AD0937A03F0030309B143F0040343F02A
:103F800008039910082B91722AD8072B22D2032BF1
:103F90002ED011D9042B13D0062B14D1D3685DF881
:103FA000044B023BD3607047937A03F0030300296C
:103FB000E7D043F00403E4E7012B0BD0022B02D13E
:103FC000D368013BD3605DF8044B70470D2BF7D0ED
:103FD0000E2BF8D1D3685DF8044B0133D3607047E2
:103FE0000C2B05D0F2D8092BD8D00B2BE8D0EAE760
:103FF000D3685DF8044B0233D36070474AF28853AC
:10400000C2F2010310B4D3F88C20136850681978F9
:104010000478507A137A044201EA03011AD0937AA1
:1040200003F0030309B143F0040343F008039910BC
:10403000082B91722AD8072B22D2032B2ED011D90C
:10404000042B13D0062B14D1D3685DF8044B023B2C
:10405000D3607047937A03F003030029E7D043F05D
:104060000403E4E7012B0BD0022B02D1D368013B00
:10407000D3605DF8044B70470D2BF7D00E2BF8D1B1
:10408000D3685DF8044B0133D36070470C2B05D027
:10409000F2D8092BD8D00B2BE8D0EAE7D3685DF82B
:1040A000044B0233D36070474AF28853C2F20103D3
:1040B00010B4D3F890201368506819780478507AB7
:1040C000137A044201EA03011AD0937A03F003033E
:1040D00009B143F0040343F008039910082B9172CF
:1040E0002AD8072B22D2032B2ED011D9042B13D080
:1040F000062B14D1D3685DF8044B023BD3607047A4
:10410000937A03F003030029E7D043F00403E4E7C4
:10411000012B0BD0022B02D1D368013BD3605DF899
:10412000044B70470D2BF7D00E2BF8D1D3685DF8F8
:10413000044B0133D36070470C2B05D0F2D8092B08
:10414000D8D00B2BE8D0EAE7D3685DF8044B0233F4
:10415000D36070474AF28853C2F2010310B4D3F817
:1041600094201368506819780478507A137A0442BE
:1041700001EA03011AD0937A03F0030309B143F073
:10418000040343F008039910082B91722AD8072BD7
:1041900022D2032B2ED011D9042B13D0062B14D1ED
:1041A000D3685DF8044B023BD3607047937A03F009
:1041B00003030029E7D043F00403E4E7012B0BD00D
:1041C000022B02D1D368013BD3605DF8044B7047EA
:1041D0000D2BF7D00E2BF8D1D3685DF8044B0133CB
:1041E000D36070470C2B05D0F2D8092BD8D00B2BFD
:1041F000E8D0EAE7D3685DF8044B0233D360704738
:104200004AF28853C2F2010310B4D3F8982013681D
:10421000506819780478507A137A044201EA03014D
:104220001AD0937A03F0030309B143F0040343F077
:1042300008039910082B91722AD8072B22D2032B3E
:104240002ED011D9042B13D0062B14D1D3685DF8CE
:10425000044B023BD3607047937A03F003030029B9
:10426000E7D043F00403E4E7012B0BD0022B02D18B
:10427000D368013BD3605DF8044B70470D2BF7D03A
:104280000E2BF8D1D3685DF8044B0133D36070472F
:104290000C2B05D0F2D8092BD8D00B2BE8D0EAE7AD
:1042A000D3685DF8044B0233D36070474AF28853F9
:1042B000C2F2010310B4D3F89C2013685068197837
:1042C0000478507A137A044201EA03011AD0937AEF
:1042D00003F0030309B143F0040343F0080399100A
:1042E000082B91722AD8072B22D2032B2ED011D95A
:1042F000042B13D0062B14D1D3685DF8044B023B7A
:10430000D3607047937A03F003030029E7D043F0AA
:104310000403E4E7012B0BD0022B02D1D368013B4D
:10432000D3605DF8044B70470D2BF7D00E2BF8D1FE
:10433000D3685DF8044B0133D36070470C2B05D074
:10434000F2D8092BD8D00B2BE8D0EAE7D3685DF878
:10435000044B0233D36070474AF28853C2F2010320
:1043600010B4D3F8A0201368506819780478507AF4
:10437000137A044201EA03011AD0937A03F003038B
:1043800009B143F0040343F008039910082B91721C
:104390002AD8072B22D2032B2ED011D9042B13D0CD
:1043A000062B14D1D3685DF8044B023BD3607047F1
:1043B000937A03F003030029E7D043F00403E4E712
:1043C000012B0BD0022B02D1D368013BD3605DF8E7
:1043D000044B70470D2BF7D00E2BF8D1D3685DF846
:1043E000044B0133D36070470C2B05D0F2D8092B56
:1043F000D8D00B2BE8D0EAE7D3685DF8044B023342
:10440000D36070474AF28853C2F2010310B4D3F864
:10441000A4201368506819780478507A137A0442FB
:1044200001EA03011AD0937A03F0030309B143F0C0
:10443000040343F008039910082B91722AD8072B24
:1044400022D2032B2ED011D9042B13D0062B14D13A
:10445000D3685DF8044B023BD3607047937A03F056
:1044600003030029E7D043F00403E4E7012B0BD05A
:10447000022B02D1D368013BD3605DF8044B704737
:104480000D2BF7D00E2BF8D1D3685DF8044B013318
:10449000D36070470C2B05D0F2D8092BD8D00B2B4A
:1044A000E8D0EAE7D3685DF8044B0233D360704785
:1044B000F8B54DF63857C2F2000704463B7C0E466D
:1044C00015467BB398422DD044F2E0501E21C0F235
:1044D00002001AF0B7FC4EF2C00000230A22214667
:1044E000C2F2000017F070F944F200600E21C0F231
:1044F00002001AF0A7FC4EF2C000397C00230A2209
:10450000C2F2000017F060F944F210600121C0F21D
:1045100002001AF097FC4EF2C000C2F2000017F041
:1045200041F907E041F2D443C2F201033146186871
:104530000AF036FE44F6AC001221013CC0F2020043
:104540001AF080FCE1B20F2915D841F69857C2F253
:10455000010741F08001B86C03681B689847B86C8C
:10456000036806F07F011B689847B86C036805F084
:104570007F011B68984744F2A4400F21C0F202005B
:104580001AF060FC2B0603F0FE43310443F40043B1
:1045900043F0080301F4FE012402194304F470649B
:1045A00041F2E0402143C2F2010015F031FC44F237
:1045B0001450C0F2020014211AF044FC4EF2C00064
:1045C000C2F20000BDE8F84017F0ECB8F8B54DF6BF
:1045D0003857C2F2000704463B7C0E4615467BB3B3
:1045E00098422DD044F2E0501E21C0F202001AF091
:1045F00029FC4EF2C00000230A222146C2F200002C
:1046000017F0E2F844F200600E21C0F202001AF046
:1046100019FC4EF2C000397C00230A22C2F20000CD
:1046200017F0D2F844F210600121C0F202001AF033
:1046300009FC4EF2C000C2F2000017F0B3F808E027
:1046400041F2D443C2F201032A46186831460AF007
:1046500067FB44F6C0001121013CC0F202001AF0D1
:10466000F1FBE1B20F2915D841F69857C2F20107C4
:1046700041F09001B86C03681B689847B86C0368F8
:1046800006F07F011B689847B86C036805F07F014E
:104690001B68984744F2A4400F21C0F202001AF0B0
:1046A000D1FB2B0603F0FE43310443F4104343F0E7
:1046B000090301F4FE012402194304F4706441F279
:1046C000E0402143C2F2010015F0A2FB44F2145075
:1046D000C0F2020014211AF0B5FB4EF2C000C2F283
:1046E0000000BDE8F84017F05DB800BFF8B54DF622
:1046F0003857C2F2000704463B7C0E4615467BB392
:1047000098422DD044F2E0501E21C0F202001AF06F
:1047100099FB4EF2C00000230A222146C2F200009B
:1047200017F052F844F200600E21C0F202001AF0B5
:1047300089FB4EF2C000397C00230A22C2F200003D
:1047400017F042F844F210600121C0F202001AF0A2
:1047500079FB4EF2C000C2F2000017F023F807E028
:1047600041F2D443C2F20103314618680AF018FD41
:1047700044F6D4001721013CC0F202001AF062FB9B
:10478000E1B20F2915D841F69857C2F2010741F05E
:104790008001B86C03681B689847B86C036806F022
:1047A0007F011B689847B86C036805F07F011B68A0
:1047B000984744F2A4400F21C0F202001AF042FBD5
:1047C0002B0603F0FE43300443F4004343F0080398
:1047D00000F4FE002402184304F47064204319F02E
:1047E000A7FC44F2B440C0F202000F211AF02AFBE9
:1047F0004EF2C000C2F20000BDE8F84016F0D2BF91
:10480000F8B54DF63857C2F2000704463B7C0E4619
:1048100015467BB398422DD044F2E0501E21C0F2E1
:1048200002001AF00FFB4EF2C00000230A222146BC
:10483000C2F2000016F0C8FF44F200600E21C0F280
:1048400002001AF0FFFA4EF2C000397C00230A225F
:10485000C2F2000016F0B8FF44F210600121C0F26D
:1048600002001AF0EFFA4EF2C000C2F2000016F099
:1048700099FF08E041F2D443C2F201032A461868C6
:1048800031460AF04DFA44F6EC001621013CC0F224
:1048900002001AF0D7FAE1B20F2915D841F698575D
:1048A000C2F2010741F09001B86C03681B68984799
:1048B000B86C036806F07F011B689847B86C036802
:1048C00005F07F011B68984744F2A4400F21C0F215
:1048D00002001AF0B7FA2B0603F0FE43300443F44B
:1048E000104343F0090300F4FE002402184304F4CB
:1048F0007064204319F01CFC44F2B440C0F2020082
:104900000F211AF09FFA4EF2C000C2F20000BDE87B
:10491000F84016F047BF00BF10B444F21044002323
:10492000C0F202044172026104600372C36041B1CB
:10493000194600E0026942F82310427A01339A4294
:10494000F8DC4AF28863C2F201031A680AB90CE083
:104950001A465369002BFBD15061002343618380C9
:10496000C38083725DF8044B70471860F5E700BFA1
:10497000F8B541F69854C2F2010447F61221A06C32
:104980000368DB69984741F68507032041F6211348
:1049900046F2097144F65D6641F6213284F86400FE
:1049A000C0F20003C0F20007C0F20001C0F200062E
:1049B000C0F2000241F2197063602760E160666135
:1049C000A261C0F2000045F6754340F6056741F26A
:1049D0009D7140F6F53640F6C1222061C0F2000319
:1049E000C0F20007C0F20001C0F20006C0F20002EF
:1049F00041F23D40E3612762A160A662E262C0F23B
:104A0000000040F6515340F6554740F6A94140F6A4
:104A1000FD4641F24102C0F200022063C0F20003F1
:104A2000C0F20007C0F20001C0F200064EF2C0055D
:104A300044F604106264C2F200056363A7630023B6
:104A40004FF6FF77E16326641721C0F2020084F875
:104A50004C3084F84E3084F84D30A365636584F89B
:104A6000E93084F8663084F8653084F8673084F87B
:104A70006830E76527661AF0E5F9284616F092FED9
:104A800013F096FB41F2E043C2F2010344F6010148
:104A900044F2ED6746F2516644F6E16441F6B13204
:104AA000C0F20001C0F20007C0F20006C0F200042C
:104AB000C0F2000241F2D950C3F86811C3F8647122
:104AC000C3F87061C3F87841C3F87C21C0F20000DC
:104AD00045F6D54141F6392741F2716641F6150494
:104AE00040F6E972C3F87401C0F20001C0F2000799
:104AF000C0F20006C0F20004C0F2000241F2C14060
:104B0000C3F88411C3F88871C3F86C61C3F890418D
:104B1000C3F89421C0F2000040F6153140F6B917F1
:104B200040F6112640F6692440F66D32C0F20002CC
:104B3000C3F89801C0F20001C0F20007C0F20006FD
:104B4000C0F2000444F61C10C3F89C11C3F8A07115
:104B5000C3F8A461C3F8A841C3F8AC211D21C0F279
:104B600002001AF06FF9284616F01CFE4AF62811CA
:104B7000C2F2010144F2CD5EC0F2000E4AF62014EA
:104B8000C1F800E0C2F2010444F2B14EC0F2000EDE
:104B90004AF62413C4F800E0C2F2010346F23D5E77
:104BA000C0F2000E4AF6F807C3F800E0C2F20107AF
:104BB00044F6797EC0F2000E4AF6E800C7F800E03D
:104BC000C2F2010041F2552EC0F2000E4AF6E40690
:104BD000C0F800E0C2F2010641F20D3EC0F2000E44
:104BE0004AF60812C6F800E0C2F2010245F6595E24
:104BF000C0F2000E4AF60011C2F800E0C2F2010154
:104C000041F6A92EC0F2000E4AF6F404C1F800E005
:104C1000C2F2010441F2B51EC0F2000E4AF61C13A6
:104C2000C4F800E0C2F2010341F6C11EC0F2000E5A
:104C30004AF60417C3F800E0C2F2010741F2551E1C
:104C4000C0F2000E4AF6CC00C7F800E0C2F2010044
:104C500041F24957C0F200074AF6FC060760C2F26B
:104C600001064AF6DC0240F66967C2F20102C0F2B0
:104C700000074AF6141140F6C9603760C2F201011C
:104C8000C0F200004AF6D4044AF6D00340F6297771
:104C9000C2F201031060C2F20104C0F2000740F644
:104CA000897641F2C50244F63C100F60C0F200065E
:104CB000C0F20002C0F20200182126601A601AF049
:104CC000C1F82846BDE8F84016F06CBD4DF20A73F5
:104CD000C3F6234306EE103A437EC17E07EE103A38
:104CE000837CB8EEC77A07EE903A70B4F8EEE76AC4
:104CF00027EE067A83B067EE267A0022FCEEE77A8A
:104D00008273CDED017A42739DF80430027301B1D4
:104D10000373827E02B14373027F02B1837390F802
:104D2000213090F8231007EE103A4DF20A73C3F6C3
:104D3000234306EE103A037CB8EEC77A07EE903AAA
:104D400027EE067AF8EEE76A67EE267AFCEEE77A57
:104D5000CDED017A9DF8043021B1017B994238BF35
:104D60001946017390F8221021B1417B994238BF56
:104D70001946417390F8244024B1817B8B4238BF9F
:104D80000B468373437FC17F07EE103A4DF20A73DF
:104D9000C3F6234306EE103A437CB8EEC77A07EE1B
:104DA000903A27EE067AF8EEE76A67EE267AFCEE8E
:104DB000E77ACDED017A9DF8043021B1017B99426B
:104DC00038BF19460173817F21B1417B994238BFB9
:104DD0001946417390F8201021B1857BAB4238BF52
:104DE0002B46837390F8253090F8275007EE103A41
:104DF0004DF20A73C3F6234306EE103AC37BB8EEB6
:104E0000C77A07EE903A27EE067AF8EEE76A67EE81
:104E1000267AFCEEE77ACDED017A9DF8043025B1D3
:104E2000057B9D4238BF1D46057390F8265025B17D
:104E3000457B9D4238BF1D46457390F8285025B1EB
:104E4000867BB34238BF3346837322B919B914B98C
:104E50000DB97F23837303B070BC704738B541F23E
:104E6000D443C2F201030C461B680546240483F8B0
:104E7000CF1003F1C00004F4FE04013DFFF726FF4C
:104E800044F4504444F658102D020D2105F4706589
:104E9000C0F2020044F00D0419F0D4FF2C4341F29B
:104EA000E0402146C2F2010014F0B2FF44F2145077
:104EB0001421C0F2020019F0C5FF204619F038F99C
:104EC00044F2B440C0F202000F2119F0BBFF4EF2D1
:104ED000C000C2F20000BDE8384016F063BC00BF5D
:104EE00041F2D443C2F2010370B51B68054683F852
:104EF000CF1003F1C0000C46FFF7E8FE44F668103F
:104F00001221013DC0F2020019F09CFFE9B20F2905
:104F10000FD841F69856C2F2010641F0D001B06CAC
:104F200003681B689847B06C036804F07F011B6836
:104F3000984744F2A4400F21C0F2020019F082FF0A
:104F4000230403F4FE03280243F4504343F00D030B
:104F500000F47060184319F0EBF844F2B440C0F26A
:104F600002000F2119F06EFF4EF2C000C2F20000E5
:104F7000BDE8704016F016BC41F2D443C2F2010302
:104F800070B51B68054683F8CF1003F1C0000C46CE
:104F9000FFF79CFE44F67C100D21013DC0F202009B
:104FA00019F050FFE9B20F290FD841F69856C2F216
:104FB000010641F0D001B06C03681B689847B06CE3
:104FC000036804F07F011B68984744F2A4400F2156
:104FD000C0F2020019F036FF230403F4FE03290295
:104FE00043F4504343F00D0301F4706141F2E0409B
:104FF0001943C2F2010014F00BFF44F21450C0F246
:105000000200142119F01EFF4EF2C000C2F200008F
:10501000BDE8704016F0C6BB10B4036841681A784A
:105020000C78417A037A0C4202EA03021AD0837A9E
:1050300003F003030AB143F0040343F008039A109A
:10504000082B82722AD8072B22D2032B2ED011D9FB
:10505000042B13D0062B14D1C3685DF8044B023B1C
:10506000C3607047837A03F00303002AE7D043F05C
:105070000403E4E7012B0BD0022B02D1C368013BF0
:10508000C3605DF8044B70470D2BF7D00E2BF8D1A1
:10509000C3685DF8044B0133C36070470C2B05D027
:1050A000F2D8092BD8D00B2BE8D0EAE7C3685DF81B
:1050B000044B0233C36070471D2810B50B4600F047
:1050C000E983024622D92C2800F064813FD82428A5
:1050D00000F0EE8340F2A880282800F0748300F2EC
:1050E000D680262800F0F58140F2D5824AF2885415
:1050F000C2F2010444F2AD21C0F2000104222720D3
:10510000C4F89C3017F0B6F8012010BD0E2800F04E
:1051100097833AD8062800F0A1836CD90A2800F0BA
:10512000058300F20781082800F07E8140F2758235
:105130004AF28854C2F2010442F2C111C0F20001E5
:1051400004220920636217F095F8012010BD34286D
:1051500000F0BD8336D8302800F0638300F2D6809B
:105160002E2800F0528140F201824AF28854C2F2A5
:10517000010442F2CD71C0F2000104222F20C4F8D4
:10518000BC3017F077F8012010BD152800F07483AB
:1051900064D9192800F0FA8100F2A580172800F0E0
:1051A0008A8140F2D1824AF28854C2F2010443F665
:1051B0009901C0F2000104221820236617F05AF862
:1051C000012010BD382800F0CE8275D8362800F0B6
:1051D000398140F27F824AF28854C2F2010442F6D9
:1051E0002D51C0F2000104223720C4F8DC3017F042
:1051F00041F8012010BD022800F0018240F27881C0
:10520000042800F04B8140F2BD824AF28854C2F279
:10521000010441F61171C0F200010422052063610E
:1052200017F028F8012010BD202800F0448240F239
:105230008981222800F0238140F2D4824AF28854E6
:10524000C2F2010443F6FD71C0F2000104222320E2
:10525000C4F88C3017F00EF8012010BD112800F0B2
:10526000B18140F25A81132800F0FB8040F2B881EE
:105270004AF28854C2F2010443F2E951C0F200013B
:1052800004221420236516F0F5FF012010BD2A2802
:1052900000F0AC8040F2E0814AF28854C2F201048E
:1052A00042F21D51C0F2000104222B20C4F8AC30A0
:1052B00016F0E0FF012010BD3A2800F08880C0F011
:1052C00072823B2840F06D824AF28854C2F2010497
:1052D00042F2C531C0F200010422C4F8EC3016F0ED
:1052E000C9FF012010BD1B2863D040F28B824AF217
:1052F0008854C2F2010443F64931C0F2000104228D
:105300001C20236716F0B6FF012010BD322824D0E0
:1053100040F292814AF28854C2F2010442F67D21A1
:10532000C0F2000104223320C4F8CC3016F0A2FFF2
:10533000012010BD0C281FD040F29E814AF28854F3
:10534000C2F2010443F23511C0F2000104220D2023
:10535000636316F08FFF012010BD4AF28854C2F239
:10536000010442F6D111C0F200010422C4F8C83091
:1053700016F080FF012010BD4AF28854C2F20104E9
:1053800043F28901C0F200010422236316F072FF88
:10539000012010BD4AF28854C2F2010442F2C95100
:1053A000C0F200010422C4F8B03016F063FF0120FF
:1053B00010BD4AF28854C2F2010443F69D21C0F2A6
:1053C00000010422E36616F055FF012010BD4AF2E9
:1053D0008854C2F2010442F21931C0F200010422E1
:1053E000C4F8E83016F046FF012010BD4AF2885498
:1053F000C2F2010442F27141C0F200010422C4F879
:10540000A83016F037FF012010BD4AF28854C2F2CE
:10541000010442F22171C0F200010422C4F8B83044
:1054200016F028FF012010BD4AF28854C2F2010490
:1054300042F21511C0F200010422236216F01AFF95
:10544000012010BD4AF28854C2F2010442F68141A3
:10545000C0F200010422C4F8D83016F00BFF01207E
:1054600010BD4AF28854C2F2010443F23D51C0F229
:1054700000010422E36416F0FDFE012010BD4AF293
:105480008854C2F2010443F65171C0F200010422B3
:10549000C4F8883016F0EEFE012010BD4AF28854A0
:1054A000C2F2010441F66561C0F20001236116F009
:1054B000E1FE012010BD4AF28854C2F2010443F219
:1054C000ED71C0F200010422E36516F0D3FE012065
:1054D00010BD4AF28854C2F2010444F20121C0F224
:1054E00000010422C4F8983016F0C4FE012010BD5B
:1054F000002800F0FF80012840F053814AF28854D0
:10550000C2F2010442F26D21C0F200010422012026
:10551000636016F0AFFE012010BD0F2800F0F88088
:10552000102840F03E814AF28854C2F2010443F24E
:105530003931C0F2000104221020236416F09AFED3
:10554000012010BD1E282FD01F2840F02A814AF2CA
:105550008854C2F2010443F64D51C0F20001042206
:105560001F20E36716F086FE012010BD4AF2885422
:10557000C2F2010442F27561C0F2000104222D2042
:10558000C4F8B43016F076FE012010BD4AF28854FB
:10559000C2F2010443F64511C0F200010422636621
:1055A00016F068FE012010BD4AF28854C2F20104D0
:1055B00043F6A141C0F200010422A36716F05AFE8F
:1055C000012010BD4AF28854C2F2010443F2E531D1
:1055D000C0F200010422636416F04CFE012010BDED
:1055E0004AF28854C2F2010443F29141C0F2000130
:1055F00004221220A36416F03DFE012010BD4AF2E1
:105600008854C2F2010441F60D51C0F20001042297
:10561000A36016F02FFE012010BD4AF28854C2F29A
:10562000010442F26901C0F2000104220720E36193
:1056300016F020FE012010BD4AF28854C2F2010487
:1056400042F62511C0F2000104223120C4F8C43012
:1056500016F010FE012010BD4AF28854C2F2010477
:1056600044F20541C0F2000104222920C4F8A4300C
:1056700016F000FE012010BD4AF28854C2F2010467
:1056800042F6DD71C0F2000104220B20E36216F045
:10569000F1FD012010BD4AF28854C2F2010444F227
:1056A0005511C0F2000104222520C4F8943016F0F0
:1056B000E1FD012010BD4AF28854C2F2010443F614
:1056C000F951C0F200010422C4F8803016F0D2FD76
:1056D000012010BD4AF28854C2F2010442F6D531CD
:1056E000C0F2000104223520C4F8D43016F0C2FD07
:1056F000012010BD4AF28854C2F2010441F6614112
:10570000C0F200010422236016F0B4FD012010BD98
:105710004AF28854C2F2010443F28D21C0F2000122
:105720000422E36316F0A6FD012010BD4AF288545E
:10573000C2F2010442F63171C0F200010422A362F8
:1057400016F098FD012010BD4AF28854C2F20104FF
:1057500043F24171C0F2000104221620A36516F045
:1057600089FD012010BD4AF28854C2F2010442F6BC
:10577000D951C0F200010422C4F8E03016F07AFDDD
:10578000012010BD4AF28854C2F2010441F6B95119
:10579000C0F2000104220320E36016F06BFD01203B
:1057A00010BD002010BD4AF28854C2F2010442F636
:1057B0008561C0F2000104223920C4F8E43016F0FB
:1057C00059FD012010BD4AF28854C2F2010444F28E
:1057D0005931C0F200010422C4F8A03016F04AFD8D
:1057E000012010BD4AF28854C2F2010443F6A561BB
:1057F000C0F2000104222120C4F8843016F03AFDE2
:10580000012010BD4AF28854C2F2010443F6F1119E
:10581000C0F2000104221A20A36616F02BFD01201D
:1058200010BD4AF28854C2F2010442F67901C0F276
:1058300000010422C4F8C03016F01CFD012010BD88
:105840004AF28854C2F2010443F2E111C0F20001AD
:105850000422A36316F00EFD012010BD4AF2885405
:10586000C2F2010441F6BD71C0F200010422A3613D
:1058700016F000FD012010BD4AF28854C2F2010466
:1058800043F29561C0F200010422636516F0F2FC58
:10589000012010BD4AF28854C2F2010443F6F531EA
:1058A000C0F200010422636716F0E4FC012010BD81
:1058B0004AF28854C2F2010444F2A901C0F2000184
:1058C0000422C4F8903016F0D5FC012010BD4AF235
:1058D0008854C2F2010442F62931C0F200010422C8
:1058E000C4F8D03016F0C6FC012010BDF8B504464F
:1058F00015460E460846022116F034FF28460221BE
:1059000016F030FF45F68423C0F20203012253F85B
:105910003600227200F50071216053F83510627272
:105920004DF2C04301F5007762F31F430022676028
:10593000E260013BFDD190F8003291F8002203F0C3
:105940000103D20744BF43F00203DBB2A372214636
:105950003046FFF7B1FB214620742846FFF7ACFB29
:10596000237C184420742046F8BD00BFF8B50646D5
:1059700044F68C100F46C0F202000B2119F062FAB7
:105980004EF2C0003946C2F2000000230A2215F090
:105990001BFF44F69810C0F20200012119F052FAE0
:1059A000B7B100252C4644F6BC400121C0F20200EC
:1059B00019F048FA01344EF2C000715DE4B2C2F24F
:1059C000000000230A2215F0FFFEA7422546EAD870
:1059D0004EF2C000C2F2000015F0E4FE4DF638535E
:1059E000C2F200031B7C73B1B07800F00F000130ED
:1059F000834208D0FBF7D6F928B944F69C10C0F2D0
:105A000002001B2107E07378432B0ED044F6B81038
:105A1000C0F202001B2119F015FA4EF2C000C2F2CA
:105A20000000BDE8F84015F0BDBE44F6D4100C21CE
:105A3000C0F2020019F006FAB1784EF2C000C1F3CC
:105A40000211C2F2000015F04FFE44F69810012139
:105A5000C0F2020019F0F6F94EF2C000C2F20000E6
:105A600015F0A0FE072F05D044F66C20C0F202000E
:105A70002021D0E7F378C3F38403002B00F0C88023
:105A8000022B40F0F180B379F72B40F0C48041F253
:105A9000D443C2F2010331791B6872794AF6AB2014
:105AA00001F07F01C3F6AA5007EE100A581802F061
:105AB0007F023171727180F8C82193F80A4293F81D
:105AC000075293F80C0293F80872C3F8C45093F885
:105AD000095293F80E2293F81012C3F8C87083F895
:105AE000D95004F00107C4F34005C4F3800493F8CF
:105AF0000BE283F8DA7083F8DB5000F0010783F8DB
:105B0000DC40C0F3400593F80D4283F8DDE0C0F3BC
:105B1000800083F8DE7002F0010E83F8DF5083F816
:105B2000E00093F80F5283F8E140C1F3400001F028
:105B30000104C2F34007C2F3800283F8E42083F833
:105B4000E64083F8E2E083F8E37083F8E55083F8F9
:105B5000E70093F81122520607EE902AF8EEE77A52
:105B6000C1F3800167EE877A83F8E810FDEEE77AEB
:105B700003F1C000C3ED357AFFF7A8F834795C343F
:105B8000E4B244F6B420C0F20200FAF70BFFF37857
:105B900013F07C0F05D144F64420C0F20200FAF75E
:105BA00001FF44F65020C0F20200FAF7FBFE4EF26D
:105BB000C00000230A223179C2F2000015F004FE71
:105BC00044F668200321C0F2020019F03BF94EF2BE
:105BD000C000717900230A22C2F2000015F0F4FD22
:105BE00044F65C200F21C0F2020019F02BF94EF2AE
:105BF000C00021460023C2F200000A2215F0E4FD95
:105C00004EF2C000C2F20000BDE8F84015F0CABD77
:105C1000B379F72B05D044F61C20C0F202002621F0
:105C2000F9E63279737941F2D444C2F2010402F008
:105C30007F0203F07F0320683271737109F0DAFC90
:105C4000F27833792068717902F0030203EBC21312
:105C5000034483F86C1109F0C1FBF478337903EB4A
:105C6000C41404F0FF048CE744F6E410C0F2020010
:105C70003621D0E638B504460D46FFF777FE44F6E8
:105C800090201021C0F2020019F0DCF841F2E0404F
:105C900000232A462146C2F2010014F0F7F844F22C
:105CA00014501421C0F2020019F0CCF82946204605
:105CB000002218F091FA44F2B440C0F202000F2121
:105CC00019F0C0F84EF2C000C2F20000BDE8384042
:105CD00015F068BD2DE9F04141F698550F46804614
:105CE000C2F20105FFF742FE44F6A4201521C0F2DE
:105CF000020019F0A7F8A86C0368F021DB6C984744
:105D000057B1444608EB0706A86C14F8011B03685A
:105D10001B689847A642F7D1A86C0368F721DB6C93
:105D2000984744F2A4400F21C0F2020019F08AF80B
:105D300039464046002218F04FFA44F2B440C0F20F
:105D400002000F2119F07EF84EF2C000C2F20000EE
:105D5000BDE8F04115F026BD2DE9F04141F698551A
:105D60000F468046C2F20105FFF700FE44F6BC2054
:105D70001021C0F2020019F065F8A86C0368F02148
:105D8000DB6C984757B1444608EB0706A86C14F83B
:105D9000011B03681B689847A642F7D1A86C0368EB
:105DA000F721DB6C984744F2A4400F21C0F20200B7
:105DB00019F048F841F2E0403A464146C2F201008B
:105DC000002314F063F844F21450C0F202001421CE
:105DD00019F038F84EF2C000C2F20000BDE8F04100
:105DE00015F0E0BCFFFFFFFF70B52DED068B4DF603
:105DF000385444F6D02082B0C2F20004B0EE40AA7B
:105E00001421C0F20200F0EE608A84ED020AC4EDB3
:105E1000030A19F017F81AEE100A1CF06FFF4EF281
:105E2000C005C2F2000544F6E82641EC100BC0F2B2
:105E3000020628460A2115F007FD3046012119F017
:105E400001F840F6DB73C4F24903A06808EE103A8B
:105E50001CF054FF41EC100B28460A2115F0F4FC0D
:105E600044F6EC200621C0F2020018F0EBFF3046A9
:105E7000012118F0E7FFE0681CF040FF41EC100B37
:105E800028460A2115F0E0FC44F6F4200221C0F275
:105E9000020018F0D7FFE36807EE903A27EE880A71
:105EA000F6EE00AA20EE2A0A19F066FFA36807EEB4
:105EB000903A60EE277A9FED3E9B17EE900A1CF019
:105EC0001DFFB0EE491AF0EE691A41EC100B1AF002
:105ED00053F82846032115F0B7FC44F6F8200121B9
:105EE000C0F2020018F0AEFFE36807EE903A27EE2A
:105EF000880A20EE2A0A19F0EFFEA36807EE903A0E
:105F000060EE277A17EE900A1CF0F8FEB0EE491A00
:105F1000F0EE691A41EC100B1AF02EF80321284616
:105F200015F092FC284615F03DFC68EE888A28EEB4
:105F3000AA8AB0EE480A19F01FFF6AEE007A17EE3F
:105F4000900A1CF0DBFEB0EE491AF0EE691A41EC43
:105F5000100B1AF011F855EC104BB0EE480A19F07E
:105F6000BBFE6AEE007A17EE900A1CF0C7FEB0EE98
:105F7000491AF0EE691A41EC100B19F0FDFF51ECD3
:105F8000100B1DF007FA2946019020461DF002FA79
:105F9000019B00EE100A00EE903A40F24850C2F227
:105FA000010002B0BDEC068BBDE870400CF01EBCD9
:105FB0000000002085EBB13F2DE9F041044644F696
:105FC000FC200D46C0F20200032118F03BFF4EF208
:105FD000C00000230A222146C2F2000015F0F4FBA3
:105FE00044F600300121C0F2020018F02BFF4EF2FF
:105FF000C000294600230A22C2F2000015F0E4FB8B
:106000004EF2C000C2F2000015F0CCFB672C00F08D
:10601000CF8150D9782C00F0A28000F28C80692CBE
:1060200000F0C080C0F09C816A2C00F05D816B2C78
:1060300040F06782002301EE903A05EB450500230E
:10604000C4F2482305EB051501EE103AC5F3C7135A
:1060500007EE903A41F69452C2F20102B8EE670A96
:10606000F0EE610AB7EE002A137003F0A7FC4FF4BC
:106070007E43C4F2FF6307EE903AB4EEE70AF1EE16
:1060800010FA00F3D5814FF47E43CCF2FF6307EEA4
:10609000903AB4EEE70AF1EE10FA40F134820023B0
:1060A000C8F2010341F24442C2F20102BDE8F041EC
:1060B000D36106F04DB8042C00F0A28140F2C980F3
:1060C0000A2C5ED040F2E480202C00F00681402CA7
:1060D00040F0308241F2D446C2F201063F2D94BF17
:1060E00000210121306809F085F9306809F08AF94A
:1060F0000546002840F0AB803068374609F01EFBAB
:10610000EBB203EB430498424FEA840440F29F80D1
:10611000306803190135DA78002AEFD093F802804D
:10612000B8F1000FEAD198680AF054FE38680444C8
:1061300084F80380E2E77B2C1AD040F29D807E2C0D
:1061400000F0C1807F2C40F0F78141F2D443C2F2CD
:10615000010300211868BDE8F04109F043B941F29C
:10616000D443C2F20103BDE8F041186809F04EB90A
:1061700041F2D443C2F20103BDE8F041186809F0CE
:1061800039BA4DF63853C2F2000300EE905A9A68BD
:10619000FBEEEC0A00EE102ABDE8F041C3ED030A65
:1061A000FFF722BE002301EE903A0023C4F296438B
:1061B00002EE103A05EB45050023C4F2482305EB37
:1061C000051501EE103AC5F3C71307EE903A40F2F9
:1061D0004452C2F20102B8EE670AF0EE610A13708F
:1061E00003F0ECFBB5EEC00AF1EE10FA00F13181DC
:1061F00047F67903C4F2302307EE103AF6EE007A40
:10620000E0EE077A49F68073C0F20103FCEEE77A0C
:1062100017EE902A9A4240F284811A464FF4507049
:1062200040F2C863C2F20103197ECC0700F1148169
:10623000DC8B1A62844241F0010138BFD8831976A1
:10624000BDE8F04105F084BF632D40F2F980BDE860
:10625000F081012C00F0E080F6D3022C40F04F8159
:1062600041F2D443C2F20103186880F8D050C03024
:10627000FEF72CFDBDE8F081792C40F0598141F208
:10628000D443C2F20103BDE8F041186809F0D2B866
:10629000072C40F04B8107EE905A0023C4F2FE23F6
:1062A000B8EE677A07EE903A87EE270A4DF6385334
:1062B000C2F20003BDE8F041DA6800EE902A83EDF7
:1062C000020AFFF791BD41F2D443C2F2010301215A
:1062D0001868BDE8F04109F085B84DF63853C2F2B0
:1062E00000031D71BDE8F08105EBC5050022C5F373
:1062F000471501EE902A07EE905A41F6104300220E
:10630000C2F20103C4F20C22B8EE670A01EE102AB1
:10631000F0EE610AB7EE002A1D7003F04FFB4FF458
:106320007E43C4F2FF6307EE903AB4EEE70AF1EE63
:1063300010FA00F381804FF47E43CCF2FF6307EE46
:10634000903AB4EEE70AF1EE10FA40F1E380002350
:10635000C8F2010341F20C42C2F20102D3616FE7BD
:106360002DB205EB850303EB830305EB8305C5F332
:10637000C71507EE905A0023C4F2C823F8EE676AE7
:1063800007EE903A86EEA77A41F2D442C2F20102B9
:1063900040F21C03C2F2010312681D70BDE8F04117
:1063A000F7EE007A77EEC77AC2ED587A05F0D0BEE4
:1063B0002DB205EB850303EB830305EB8305C5F3E2
:1063C000C71507EE905A0023C4F2C823F8EE676A97
:1063D00007EE903A86EEA77A41F2D442C2F2010269
:1063E00041F61143C2F2010312681D70BDE8F0418D
:1063F000F7EE007A77EEC77AC2ED597A05F0A8BEBB
:1064000041F2D443C2F20103186880F8D150C03081
:10641000FEF75CFCBDE8F08141F2D443C2F2010317
:10642000186880F8D250C030FEF750FCBDE8F0810B
:106430000023C7F6FF7335E60023C7F6FF7389E72D
:106440004DF63853C2F200031D71BDE8F04105F06E
:106450007FBE01200022E3E61C6AA24205D9D98B47
:106460001A62884288BFD883EAE602F17F00C00939
:10647000013000281A62024638BF0022880706D57C
:10648000586A7F30C0090130824238BF02464F0748
:1064900006D5986A7F30C0090130824238BF024673
:1064A0000E0706D5D86A7F30C0090130824238BF56
:1064B0000246CD0606D5186B7F30C00901308242F6
:1064C00038BF02468C0606D5586B7F30C0090130B4
:1064D000824238BF0246480606D5986B7F30C00915
:1064E0000130824238BF0246C90906D0D96B7F31DC
:1064F000C90901318A4238BF0A46DA83A0E6BDE8FD
:10650000F081BDE8F081F0EE407AFEEEC87A17EE39
:10651000903AC7E5F0EE407AFEEEC87A17EE903A70
:1065200018E702F17F00C009013079E6BDE8F0818B
:10653000BDE8F081BDE8F081BDE8F081F8B54DF629
:106540003857C2F2000704463B7C0E4615467BB323
:1065500098422DD044F2E0501E21C0F2020018F003
:1065600071FC4EF2C00000230A222146C2F2000054
:1065700015F02AF944F200600E21C0F2020018F072
:1065800061FC4EF2C000397C00230A22C2F20000F6
:1065900015F01AF944F210600121C0F2020018F05F
:1065A00051FC4EF2C000C2F2000015F0FBF803E00F
:1065B00029463046FFF700FD44F604300D21013C2A
:1065C000C0F2020018F03EFCE1B20F2915D841F6E6
:1065D0009857C2F2010741F0B001B86C03681B681C
:1065E0009847B86C036806F07F011B689847B86C41
:1065F000036805F07F011B68984744F2A4400F210F
:10660000C0F2020018F01EFC2B0603F0FE4331041A
:1066100043F4304343F00B0301F4FE012402194319
:1066200004F4706441F2E0402143C2F2010013F02F
:10663000EFFB44F21450C0F20200142118F002FCE7
:106640004EF2C000C2F20000BDE8F84015F0AAB852
:10665000F8B54DF63853C2F200030E461B7C1446C3
:10666000054623B1984202D0FAF79CFB18B12146A7
:106670003046FFF7A1FC44F614301221013DC0F270
:10668000020018F0DFFBE9B20F2915D841F6985740
:10669000C2F2010741F0B001B86C03681B6898476B
:1066A000B86C036806F07F011B689847B86C0368F4
:1066B00004F07F011B68984744F2A4400F21C0F208
:1066C000020018F0BFFB230603F0FE43310443F43D
:1066D000304301F4FE01280243F00B030B4300F4A6
:1066E0007060184317F024FD44F2B440C0F2020079
:1066F0000F2118F0A7FB4EF2C000C2F20000BDE867
:10670000F84015F04FB800BF70B54DF63853C2F2DF
:1067100000030E461B7C1446054623B1984202D066
:10672000FAF740FB18B121463046FFF745FC44F626
:1067300028300D21C0F2020018F084FB230603F07C
:10674000FE43340443F43043013D43F00B0304F4AF
:10675000FE042D021C4305F470652C4341F2E04019
:106760002146C2F2010013F053FB44F214501421ED
:10677000C0F2020018F066FB204617F0D9FC44F284
:10678000B440C0F202000F2118F05CFB4EF2C000D2
:10679000C2F20000BDE8704015F004B84AF234734C
:1067A000C2F2010382B01B68019341F69052C2F21B
:1067B000010240F27C53C2F20103019911600122EF
:1067C0001A7002B0704700BF44F248432DE9F04F01
:1067D000C0F202031C460FCCB1B020AD0FC50FCCE8
:1067E0000FC50FCC0FC594E80F0010944DF6385725
:1067F00040F27C54C2F20007C2F201044FF0000ED6
:1068000084F800E01F9585E80F00BD7A0395FD7AB6
:106810003B7904953D7B05957D7B06956FEA0309E1
:10682000BD7B079509F00F0930AD05EB8909BA79F1
:1068300097F80580787A02901D1159F8403C11951F
:106840001146FA79139183F070431446DB433A7A88
:10685000019283EA05020DF1C00E02F00F020EEB69
:1068600082024FEA281E52F8402C82EA1313DB43BF
:1068700083EA0802754602F00F020DF1C00E0EEB1E
:1068800082020DF1C00E52F8402C129582EA1313C9
:1068900083EA050202F00F020EEB82020DF1C00E38
:1068A00052F8402C82EA1313DB4383EA010202F020
:1068B0000F020EEB8202081152F8402C0199064695
:1068C00082EA131383EA06020DF1C00E02F00F02F2
:1068D0000EEB8202081114960990029852F8402C8F
:1068E000159482EA1313DB4383EA04020DF1C00E10
:1068F00002F00F020EEB8202251152F8402C039C8D
:10690000169582EA131383EA05020DF1C00E02F018
:106910000F020EEB82020DF1C00E52F8402C82EAFB
:1069200013136FEA030C8CEA010202F00F020599BF
:106930000EEB82020B1152F8402C0C93099B82EA59
:106940001C1C8CEA03020DF1C00E02F00F020EEBCC
:106950008202069B52F8402C1B110D9382EA1C13F5
:10696000DB4383EA0002061102F00F0207980A9641
:106970000DF1C00E0EEB820E02110E925EF8402C4D
:1069800082EA13130A9A5A4002F00F020DF1C00E68
:106990000EEB820E109AA2F1300C5EF8402C82EAC7
:1069A0001313DB4383EA04020DF1C00E02F00F0261
:1069B0000EEB820226110B9652F8402C0B9C049E83
:1069C00082EA131383EA04020DF1C00A02F00F02F7
:1069D0000AEB8202351152F8402C179582EA131304
:1069E000DB4383EA060202F00F020AEB82020DF19A
:1069F000C00A52F8402C0C9E82EA131383EA050267
:106A000002F00F020AEB82020DF1C00A52F8402C8C
:106A100082EA1313DB4383EA010202F00F020AEB5E
:106A200082020DF1C00A52F8402C82EA131383EA65
:106A3000060202F00F020AEB82020DF1C00A52F8C0
:106A4000402C069E0E9D97F813B082EA1313DB4389
:106A500083EA060202F00F020AEB82020D9E52F850
:106A6000402C82EA131383EA06020DF1C00A02F0F9
:106A70000F020AEB82020DF1C00A52F8402C82EAA2
:106A80001313DB4383EA000202F00F020AEB8202D7
:106A90000DF1C00A52F8402C82EA131383EA050272
:106AA00002F00F020AEB820297F80FA052F8402C76
:106AB000564697F810A01896514697F811A01A91CB
:106AC00082EA13135046DB4397F812A083EA0602CA
:106AD000554602F00F020DF1C00A0AEB8202361190
:106AE00052F8402C199682EA131383EA06020DF13C
:106AF000C00A02F00F020AEB82020DF1C00A52F83E
:106B0000402C1D9582EA1313DB4383EA010202F055
:106B10000F020AEB82020E1152F8402C0F9682EA05
:106B200013130F9A5A400DF1C00A02F00F020AEB3C
:106B30008202064652F8402C1B9682EA1313DB436E
:106B400083EA06020DF1C00A02F00F020AEB82028C
:106B5000011152F8402C1C9182EA131383EA0102BE
:106B60004FEA2B1ACDF820A002F00F020DF1C00A57
:106B70000AEB82020DF1C00A52F8402C82EA13138C
:106B8000DB4383EA050202F00F020AEB82022811BE
:106B900052F8402C1E9082EA131383EA00020DF192
:106BA000C00A02F00F020AEB820230AE52F8402C0B
:106BB00082EA1313DB438BEA030202F00F020AEBB3
:106BC00082020DF1800E52F8402C82EA131A089BC3
:106BD00055468AEA030ABCE80F000AF00F0A06EBE2
:106BE0008A0A3C465AF840ACAEE80F00BCE80F00F9
:106BF000AEE80F00BCE80F00AEE80F0059F8402CDB
:106C00008AEA151A82F07042119DD24382EA050386
:106C100003F00F0306EB83030DF1C00E53F8403C65
:106C200083EA1212D24382EA080303F00F0306EB51
:106C300083036FEA0A0A53F8403CC7F800A083EACE
:106C40001212129B534003F00F030EEB83030DF15E
:106C5000C00E53F8403C1398019983EA1212D243B4
:106C600082EA000303F00F030EEB8303149853F83A
:106C7000403C83EA121282EA00030DF1C00E03F0D9
:106C80000F030EEB8303159853F8403C83EA12126E
:106C9000D24382EA00030DF1C00E03F00F030EEBA6
:106CA0008303169853F8403C83EA121282EA0003E9
:106CB0000DF1C00E03F00F030EEB83030DF1C00EB8
:106CC00053F8403C099883EA1212D24382EA010346
:106CD00003F00F030EEB83030DF1C00E53F8403C9D
:106CE000059983EA121282EA000303F00F030EEB08
:106CF0008303029853F8403C83EA1212D24382EA9B
:106D000000030DF1C00E03F00F030EEB83030A988E
:106D100053F8403C83EA121282EA00030DF1C00EE0
:106D200003F00F030EEB83030DF1C00E53F8403C4C
:106D30000B9883EA1212039BD243534003F00F03D4
:106D40000EEB83030DF1C00E53F8403C83EA1212A0
:106D500082EA000303F00F030EEB83030DF1C00E74
:106D600053F8403C179883EA1212049BD2435340D5
:106D700003F00F030EEB83030DF1C00E53F8403CFC
:106D800083EA121282EA000303F00F030EEB83037F
:106D90000DF1C00E53F8403C0C9883EA1212D24316
:106DA00082EA010303F00F030EEB83030DF1C00E23
:106DB00053F8403C83EA121282EA000303F00F0307
:106DC0000EEB83030DF1C00E53F8403C0D9883EA9F
:106DD0001212069BD243534003F00F030EEB8303C2
:106DE0000DF1C00E53F8403C83EA121282EA000310
:106DF00003F00F030EEB83030DF1C00E53F8403C7C
:106E000007981A9983EA1212D24382EA000303F028
:106E10000F030EEB83030E9853F8403C83EA1212E3
:106E200082EA00030DF1C00E03F00F030EEB8303A3
:106E30000DF1C00E53F8403C199883EA1212189BCA
:106E4000D243534003F00F030EEB83030DF1C00E4A
:106E500053F8403C83EA121282EA000303F00F0366
:106E60000EEB83030DF1C00E53F8403C1E9883EAED
:106E70001212D24382EA010303F00F030EEB8303E5
:106E80000F9953F8403C83EA121282EA01030DF194
:106E9000C00E03F00F030EEB83030DF1C00E53F889
:106EA000403C1C9983EA12121B9BD243534003F0CF
:106EB0000F030EEB830307F1140553F8403C83EAFC
:106EC000121282EA010303F00F030EEB8303FE4369
:106ED00053F8403C83EA12121D9BD243534003F007
:106EE0000F030EEB830353F8403C83EA121282EA4D
:106EF000000303F00F030EEB830353F8403C83EAD7
:106F00001212D2438BEA020303F00F030EEB83034A
:106F100053F8403C83EA1212089B534003F00F03DE
:106F20000EEB830353F8403C83EA1213DB433B70C0
:106F300014F8018BA719384614F088FE80454146A5
:106F4000384601D014F09CFEAC42F1D144F6383002
:106F50002721C0F2020017F075FF4EF2C000C2F206
:106F6000000031B0BDE8F04F14F01CBCF0B597B094
:106F700001AD2C4606AE601B14F068FE04F8010B50
:106F8000B442F8D144F24845C0F202050FCD0FC417
:106F90000FCD0FC40FCD0FC495E80F0084E80F008C
:106FA0009DF808609DF809509DF80A409DF80B2057
:106FB0009DF80C309DF80D009DF80E10F7430DF173
:106FC000580E07F00F070EEB870757F8407C87F045
:106FD0007047FF4387EA161606F00F060EEB86068B
:106FE00056F8406C86EA1716F64385EA060707F05E
:106FF0000F070EEB870757F8407C87EA161787EADA
:10700000151606F00F060EEB86069DF80F5056F883
:10701000406C86EA1716F64384EA060707F00F0766
:107020000EEB870757F8407C87EA161787EA141695
:1070300006F00F060EEB86069DF8104056F8406CE1
:1070400086EA1716F64382EA060707F00F070EEBEB
:10705000870757F8407C87EA161787EA121606F06A
:107060000F060EEB86069DF8112056F8406C86EA56
:107070001716F64383EA060707F00F070EEB87079C
:1070800057F8407C87EA161787EA131606F00F06B2
:107090000EEB86069DF8123056F8406C86EA1716FD
:1070A000F64380EA060707F00F070EEB870757F84D
:1070B000407C87EA161787EA101606F00F060EEBDB
:1070C000860644F6603056F8406C86EA1716F6439A
:1070D00081EA060707F00F070EEB8707C0F20200F0
:1070E00057F8407C87EA161787EA111606F00F0654
:1070F0000EEB8606132156F8406C86EA1716F64307
:1071000085EA060707F00F070EEB870757F8407C64
:1071100087EA161686EA151505F00F050EEB8505AC
:1071200055F8405C85EA1615ED4384EA050606F03D
:107130000F060EEB860656F8406C86EA151585EAB2
:10714000141404F00F040EEB840454F8404C84EA49
:107150001514E44382EA040505F00F050EEB8505DE
:1071600055F8405C85EA141484EA121202F00F020A
:107170000EEB820252F8402C82EA1412D24383EAC8
:10718000020404F00F040EEB840454F8406C86EA09
:10719000121787EA131303F00F030EEB830353F860
:1071A000406C9DF813309DF814509DF815409DF8E3
:1071B000162086EA1716F64383EA060707F00F073C
:1071C0000EEB870757F8407C87EA161787EA1316F5
:1071D00006F00F060EEB86069DF8173056F8406C49
:1071E00086EA1716F64385EA060707F00F070EEB47
:1071F000870757F8407C87EA161686EA151505F0CA
:107200000F050EEB850555F8405C85EA1615ED4334
:1072100084EA050606F00F060EEB860656F8406C6B
:1072200086EA151585EA141404F00F040EEB8404A5
:1072300054F8404C84EA1514E44382EA040505F04E
:107240000F050EEB850555F8405C85EA141484EAB9
:10725000121202F00F020EEB820252F8402C82EA68
:107260001412D24383EA020404F00F040EEB8404E8
:1072700054F8404C84EA121484EA131303F00F0309
:107280000EEB830353F8403C83EA141417F0DAFD45
:10729000019D4EF2C000002310222946C2F20000D8
:1072A00014F092FA44F674300521C0F2020017F08F
:1072B000C9FDE4434EF2C0002146C2F200000023A3
:1072C000102214F081FAA5421DD14DF63855C2F2B4
:1072D000000505F114062C46601B14F0B7FC04F8F9
:1072E000010BB442F8D144F6A030C0F202000F21E5
:1072F00017F0A8FD4EF2C000C2F2000017B0BDE8C2
:10730000F04014F04FBA44F67C302321C0F2020062
:1073100017F098FDFFF758FAECE700BF2DE9F843A6
:107320004AF20E79C2F2010944F6B0302DED028B1B
:107330000521C0F2020017F085FDB9F8003007EE14
:10734000103A43F23333C4F2233308EE903AB8EEE6
:10735000C77A43F23333C4F2A33308EE103A37EE60
:10736000287A4EF2C004C7EE087AC2F200044AF24C
:107370000877C2F201074AF20C78C2F201084AF219
:107380008C66C2F2010640F22C05C2F2010517EE2E
:10739000900A1BF0B3FC41EC100B0221204614F0C4
:1073A00053FA44F6B8300D21C0F2020017F04AFD3E
:1073B0003B8807EE903AF8EEE77A77EEA87A87EE08
:1073C000887A17EE100A1BF099FC41EC100B022191
:1073D000204614F039FA44F6C8300821C0F2020001
:1073E00017F030FDB8F80010204614F07DF944F68F
:1073F000D4300C21C0F2020017F024FD3188204661
:1074000014F072F944F6E4301421C0F2020017F0CF
:1074100019FD2988204614F067F944F6FC3009214B
:10742000C0F2020017F00EFD41F2A843C2F20103C0
:107430000A2219682046002314F0C6F944F60840D1
:107440000D21C0F2020017F0FDFC40F22003C2F251
:1074500001030A2219682046002314F0B5F944F606
:1074600018400921C0F2020017F0ECFC41F6C033CD
:10747000C2F201030A2219682046002314F0A4F97D
:1074800044F624400C21C0F2020017F0DBFC8021FE
:10749000204614F029F944F634401021C0F20200CD
:1074A00017F0D0FC41F6ED33C2F201030A2219783D
:1074B0002046002314F088F9204614F073F9BDEC3F
:1074C000028BB9F80030B8F800203B8000233280EE
:1074D0002B80BDE8F88300BF70B584B0002441F272
:1074E000D44502940194CDF80B40C2F20105062662
:1074F00044F648400221C0F2020017F0A3FC4EF20D
:10750000C0003146C2F2000014F0EEF844F6A85074
:107510000221C0F2020017F095FC4EF2C000C2F248
:10752000000014F03FF944F64C405621C0F202002E
:1075300017F088FC4EF2C000C2F2000014F032F9DD
:107540002B6823444EF2C00093F86C110A220023EA
:10755000C2F2000014F038F944F6BC400121C0F238
:10756000020017F06FFC2B6823444EF2C00093F822
:107570006D110A220023C2F2000014F025F944F62E
:10758000BC400121C0F2020017F05CFC2B682344D0
:107590004EF2C00093F86E110A220023C2F20000DE
:1075A00014F012F944F6BC400121C0F2020017F0B9
:1075B00049FC2B6823444EF2C00093F86F110A2255
:1075C0000023C2F2000014F0FFF844F6BC40012191
:1075D000C0F2020017F036FC2B6823444EF2C000C4
:1075E00093F870110A220023C2F2000014F0ECF8A4
:1075F00044F6BC400121C0F2020017F023FC2B68C6
:1076000023444EF2C00093F871110A220023C2F203
:10761000000014F0D9F844F6BC400121C0F2020089
:1076200017F010FC2B6823444EF2C00093F872113F
:107630000A220023C2F2000014F0C6F844F6BC404F
:107640000121C0F2020017F0FDFB2B6823444EF22B
:10765000C00093F873110A220023C2F2000014F054
:10766000B3F844F6A4400821C0F2020017F0EAFB88
:107670002B6823444EF2C00093F874110A220023B1
:10768000C2F2000014F0A0F844F6B0400D21C0F2A0
:10769000020017F0D7FB2B6823444EF2C00093F88A
:1076A00075110A220023C2F2000014F08DF844F68E
:1076B000B0400D21C0F2020017F0C4FB2B68234438
:1076C0004EF2C0000A2293F87611C2F200000023A5
:1076D00014F07AF84EF2C000C2F2000014F062F822
:1076E00044F6C0405C21C0F2020017F0ABFB4EF242
:1076F000C000C2F2000014F055F844F620500621F4
:10770000C0F2020017F09EFB2B6823444EF2C0002B
:1077100093F877110A220023C2F2000014F054F803
:1077200044F6B4400921C0F2020017F08BFB2B682D
:1077300023444EF2C00093F878110A220023C2F2CB
:10774000000014F041F844F6B4400921C0F20200F0
:1077500017F078FB2B6823444EF2C00093F87911A0
:107760000A220023C2F2000014F02EF844F6A440CE
:107770000821C0F2020017F065FB2B6823444EF28B
:10778000C00093F87A110A220023C2F2000014F01C
:107790001BF844F6B8400521C0F2020017F052FB76
:1077A0002B6823444EF2C00093F87B110A22002379
:1077B000C2F2000014F008F844F620500621C0F28E
:1077C000020017F03FFB2B6823444EF2C00093F8F1
:1077D0007C110A220023C2F2000013F0F5FF44F6E8
:1077E00020500621C0F2020017F02CFB2B68234426
:1077F0004EF2C00093F87D110A220023C2F200006D
:1078000013F0E2FF44F6A8400421C0F2020017F092
:1078100019FB2B6823444EF2C00093F87E110A2214
:107820000023C2F2000013F0CFFF44F6B840052158
:10783000C0F2020017F006FB2B6823444EF2C00092
:1078400093F87F110A220023C2F2000013F0BCFF5C
:1078500044F6B8400521C0F2020017F0F3FA2B6895
:1078600023444EF2C00093F880110A220023C2F292
:10787000000013F0A9FF4EF2C0001534C2F2000060
:1078800013F090FF7E2C06F1FF367FF431AE44F604
:1078900028502D21C0F2020017F0D4FA4EF2C00099
:1078A000C2F2000013F07EFF44F6BC40C0F20200BA
:1078B000012117F0C7FA2B6823444EF2C00093F859
:1078C0006C110A220023C2F2000013F07DFF44F67F
:1078D00024500134C0F20200022141F2D44617F0D4
:1078E000B1FA862CC2F20106E5D14EF2C000C2F216
:1078F000000013F057FF44F658500521C0F2020073
:1079000017F0A0FA33684EF2C00093F8F2110A2281
:107910000023C2F2000013F057FF4EF2C000C2F283
:10792000000013F03FFF44F660500421C0F2020053
:1079300017F088FA33684EF2C00093F8F3110A2268
:107940000023C2F2000013F03FFF4EF2C000C2F26B
:10795000000013F027FF44F668500521C0F2020032
:1079600017F070FA33684EF2C00093F8F4110A224F
:107970000023C2F2000013F027FF4EF2C000C2F253
:10798000000013F00FFF44F670500921C0F202000E
:1079900017F058FA33684EF2C00093F8F5110A2236
:1079A0000023C2F2000013F00FFF4EF2C000C2F23B
:1079B000000013F0F7FE44F67C500921C0F20200EB
:1079C00017F040FA33684EF2C00093F8F6110A221D
:1079D0000023C2F2000013F0F7FE4EF2C000C2F224
:1079E000000013F0DFFE44F688500921C0F20200C7
:1079F00017F028FA33684EF2C00093F8F7110A2204
:107A00000023C2F2000013F0DFFE4EF2C000C2F20B
:107A1000000013F0C7FE44F694500921C0F20200A2
:107A200017F010FA33684EF2C00093F8F8110A22EA
:107A30000023C2F2000013F0C7FE4EF2C000C2F2F3
:107A4000000013F0AFFE44F6A0500A21C0F202007D
:107A500017F0F8F933684EF2C00093F8F9110A22D2
:107A60000023C2F2000013F0AFFE4EF2C000C2F2DB
:107A7000000013F097FE44F6AC500D21C0F2020056
:107A800017F0E0F933684EF2C00093F8FA110A22B9
:107A90000023C2F2000013F097FE4EF2C000C2F2C3
:107AA000000013F07FFE44F6BC500921C0F2020032
:107AB00017F0C8F933684EF2C00093F8FB110A22A0
:107AC0000023C2F2000013F07FFE4EF2C000C2F2AB
:107AD000000013F067FE44F6C8500921C0F202000E
:107AE00017F0B0F933684EF2C00093F8FC110A2287
:107AF0000023C2F2000013F067FE4EF2C000C2F293
:107B0000000013F04FFE44F6D4500621C0F20200EC
:107B100017F098F931680A2201F2FD1101A81CF052
:107B20007DF944F6E8200121C0F2020017F08AF93D
:107B300001A81CF005F9014601A817F083F944F6E5
:107B400098100121C0F2020017F07CF94EF2C0003B
:107B5000C2F2000013F026FE9B244EF2C000002368
:107B60000A222146C2F2000013F02EFE44F6A8506D
:107B70000221C0F2020017F065F92B6823444EF28F
:107B8000C00093F86C110A220023C2F2000013F027
:107B90001BFE4EF2C0000134C2F2000013F002FEE0
:107BA000AD2CDAD14EF2C000C2F2000013F0FAFDA3
:107BB00004B070BD2DE9F04141F6805086B0C2F2AC
:107BC000010013F041F841F68050C2F2010012F0BA
:107BD000D1FE41F68050C2F2010012F0C3FE41F620
:107BE0008050C2F2010012F04FFD41F68050C2F207
:107BF000010012F0C7FE41F68050C2F2010012F0FF
:107C000079FE41F68050C2F2010012F0A3FE44F664
:107C1000DC53C0F2020393E8070000244FF0203742
:107C20006B46029703940494CDF80B708DF81440C2
:107C300003C341F680501A8021462246C2F2010059
:107C400012F064FE68461CF07BF8024641F6805054
:107C50006946C2F2010013F031FD4EF2C000234626
:107C60000A222146C2F2000013F0AEFD44F6F820CD
:107C70000121C0F2020017F0E5F84EF2C0002346E1
:107C80000A222146C2F2000013F09EFD44F6E8509D
:107C90000321C0F2020017F0D5F868461CF050F836
:107CA0000146684617F0CEF844F698100121C0F25C
:107CB000020017F0C7F844F6EC564EF2C000C0F2CE
:107CC0000206C2F2000013F06DFD96E8030000907A
:107CD00041F68050019722468DF80410C2F201004F
:107CE0000B21029703940494CDF80B708DF8144087
:107CF00012F00CFE68461CF023F8024641F6805054
:107D00006946C2F2010013F0D9FC4EF2C0002346CE
:107D10000A222146C2F2000013F056FD44F6F82074
:107D20000121C0F2020017F08DF84EF2C000234688
:107D30000A220B21C2F2000013F046FD44F6E8507F
:107D40000321C0F2020017F07DF868461BF0F8FF2F
:107D50000146684617F076F844F698100121C0F203
:107D6000020017F06FF84EF2C000C2F2000013F0EC
:107D700019FD44F6F453C0F202030FCB8DE80F0057
:107D800041F6805021460122C2F2010004948DF890
:107D9000144012F0BBFD68461BF0D2FF024641F6CC
:107DA00080506946C2F2010013F088FC4EF2C00018
:107DB00023460A220121C2F2000013F005FD44F619
:107DC000F8200121C0F2020017F03CF84EF2C0008A
:107DD0000A2223462146C2F2000013F0F5FC44F6C5
:107DE000E8500321C0F2020017F02CF868461BF09F
:107DF000A7FF0146684617F025F844F698100121C0
:107E0000C0F2020017F01EF84EF2C000C2F20000ED
:107E100013F0C8FC0221042014F0A4FC02211E204F
:107E200014F0A0FCDC2014F001FD44F608603421BD
:107E3000C0F2020017F006F84EF2C000C2F20000D5
:107E400013F0B0FC44F640602E21C0F2020016F0A0
:107E5000F9FF4EF2C000C2F2000013F0A3FC44F69A
:107E600070602721C0F2020016F0ECFF4EF2C00055
:107E7000C2F2000013F096FC44F698600921C0F2AB
:107E8000020016F0DFFF0521304616F0DBFF4EF250
:107E9000C000C2F2000013F085FC44F6A4600D217E
:107EA000C0F2020016F0CEFF4EF2C000C2F2000097
:107EB00013F078FCFFF75AF8FCF75AFD4EF28813DE
:107EC000CEF20003012740F2002040F24855C2F2F2
:107ED00001051F604FF4E171C1F6FF7012F0C6FE9C
:107EE00028460AF039FF28460AF0A4FAEA88242135
:107EF00022F0100228460AF06DF9EA88242122F4C3
:107F0000807228460AF066F928460AF013FAF7EE5E
:107F1000000AB0EE600A28460AF086FB4CF6CD4611
:107F20001F2128460AF0FCFAC3F64C5628460AF0F0
:107F300069FD01EE106A4DF20A76C3F6234600EEA3
:107F4000906A46F26666C3F666763A4600EE106AB6
:107F50003B46394628460AF09FFD28460AF068F954
:107F600044F6B4601B21C0F202004DF6385616F0FC
:107F700069FFC2F200064EF2C000C2F2000013F028
:107F800011FCF36800EE903AB36800EE103AFDF78A
:107F90002BFF4DF66850C2F200000B210CF0DEF80A
:107FA0004DF66850C2F200000D210CF03FF948F682
:107FB0003070C2F20100FE210CF076FA002840F089
:107FC000028144F6D0601721C0F2020016F03AFF99
:107FD0004EF2C000C2F2000013F0E4FB44F6E86386
:107FE000C0F2020393E8030041F6D83241F674531D
:107FF000C2F20102C2F2010382E8030083E8030037
:108000000023C4F2C82306EE903A0023C4F22C23C6
:1080100007EE903A002306EE103AB36807EE103AE6
:1080200027EE267A27EE277AC7EE267A77EE867A2B
:10803000FDEEE77A17EE903A9B0072B641F27C446F
:10804000C2F20104E36062B6237C012B40F2248378
:1080500072B6E36862B640F22402002BC2F201025B
:10806000B8BF03339B101360737972B69B00236211
:1080700062B694F82430012B40F2188372B6236A5A
:1080800062B640F22402002BB8BF0333C2F20102F1
:1080900041F6F0309B10C2F20100536012F096FAE4
:1080A00041F60040C2F2010012F090FA4AF20E745A
:1080B0004AF20C71C2F20104C2F201014AF20872E2
:1080C0004AF28C63C2F20102C2F2010344F60C7060
:1080D00025880C8815801821C0F202001C8016F03B
:1080E000B1FE4EF2C00000230A223179C2F2000034
:1080F00013F06AFB44F6F8200121C0F2020016F0EA
:10810000A1FE4EF2C00000230A227179C2F20000E3
:1081100013F05AFB44F698100121C0F2020016F049
:1081200091FE4EF2C000C2F2000013F03BFBFFF7DD
:10813000D3F944F628701421C0F2020016F082FE32
:108140004EF2C0008021C2F2000013F0CDFA44F6D6
:1081500040701121C0F2020016F074FE4EF2C00011
:1081600040F65A31C2F2000013F0BEFA44F65470E1
:108170000321C0F2020016F065FE4EF2C000C2F20A
:10818000000013F00FFBFFF7C9F841F68050C2F270
:10819000010012F0AFFB01F033FC4EF20813CEF2F7
:1081A0000003012244F658701A600B21C0F202004D
:1081B00016F048FE4EF2C000C2F2000013F0F2FAD0
:1081C00006B0BDE8F08144F6F0600E21C0F2020076
:1081D00016F038FE4EF2C000C2F2000013F0E2FAD0
:1081E00041F2AD42C2F2010240F23008177008F0CD
:1081F00055F8327941F6EC3EC2F2010E02EB420331
:1082000002EB8302C2F2010841F6D8318EF8000079
:10821000C2F2010108EB020007F0CEFE307907F050
:10822000E9FE44F600700621C0F2020016F00AFED4
:10823000337903EB430503EB850308EB030528467D
:108240001BF07EFD0146284616F0FCFD44F6F820A2
:108250003946C0F2020016F0F5FD41F6D830C2F200
:1082600001001BF06DFD014641F6D830C2F201005D
:1082700016F0E8FD44F698103946C0F2020016F0F8
:10828000E1FD4EF2C000C2F2000041F6144513F0C9
:1082900089FAC2F201052FE044F608700321C0F20A
:1082A000020016F0CFFD4EF2C00000230A22214644
:1082B000C2F2000013F088FA44F6E8200121C0F26F
:1082C000020016F0BFFD28461BF03AFD0146284685
:1082D00016F0B8FD44F698100121C0F2020016F025
:1082E000B1FD4EF2C0000134C2F2000013F05AFAA0
:1082F000202C05F10B0509D0092CCDD844F6BC4043
:108300000121C0F2020016F09DFDC5E741F61044C0
:10831000C2F20104002301EE903A237800EE103AF5
:108320000023C4F2964302EE103A0023C4F248231D
:1083300001EE103AB8EE400AF0EE610A01F03EFBA1
:10834000B5EEC00AF1EE10FA00F1818147F679032B
:10835000C4F2302307EE103AF6EE007AE0EE077A28
:1083600049F68073C0F20103FCEEE77A17EE902A1B
:108370009A4240F296811A464FF4507140F2C86317
:10838000C2F20103187EC50700F11481DD8B1A6269
:10839000A94240F0010088BFD9831876237800EE07
:1083A000103A002301EE903A41F20C450023C4F24A
:1083B0000C23C2F2010501EE103AB8EE400A4FF468
:1083C0008033F0EE610AB7EE002AAB6101F0F6FAF5
:1083D0004FF47E43C4F2FF6307EE903AB4EEE70A2F
:1083E000F1EE10FA0FDC4FF47E43CCF2FF6307EEA0
:1083F000903AB4EEE70AF1EE10FA40F12B81002337
:10840000C8F2010302E00023C7F6FF7341F694545B
:10841000C2F20104002201EE902A2278EB6100EE04
:10842000102A0022C4F2482201EE102AB8EE400AB7
:10843000F0EE610AB7EE002A01F0C0FA4FF47E4375
:10844000F7EE007AC4F2FF6337EEC00A07EE903A07
:10845000B4EEE70AF1EE10FA0FDC4FF47E43CCF2F3
:10846000FF6307EE903AB4EEE70AF1EE10FA40F13E
:108470000C810023C8F2010302E00023C7F6FF735A
:10848000227800EE102A002201EE902A41F24445A3
:108490000022C4F24822C2F2010501EE102AB8EE11
:1084A000400AF0EE610AB7EE002AAB6101F086FAED
:1084B0004FF47E43C4F2FF6307EE903AB4EEE70A4E
:1084C000F1EE10FA0FDC4FF47E43CCF2FF6307EEBF
:1084D000903AB4EEE70AF1EE10FA40F1CF800023B3
:1084E000C8F2010302E00023C7F6FF732278EB61B4
:1084F00000EE102A002201EE902A0022C4F2482247
:1085000001EE102AB8EE400AF0EE610AB7EE002A3A
:1085100001F054FA4FF47E43C4F2FF6307EE903A41
:10852000B4EEE70AF1EE10FA0FDC4FF47E43CCF222
:10853000FF6307EE903AB4EEE70AF1EE10FA40F16D
:1085400096800023C8F2010302E00023C7F6FF7300
:1085500041F6114140F21C02C2F20101C2F20102D5
:10856000097812782B6207EE101A07EE902A002283
:10857000C4F2C82206EE102AB8EE477AF8EE677AFF
:10858000C7EE066A41F2D443C2F2010371791B6857
:10859000307987EE867AF7EE007A77EEE66A37EE84
:1085A000C77AC3ED596A83ED587AC3ED5A7A08F059
:1085B00009F825E51D6AAA4253D802F17F01C909CD
:1085C000013100291A620A4638BF0022870706D502
:1085D000596A7F31C90901318A4238BF0A464507C5
:1085E00006D5996A7F31C90901318A4238BF0A46E6
:1085F000010706D5D96A7F31C90901318A4238BFDE
:108600000A46C70606D5196B7F31C90901318A426E
:1086100038BF0A46850606D5596B7F31C909013135
:108620008A4238BF0A46410606D5996B7F31C9098F
:1086300001318A4238BF0A46C10906D0D96B7F3161
:10864000C90901318A4238BF0A46DA83A6E6012108
:10865000002293E6F0EE407AFEEEC87A17EE903AEA
:10866000D4E6D88B1A62814288BFD98396E6F0EEB1
:10867000407AFEEEC87A17EE903A69E7F0EE407A5B
:10868000FEEEC87A17EE903A30E7F0EE407AFEEE52
:10869000C87A17EE903AF3E672B62046FCF7BCFCB7
:1086A000D7E402F17F01C909013167E672B641F2F0
:1086B0009040C2F20100FCF7AFFCE0E42DE9F04786
:1086C0009DF82040013CE4B20F2C03D84EB2002E9E
:1086D0000D4601DBBDE8F087E0290FD9F729F9D96C
:1086E0000835EDB2012303FA05F515F0DD0FF1D0E1
:1086F000806C0368BDE8F0471B6818478146806CB2
:108700001F46036846EA0401C9B21B6890469847B1
:10871000D9F84800036808F07F011B6805F0EF05F1
:108720009847C02DD6D0D9F84800036807F07F01DC
:108730001B68BDE8F0471847F8B50446806C03682D
:108740001B69984708B90020F8BDA06C03685B69F5
:108750009847C3B203F0FB01F929F4D0A26D82B9A6
:1087600094F84D2084F84F30150600F19C8040B2FB
:108770000028C0F25081002084F84D00A06560659B
:10878000F8BD010667D494F84F10F02904EB0201FC
:1087900040D081F84F30616D4B1E9A4240D394F81F
:1087A0004F20F02AE7D013063DD4002384F866302A
:1087B000B02B4CD0A02B4AD0D02B48D0E02B46D0A9
:1087C000C02B44D0002094F8505084F867500329FF
:1087D00008BF94F8515084F8650018BF00250021A7
:1087E0000120B02B84F86850A165616584F8E90028
:1087F00000F0B58000F2AC80902B00F0B080A02B90
:1088000000F0AD80802B00F0AA80002384F84D306A
:108810000120F8BD81F86930636D013B9A42AAD20C
:108820000132A2658FE702F10C03DBB2012BBCD948
:1088300002F0FB03F92BB8D0EF2A00F2DB8002F044
:10884000F003802B84F8663001D0902BB0D102F079
:108850000F000130B7E7A3F1F701082993D80125EC
:1088600005FA01F010F4DD7F40F0968000298AD1EE
:1088700094F86930F02B7FF47EAF561C2244F72029
:10888000370A82F8690084F8676084F8687084F8B1
:10889000651084F84D10284684F8663084F8E95055
:1088A000A1656165F8BD02F10C05EEB2012E7FF6FF
:1088B0005EAF02F0FB0EBEF1F90F3FF458AFEF2AA6
:1088C0002DD802F0F007802F2AD140B20028FFF601
:1088D0004FAF012184F84F2084F85030A165EDB2EC
:1088E000012D7FF648AFBEF1F90F3FF444AFEF2AF8
:1088F0005FD802F0F003B02B26D01ED9D02B04D0C5
:10890000E02B21D0C02B7FF436AF02236365012119
:10891000A36D994227D90133A3650020F8BD1746FE
:1089200007F0DF06902ED0D007F0BF06A02ECCD0E7
:1089300007F0EF07C02FC8D019E7902B04D0A02B69
:1089400002D0802B7FF417AF032363650221DFE79A
:10895000D02B04D0E02B02D0C02B7FF456AF84F88C
:108960004D200120F8BDEF2A94BF02F0F005154616
:1089700002F00F020023013294F8501084F86520B1
:10898000012084F8671084F8683084F86650A36585
:10899000636584F8E900F8BD002284F8672084F854
:1089A000682084F8652084F8663084F8E950284609
:1089B000F8BDF62A0FD007D8F12AA6D01CD9F22A82
:1089C000C2D0F32AA1D0D6E6FC2A21D8FA2A02D2B4
:1089D000F82A7FF4D0AE0023012084F8653084F8B3
:1089E000673084F8683084F86620A365636584F88E
:1089F000E900F8BD1346D9E6F02A7FF4BCAE802129
:108A00000023616584F8692084F84D307F217FE779
:108A1000FE2AE0D2AFE61A468E4603F10C055EE769
:108A200090F86630F12B7CD00ED9FA2B2BD01FD8C2
:108A3000F32B38D0C0F08180F62B7AD0F82B40F0A1
:108A40008B80036BF3B11847B02B6ED031D9D02B8C
:108A500021D03ED9E02B42D0F02B7ED1C3698BB11F
:108A6000B0F86710802900F1690028BF80211847FD
:108A7000FC2B0CD051D3FE2B4BD0FF2B6BD1436C76
:108A8000002BE0D17047436B002BDCD1FAE7C36BBE
:108A9000002BD8D1F6E74369002BF3D090F867108C
:108AA00090F865001847836A002BEBD090F86700B8
:108AB0001847902B29D0A02B23D0802BE2D103681C
:108AC000002BDFD090F8682090F8671090F86500D0
:108AD0001847C02B42D10369002BDFD1D2E782694E
:108AE000002ACFD090F8681090F8673090F86500B1
:108AF000C90101F47E5103F07F031943A1F5005130
:108B000010478368002BDDD1BCE74368002BD9D127
:108B1000B8E7036C002B96D1B4E7836B002B92D19E
:108B2000B0E7036A002BC1D1ACE7C368002BC9D101
:108B3000A8E7C36A002B86D1A4E7426A002AA1D025
:108B400090F8683090F86700DB0103F47E5300F082
:108B50007F0018431047704770477047704700BF49
:108B600090F86430DA0725D513F0FE0F22D070B5E7
:108B700090F8665085F08002602A82B004461AD9C7
:108B8000F62D6ED067D8F12D7ED04FD9F22D2DD095
:108B9000F32D1AD1806C94F86760036829461B682E
:108BA0009847A06C0368DB6C06F07F0102B0BDE85B
:108BB00070401847704790F865608E4207D031B119
:108BC0005B08012B08D0032B27D002B070BD5B08D7
:108BD000012B01D0022BF8D194F8683094F867206B
:108BE000009629462046FFF769FDEEE7806C94F871
:108BF0006730026894F868601268294643EAC6152F
:108C00009047A06C036805F07F019B6C9847A06CAF
:108C10000368C5F3C6119B6CC8E794F8683094F8F4
:108C2000672000962946FFF749FDCEE7F02DCCD10D
:108C3000B0F86760802E28BF802600F16905002EFD
:108C4000C3D02E44A06C15F8011B03681B6898471D
:108C5000AE42F7D1B9E7FC2D26D8FA2D01D2F82D76
:108C6000B3D105F10803DBB2072BAED8012202FA1B
:108C700003F313F0DD0FA8D0A06C03681B6829462E
:108C800002B0BDE870401847806C94F8672094F8F3
:108C9000683006681201294603F00F0302F07005E0
:108CA00032681D439047E7E7FE2D8ED3D9E700BF1A
:108CB00070B540F2805086B0C2F201000BF01CF992
:108CC000002840F09F804AF23474C2F2010441F659
:108CD000905223680193C2F20102019B116841F294
:108CE00087325B1A934206D941F6ED33C2F2010393
:108CF0001B78002B42D041F69855C2F2010595F839
:108D00004C60102E4BD9002015F0B4FC10F086FA00
:108D100041F2E0400021C2F2010011F071F941F28C
:108D2000A44322680292C2F20103029A1868121A3E
:108D30004AF23471C82AC2F201014DD841F2D0433F
:108D400022680492C2F20103049A1968521A632A33
:108D500053D840F2606322680592C2F20103059A7B
:108D6000196841F28730521A824205D901F59C51A7
:108D700008311960FEF7D2FA06B070BD40F27C539C
:108D8000C2F201031B78002BB5D041F69855C2F210
:108D90000105FDF719FD95F84C60102EB3D8284653
:108DA000FFF7CAFC0028AED095F86630902B00F093
:108DB000AC8083F08003602B40F2AA8041F698508B
:108DC000C2F20100FFF72CFE41F698503146C2F284
:108DD0000100FFF7C5FE96E741F2D442096803910E
:108DE000C2F2010203991068196006F0ABFC41F66B
:108DF000ED33C2F201031870A0E76431196003F08B
:108E0000A7F9A6E740F25454C2F2010413F0E6FCBD
:108E10002368C01AB0F5356F7FF655AF13F0DEFC4E
:108E2000206040F28050C2F201000BF075F8044659
:108E300013F0D4FC41F2D443C2F2010305462246AA
:108E40001868802105F072FE13F0C8FC40F65A3312
:108E5000401B984251D840F22C0413F0BFFCC2F2E0
:108E60000104401B238883425FD372B640F25853FB
:108E7000C2F201031A7F02F0FF010AB100221A7741
:108E800062B699B372B647F6FF744FF40040B3F977
:108E90001E10B3F92020DC83188462B6002982EA10
:108EA000E273A3EBE273B8BF49428B42B8BF0B46F3
:108EB00007EE903A4FF47E43C4F2FF6306EE103A99
:108EC000F8EEE77A47F2A403C7EE866AC3F67D732D
:108ED00007EE103AF4EEC76AF1EE10FA06DD41F63D
:108EE000C033C2F201031A6801321A6040F28050A6
:108EF000C2F201000BF022F8E5E641F2A843C2F20B
:108F000001031A6801321A60A5E795F8683043B189
:108F100095F865309E423FF451AF002E3FF44EAFBE
:108F200052E7802385F86630F2E713F057FC401BC8
:108F300020809AE72DE9F04F41F69855C2F20105DD
:108F400089B012F031FE95F86430002401264DF608
:108F5000F06743F001034FF6FF7E66F347032146B7
:108F600085F8654085F8664085F8674085F8684073
:108F700085F8E940C2F2000705F169008022C5F8D2
:108F80005CE0C5F860E085F86430AF6485F84C407B
:108F900085F84D4085F84E406C65AC651AF098FD3B
:108FA0004DF6301240F695112846C2F20002C0F28A
:108FB000000141F2E047C2F201072C606C60AC6036
:108FC000EC602C616C61AC61EC612C626C62AC6237
:108FD000EC622C636C63AC63EC632C646C641AF01D
:108FE00029FA45F6C812C0F2020207F59B6307F59D
:108FF000B36107F5A36007F5AB653A607B6140227A
:1090000050237C60BC60B861FD61384679627A8526
:10901000BB8510F0B9FE41F6805844F21C43C2F201
:109020000108C0F202033B604046022310222721C0
:1090300011F01CFB41F27C4044F23843C0F20203C1
:1090400002220321C2F20100C8F80030FCF74EFCF6
:1090500041F290401D221C21C2F20100FCF746FCA7
:1090600041F6F030142204214AF2347AC2F20100AF
:1090700011F094FAC2F2010A41F6004014221E21B6
:10908000C2F2010011F08AFADAF80030029341F2DC
:10909000D043C2F2010340F28058C2F20108029AA2
:1090A0001A602146224640F2585B4046FBF734FCEA
:1090B000C2F2010B45F65803C0F202030BF118028D
:1090C0003146584688F89C40C8F8984088F89D403A
:1090D000C8F8003040F2C865FBF71EFC4FF40041B1
:1090E000C2F2010547F6FF7245F60C03ABF82010FB
:1090F00044F21041C0F20203ABF81E20C0F202019C
:1091000005F55462CBF800302C722346EC60204603
:109110006E722A6129602C4600E0226942F8230021
:10912000697A013340F2C8629942C2F20102F4DC6A
:109130004AF28863C2F201030093196809B9D2E1C7
:1091400019464B69002BFBD14D61002441F20C47BD
:1091500045F6340340F20870C2F20107C0F2020380
:1091600021466C61AC80EC80AC724FF45062C2F26C
:1091700001002B602C766C83AC83EC831AF0A8FC86
:1091800007F1280238460421FBF7C6FB41F24446AA
:1091900045F64003C2F20106C0F202033B6006F14D
:1091A00028024FF4803304213046BB61FB613B62EF
:1091B0007B62019340F22469FBF7AEFB45F6400366
:1091C000C2F20109C0F2020348463360019BB36159
:1091D000F3613362736289E8000989F8084089F80D
:1091E0000940C9F80C4089F8104040F2386B11F082
:1091F0009BFE4DF6301240F69911C2F2010BC2F2FD
:109200000002C0F2000148461AF014F95846CBF8A3
:109210000470CBF800808BF808408BF80940CBF83D
:109220000C408BF8104040F24C6911F07DFE4DF679
:10923000301240F69911C2F20109C2F20002C0F2E6
:10924000000158461AF0F6F84846C9F8008089F837
:10925000084089F80940C9F80C4089F81040C9F85D
:10926000046041F6C43811F05FFE4DF6301240F64E
:109270009911C2F20108C2F20002C0F20001484690
:109280001AF0D8F84FF0010B404688E8A00088F8A3
:109290000840C8F80C4088F8104088F809B040F23F
:1092A000646911F041FE4DF6301240F69911C2F298
:1092B0000109C2F20002C0F2000140461AF0BAF8F9
:1092C0000223484689F80930019389E8600089F84B
:1092D0000840C9F80C4089F8104040F2786811F055
:1092E00023FE4DF6301240F69911C2F20108C2F287
:1092F0000002C0F2000148461AF09CF84046C8F847
:109300000070C8F8045088F8084088F80940C8F888
:109310000C4088F8104040F28C6511F005FE4DF6C7
:10932000301240F69911C2F20105C2F20002C0F2F9
:10933000000140461AF07EF828462F602C72EC603F
:109340002C7485F809B06E6041F2B04711F0ECFD65
:109350004DF6301240F69911C2F20107C2F2000236
:10936000C0F2000128461AF065F8019B7B7244F2B6
:10937000104307F11801C0F2020322463B603C7221
:10938000FC60204639610B463C4600E0236943F807
:109390002200797A013241F2B0439142C2F20103D4
:1093A000F4DC009A12684AF28861C2F201010AB93B
:1093B0009BE01A465369002BFBD15761002441F210
:1093C000B04040F2A06845F64C03C2F20108C0F27A
:1093D00002037C61BC80FC80BC72C2F201003B6075
:1093E0000AF00AFC404688E8C00088F8084088F87F
:1093F0000940C8F80C4088F8104040F2B46511F0FC
:1094000093FD4DF6301240F69911C2F20105C2F2F9
:109410000002C0F2000140461AF00CF80123284671
:1094200085E8C0006B722C72EC602C7411F07CFD2E
:109430004DF6301240F69911C0F200012846C2F2F2
:10944000000219F0F7FF40F24853C2F2010345F65B
:109450001802C0F202021A604FF419700A221A723E
:1094600012F0D4FE4AF64441064605F0E1F8DAF877
:1094700000300393039DDAF800300493049CDAF87B
:109480000030059341F2D440C2F2010041F6905100
:1094900040F2206241F6E833C2F20101C2F2010259
:1094A000C2F20103066005980D601460186013F0A5
:1094B00095F9DAF800300693069DDAF80030079344
:1094C00040F2545141F2A44240F26063C2F2010101
:1094D000C2F20102C2F20103079C086015601C6021
:1094E00009B0BDE8F08F1A602FE60B6066E700BF99
:1094F0004FF07E520021416702678267704700BFCC
:1095000070B507EE901A2DED048BB8EEE79AB7EE22
:10951000008A88EE097A4FF46043C4F22B73002569
:1095200000260446866305638561C561C560856064
:109530004560056007EE903A80ED057A87EE897AFE
:109540000562456380ED049A17EE100A19F0D6FB08
:1095500041EC100B16F0ACFE51EC100B19F01AFF99
:1095600049F6AB03C3F6B44308EE900A07EE903A0F
:1095700068EEA77A40F6DB7388EE277AC4F24903D7
:1095800006EE903A2369C4ED097A05EE903AB6EEFC
:10959000006ABAEE040AA5EE860A636907EE903AFD
:1095A00020EE260A84ED0A7A20EE270A16F02EFC19
:1095B0004BF60B43C3F6324307EE103A0023C4F2D6
:1095C000FC2307EE903A68EE878A87EE897A0123BA
:1095D00023660023CBF6807384F854606566A56625
:1095E000E364A364C8EE287A38EE478AC4ED168A8D
:1095F00084ED1B8ABDEC048B84ED0B0AC4ED177A55
:1096000070BD00BFF8B50B6806EE903A436E07EEEA
:10961000903AC36E07EE103A836E76EEE77A06EE66
:10962000103AE7EE067A02F18047012A2DED108B01
:1096300007F1FF37C1ED007AC0ED196A19DD01EBC2
:1096400087040B465D6807EE905A37EEE67A06EE21
:10965000905AC56E06EE105A1D6805EE905AA6EE99
:10966000257A17EE105A43F8045FA342C0ED197A29
:10967000E8D1846FBF0007EE904ACB19B7EE007AAD
:10968000F4EE477A1B688366F1EE10FA11D0002AD7
:109690000FDD3C1D0C440B4602E0856F07EE905A2F
:1096A0001D6807EE105A67EE277AE3EC017AA342B1
:1096B000F3D1036F07EE903AB7EE007AF4EE477AF3
:1096C000F1EE10FA00F0FB80C36C07EE103A436F26
:1096D000F4EE477AF1EE10FA16460D46044600EE17
:1096E000103A40F0EF80836C07EE903AB4EE670AD0
:1096F000F1EE10FA40F0E680C36B0CEE903AF7EE14
:1097000000BA3CEEABDA002E8CEE8DBA40F3D78077
:1097100040F6DB73C4F249030437A66B2F440AEE0C
:10972000103A2BEE0B8A46F26663C3F6E6630DEE43
:10973000903A28EE0B8A4CF67743C3F22B2309EEBE
:10974000903A8BEE8D9AF2EE0E8A28EE0B8A10E09C
:10975000022E00F02981032E40F02281F0EE6B7A78
:10976000ECEE2D7A67EEAA7AE5EC017AAF4200F0D2
:10977000A6802B6807EE903AE36905EE903AA3695C
:1097800006EE103AE36A04EE103A23680AEE903AC5
:1097900063680EEE103AA3680FEE103AE3680EEE1F
:1097A000903A236A0CEE103A636907EE103A27EEFE
:1097B000287A37EEE55A27EE0A7AF0EE4E3A25EE91
:1097C000075A37EE2B7AEBEE2A3A636AC5EE076A40
:1097D000B0EE4F7A75EEA65AABEE237AE5EEED7A4F
:1097E00074EE2B4A77EEC67AB0EE6E5A67EE847A44
:1097F000ABEE075A87EEA47A29EE455A36EE076A91
:10980000F0EE6B3AF0EE467AE5EE0C7AECEE083AC2
:1098100076EEA55AC7EEA36A37EE066A76EEA96A17
:1098200007EE903A76EEEA6AC4ED075AEBEE26AA06
:1098300084ED066AB0EE6A0AABEE260A20EE270A2D
:1098400016F06EF97AEECE7AA36A67EEAC7A07EE7E
:10985000103A27EE000A87EE8D7A012E84ED000A79
:1098600077EE0E7A37EECF6A37EE277A26EE2C6A3D
:1098700084ED017AC6EE0D6A36EE8F7A77EE6E5A77
:1098800076EE876A65EEAC5AC4ED026A85EE8D6AA3
:1098900076EE2E6A36EE266A84ED036A74D03FF7C0
:1098A00057AF002E7CD1636B06EE103A66EE077A56
:1098B0003BEEC66AE6EE267AF0EE67AA4EE7BDEC0E
:1098C000108BF8BD4BF61423B7EE008AC4F23F03A9
:1098D00009EE103A38EE400AF3EE038A20EE090A48
:1098E00016F046FD30EE480A4BF22D2380EE286A32
:1098F000C3F67D7307EE103A002307EE903AE6EECA
:10990000077A236FF0EE0C6A77EE677A06EE103A6C
:1099100027EEA67A26EE090AC4ED107A84ED087ABD
:1099200016F026FD30EE480A4FF4784380EE286AA0
:10993000C4F2936306EE903A0023C4F2702307EE5C
:10994000903A40F6DB73C4F24903E6EE267A07EE5E
:10995000103A636906EE903A27EEA60A20EE070A4F
:1099600016F054FA216C226F636F84ED0F0A07EE34
:10997000901A38EE678AF0EE40CABDEEC88AE264FB
:10998000A36484ED188ABAE6636B06EE903A66EE3D
:10999000A77A7BEEE66AE6EE877AF0EE67AADDE666
:1099A00000230AEE903AD9E6636B06EE903A6AEE2F
:1099B000A6AA7BEEE66AE6EEA7AACFE630EE600A3C
:1099C00032EE612A31EE601A20EE022A82EE010A9E
:1099D00030EE210A704700BF00B583B012F0E4F802
:1099E0004AF23472C2F2010241F6846312680192B3
:1099F000C2F20103019A1A6003B05DF804FB00BFD4
:109A00002DE9F04340F21D07C2F201078DB03B780B
:109A1000002B40F094854DF63856C2F20006694698
:109A20000A22307919F058FD04461AF089F9C0B2BB
:109A30000228024628BF0222C2F1020006AB2146DC
:109A40001844002443F2300306940794ADF818300C
:109A5000089409940A948DF82C401AF0DFF941F625
:109A6000805022462146C2F2010010F04FFF06A8A6
:109A70001AF066F9024641F6805006A9C2F20100CA
:109A800011F01CFE4EF2C00023460A222146C2F20B
:109A9000000011F099FE44F6F8200121C0F2020006
:109AA00015F0D0F94EF2C00023460A222146C2F238
:109AB000000011F089FE44F6E8500321C0F20200D4
:109AC00015F0C0F906A81AF03BF9014606A815F0F2
:109AD000B9F944F698100121C0F2020015F0B2F96C
:109AE0004EF2C000C2F2000011F05CFE41F6805060
:109AF00022460221C2F201004FF020090694079489
:109B0000089409940A948DF82C408DF8189010F060
:109B1000FDFE06A81AF014F9024641F6805006A987
:109B2000C2F2010011F0CAFD4EF2C00023460A2223
:109B30002146C2F2000011F047FE44F6F820012150
:109B4000C0F2020015F07EF94EF2C00023460A2250
:109B50000221C2F2000011F037FE44F6E850032162
:109B6000C0F2020015F06EF906A81AF0E9F80146F5
:109B700006A815F067F944F698100121C0F202001A
:109B800015F060F94EF2C000C2F2000011F00AFEBA
:109B9000337940F2300003EB43024DF6365803EBC5
:109BA0008203C2F2010041F6D831C2F20008184423
:109BB000C2F2010106F000FA98F8005041F6805018
:109BC00015F0FD05C2F2010000F0D082224602210C
:109BD00006940794089409940A948DF82C408DF803
:109BE000189010F093FE06A81AF0AAF8024641F663
:109BF000805006A9C2F2010011F060FD4EF2C000D3
:109C000023460A222146C2F2000011F0DDFD44F68F
:109C1000F8200121C0F2020015F014F94EF2C00044
:109C200023460A220221C2F2000011F0CDFD44F6C3
:109C3000E8500321C0F2020015F004F906A81AF05A
:109C40007FF8014606A815F0FDF844F698100121AA
:109C5000C0F2020015F0F6F84EF2C000C2F20000A9
:109C600011F0A0FD41F6D830C2F201001AF068F8F8
:109C7000C2B2082A41F6D83128BF08224FF020335B
:109C8000C2F2010106A8069307940894CDF81B3090
:109C900009940A948DF82C401AF0C0F841F68050CF
:109CA00022460321C2F2010010F030FE06A81AF08D
:109CB00047F8024641F6805006A9C2F2010011F0B1
:109CC000FDFC4EF2C00023460A222146C2F20000EB
:109CD00011F07AFD44F6F8200121C0F2020015F0DF
:109CE000B1F84EF2C00023460A220321C2F200005E
:109CF00011F06AFD44F6E8500321C0F2020015F0AD
:109D0000A1F806A81AF01CF8014606A815F09AF862
:109D100044F698100121C0F2020015F093F84EF2BB
:109D2000C000C2F2000011F03DFD41F68050224615
:109D30000B21C2F2010006940794089409940A9436
:109D40008DF82C408DF8189010F0E0FD06A819F061
:109D5000F7FF024641F6805006A9C2F2010011F059
:109D6000ADFC4EF2C00023460A222146C2F200009A
:109D700011F02AFD44F6F820C0F20200012115F08E
:109D800061F823464EF2C0000A220B21C2F2000005
:109D900011F01AFD44F6E8500321C0F2020015F05C
:109DA00051F806A819F0CCFF014606A815F04AF8AC
:109DB00044F698100121C0F2020015F043F84EF26B
:109DC000C000C2F2000011F0EDFC707969460A2271
:109DD000013019F081FB044619F0B2FFC0B202282D
:109DE000024628BF0222C2F1020006AB21461844F7
:109DF000002443F2300306940794ADF81830089419
:109E000009940A948DF82C401AF008F841F6805015
:109E100021460122C2F2010010F078FD06A819F0D7
:109E20008FFF024641F6805006A9C2F2010011F0F0
:109E300045FC4EF2C00023460A220121C2F2000076
:109E400011F0C2FC44F6F8200121C0F2020014F027
:109E5000F9FF4EF2C00023460A222146C2F200005A
:109E600011F0B2FC44F6E8500321C0F2020014F0F5
:109E7000E9FF06A819F064FF014606A814F0E2FF06
:109E800044F698100121C0F2020014F0DBFF4EF2FC
:109E9000C000C2F2000011F085FC41F680500122A2
:109EA0000221C2F201002025069407940894099427
:109EB0000A948DF82C408DF8185010F027FD06A854
:109EC00019F03EFF024641F6805006A9C2F2010099
:109ED00011F0F4FB4EF2C00023460A220121C2F227
:109EE000000011F071FC44F6F8200121C0F20200DC
:109EF00014F0A8FF4EF2C00023460A220221C2F24B
:109F0000000011F061FC44F6E8500321C0F20200A9
:109F100014F098FF06A819F013FF014606A814F0E4
:109F200091FF44F698100121C0F2020014F08AFF5C
:109F30004EF2C000C2F2000011F034FC98F800802C
:109F400008F0FD084DF6385641F68050B8F1010F83
:109F5000C2F20006C2F2010000F0E78101220221F4
:109F600006940794089409940A948DF82C408DF86F
:109F7000185010F0CBFC06A819F0E2FE024641F69C
:109F8000805006A9C2F2010011F098FB4EF2C00009
:109F900023460A220121C2F2000011F015FC44F60A
:109FA000F8200121C0F2020014F04CFF4EF2C00074
:109FB00023460A220221C2F2000011F005FC44F6F9
:109FC000E8500321C0F2020014F03CFF06A819F08B
:109FD000B7FE014606A814F035FF44F6981001219B
:109FE000C0F2020014F02EFF4EF2C000C2F20000D8
:109FF00011F0D8FB727941F6144302EB820602EBB2
:10A000004606C2F201031E44304619F099FEC2B260
:10A010000A2A28BF0A224FF02033314606A80693A9
:10A020000793089409940A948DF82C408DF82050D9
:10A0300019F0F4FE41F6805001220321C2F2010022
:10A0400010F064FC06A819F07BFE024641F6805031
:10A0500006A9C2F2010011F031FB4EF2C000234606
:10A060000A220121C2F2000011F0AEFB44F6F820F2
:10A070000121C0F2020014F0E5FE4EF2C0002346BA
:10A080000A220321C2F2000011F09EFB44F6E850C0
:10A090000321C0F2020014F0D5FE06A819F050FE0C
:10A0A000014606A814F0CEFE44F698100121C0F235
:10A0B000020014F0C7FE4EF2C000C2F2000011F020
:10A0C00071FB41F6805001220E21C2F2010006947C
:10A0D0000794089409940A948DF82C408DF8185030
:10A0E00010F014FC06A819F02BFE024641F6805031
:10A0F00006A9C2F2010011F0E1FA4EF2C0002346B7
:10A100000A220121C2F2000011F05EFB44F6F820A1
:10A110000121C0F2020014F095FE4EF2C000234669
:10A120000A220E21C2F2000011F04EFB44F6E85064
:10A130000321C0F2020014F085FE06A819F000FE0B
:10A14000014606A814F07EFE44F698100121C0F2E4
:10A15000020014F077FE4EF2C000C2F2000011F0CF
:10A1600021FB00233B700DB0BDE8F0835B232A4642
:10A170000221069507958DF81830089509950A95DE
:10A180008DF82C5010F0C2FB06A819F0D9FD02463C
:10A1900041F6805006A9C2F2010011F08FFA4EF28A
:10A1A000C0002B460A222946C2F2000011F00CFB27
:10A1B00044F6F8200121C0F2020014F043FE4EF2F2
:10A1C000C0002B460A220221C2F2000011F0FCFA64
:10A1D00044F6E8500321C0F2020014F033FE06A852
:10A1E00019F0AEFD014606A814F02CFE44F69810B6
:10A1F0000121C0F2020014F025FE4EF2C000C2F2AE
:10A20000000011F0CFFA41F6D830C2F2010019F087
:10A2100097FDC2B2082A41F6D83128BF08224FF074
:10A220002033C2F2010106A8069307950895CDF8E0
:10A230001B3009950A958DF82C5019F0EFFD41F669
:10A2400080502A460321C2F2010010F05FFB06A8ED
:10A2500019F076FD024641F6805006A9C2F20100CF
:10A2600011F02CFA4EF2C0002B460A222946C2F207
:10A27000000011F0A9FA44F6F8200121C0F2020012
:10A2800014F0E0FD4EF2C0002B460A220321C2F278
:10A29000000011F099FA44F6E8500321C0F20200E0
:10A2A00014F0D0FD06A819F04BFD014606A814F0E5
:10A2B000C9FD44F698100121C0F2020014F0C2FD5D
:10A2C0004EF2C000C2F2000011F06CFA41F680506C
:10A2D0005D232A460B21C2F20100069507958DF8F1
:10A2E0001830089509950A958DF82C5010F00EFB42
:10A2F00006A819F025FD024641F6805006A9C2F2D3
:10A30000010011F0DBF94EF2C0002B460A2229466B
:10A31000C2F2000011F058FA44F6F820C0F2020030
:10A32000012114F08FFD2B462CE55B2342460221D0
:10A33000069407948DF81830089409940A948DF8BF
:10A340002C4010F0E3FA06A819F0FAFC024641F698
:10A35000805006A9C2F2010011F0B0F94EF2C0001F
:10A3600023460A224146C2F2000011F02DFA44F6BB
:10A37000F8204146C0F2020014F064FD4EF2C00025
:10A3800023460A220221C2F2000011F01DFA44F60F
:10A39000E8500321C0F2020014F054FD06A819F0A1
:10A3A000CFFC014606A814F04DFD44F69810414636
:10A3B000C0F2020014F046FD4EF2C000C2F20000EE
:10A3C00011F0F0F9727941F6144302EB820602EBC8
:10A3D0004606C2F201031E44304619F0B1FCC2B277
:10A3E0000A2A28BF0A224FF02033314606A80693D6
:10A3F0000793089409940A948DF82C408DF8205006
:10A4000019F00CFD41F6805042460321C2F20100D2
:10A4100010F07CFA06A819F093FC024641F6805031
:10A4200006A9C2F2010011F049F94EF2C00023461C
:10A430000A224146C2F2000011F0C6F944F6F820A3
:10A440004146C0F2020014F0FDFC4EF2C00023466B
:10A450000A220321C2F2000011F0B6F944F6E850D6
:10A460000321C0F2020014F0EDFC06A819F068FC0C
:10A47000014606A814F0E6FC44F698104146C0F2E6
:10A48000020014F0DFFC4EF2C000C2F2000011F036
:10A4900089F941F680505D2342460E21C2F2010047
:10A4A000069407948DF81830089409940A948DF84E
:10A4B0002C4010F02BFA06A819F042FC024641F697
:10A4C000805006A9C2F2010011F0F8F84EF2C00067
:10A4D00023460A224146C2F2000011F075F944F603
:10A4E000F8204146C0F2020014F0ACFC4EF2C0006D
:10A4F00023460A220E21C2F2000011F065F944F64B
:10A50000E8500321C0F2020014F09CFC06A819F0E8
:10A5100017FC014606A814F095FC44F69810414635
:10A52000C0F2020014F08EFC4EF2C000C2F2000035
:10A5300011F038F900233B700DB0BDE8F08341F60F
:10A540008050C2F2010010F0D5F9FFF764BA00BFE5
:10A550002DE9F0412DED028B4AF23473C2F2010372
:10A5600040F21D0790B0C2F201071B6803933A78CE
:10A57000039941F68463C2F20103012A196000F0D5
:10A58000C38141F68050C2F2010010F0B3F944F6E5
:10A590006473C0F2020393E803000AAC00254FF095
:10A5A0002033A3606360E5602561C4F80B30257536
:10A5B0000A9041F680502A46ADF82C10C2F20100F4
:10A5C000294610F0A3F9204619F0BAFB024641F6DD
:10A5D00080502146C2F2010011F070F84EF2C00026
:10A5E0002B460A222946C2F2000011F0EDF844F68B
:10A5F000F8200121C0F2020014F024FC4EF2C00049
:10A600002B460A222946C2F2000011F0DDF844F67A
:10A61000E8500321C0F2020014F014FC204619F0A7
:10A620008FFB0146204614F00DFC44F69810C0F252
:10A630000200012114F006FC4EF2C000C2F200003C
:10A6400011F0B0F84DF63858C2F20008D8ED027A91
:10A650009FEDE08ADFEDE08A67EE887A0A22FDEE60
:10A66000E77A04A917EE900A18F036FF054619F0AC
:10A6700067FBC0B20328024628BF0322C2F10300D1
:10A6800043F23003C0F230032946204400250A95E6
:10A690006560A560E56025612575ADF82830A3707B
:10A6A00019F0BCFB41F680502A460D21C2F2010090
:10A6B00010F02CF9204619F043FB024641F6805079
:10A6C0002146C2F2010010F0F9FF4EF2C0002B4605
:10A6D0000A222946C2F2000011F076F844F6F8206A
:10A6E0000121C0F2020014F0ADFB4EF2C0002B4677
:10A6F0000A220D21C2F2000011F066F844F6E8507B
:10A700000321C0F2020014F09DFB204619F018FB53
:10A710000146204614F096FB44F698100121C0F241
:10A72000020014F08FFB4EF2C000C2F2000011F0E4
:10A7300039F8D8ED027AF4EE687AF1EE10FA00F00A
:10A74000E5809FEDA67AF4EEC77AF1EE10FA00F1FB
:10A75000328167EE887AB3EE007A27EE877AC7EE09
:10A76000087A77EEA87AF5EEC07AF1EE10FA67DD96
:10A7700041F6805000262A2329460122C2F2010018
:10A7800026606660A660E660266126758DF8283032
:10A7900010F0BCF8204619F0D3FA024641F680507A
:10A7A0002146C2F2010010F089FF4EF2C00033468C
:10A7B0000A220121C2F2000011F006F844F6F82046
:10A7C0000121C0F2020014F03DFB4EF2C0003346FE
:10A7D0000A222946C2F2000010F0F6FF44F6E850C3
:10A7E0000321C0F2020014F02DFB204619F0A8FA54
:10A7F0000146204614F026FB44F698100121C0F2D1
:10A80000020014F01FFB4EF2C000C2F2000010F074
:10A81000C9FFD8ED027A67EE887AB3EE007A67EE68
:10A82000877A013587EE887AEDB207EE905AF8EE16
:10A83000E76A77EE287AF4EEE76AF1EE10FA97D439
:10A84000FCEEE77ACDED017A9DF804600F2E54D826
:10A8500041F680500025202331460122C2F201003A
:10A8600025606560A560E560256125758DF8283057
:10A8700010F04CF8204619F063FA024641F6805079
:10A880002146C2F2010010F019FF4EF2C0002B4623
:10A890000A220121C2F2000010F096FF44F6F820CF
:10A8A0000121C0F2020014F0CDFA4EF2C0002B4696
:10A8B0000A223146C2F2000010F086FF44F6E8504A
:10A8C0000321C0F2020014F0BDFA204619F038FA54
:10A8D0000146204614F0B6FA44F698100121C0F261
:10A8E000020014F0AFFA01364EF2C000C2F20000CE
:10A8F000F6B210F057FF102EAAD101233B7010B012
:10A90000BDEC028BBDE8F0810AAC9BE64FF0203332
:10A9100041F68050E56025612575C2F201000A9379
:10A92000202601222946A3606360C4F80B308DF80D
:10A9300028600FF0EBFF204619F002FA024641F6BC
:10A9400080502146C2F2010010F0B8FE4EF2C00065
:10A950002B460A220121C2F2000010F035FF44F616
:10A96000F8200121C0F2020014F06CFA4EF2C0008F
:10A970002B460A222946C2F2000010F025FF44F6B9
:10A98000E8500321C0F2020014F05CFA204619F0EE
:10A99000D7F90146204614F055FA44F698100121E3
:10A9A000C0F2020014F04EFA4EF2C000C2F20000F3
:10A9B00010F0F8FEA1E74FF0203341F68050C2F2CC
:10A9C00001002A2601222946E56025612575A3603C
:10A9D0002360A9E70000C842000000000AD7233E18
:10A9E0002DE9F04140F21D06C2F201068CB0337829
:10A9F000032B00F03E8341F68050C2F201000FF0BD
:10AA000079FF44F66C73C0F2020393E8030006ACCE
:10AA100000254FF02033A3606360E5602561C4F832
:10AA20000B302575069041F680502A46ADF81C1073
:10AA3000C2F2010029460FF069FF204619F080F9A3
:10AA4000024641F680502146C2F2010010F036FE67
:10AA50004EF2C0002B460A222946C2F2000010F036
:10AA6000B3FE44F6F8200121C0F2020014F0EAF926
:10AA70004EF2C0002B460A222946C2F2000010F016
:10AA8000A3FE44F6E8500321C0F2020014F0DAF904
:10AA9000204619F055F90146204614F0D3F944F642
:10AAA00098100121C0F2020014F0CCF94EF2C0005F
:10AAB000C2F2000010F076FE46F2525341F680508A
:10AAC000C3F6732329460122C2F201006560A56026
:10AAD000E5602561257506930FF018FF204619F0F3
:10AAE0002FF9024641F680502146C2F2010010F0D3
:10AAF000E5FD4EF2C0002B460A220121C2F2000001
:10AB000010F062FE44F6F8200121C0F2020014F0B9
:10AB100099F94EF2C0002B460A222946C2F20000E3
:10AB200010F052FE44F6E8500321C0F2020014F087
:10AB300089F9204619F004F90146204614F082F9FB
:10AB400044F698100121C0F2020014F07BF94EF295
:10AB5000C000C2F2000010F025FE47F2435341F658
:10AB60008050C3F6742301220821C2F201006560FF
:10AB7000A560E5602561257506930FF0C7FE2046A8
:10AB800019F0DEF8024641F680502146C2F201007B
:10AB900010F094FD4EF2C0002B460A220121C2F2B1
:10ABA000000010F011FE44F6F8200121C0F202006E
:10ABB00014F048F94EF2C0002B460A220821C2F2D6
:10ABC000000010F001FE44F6E8500321C0F202003C
:10ABD00014F038F9204619F0B3F80146204614F075
:10ABE00031F944F69810C0F20200012114F02AF95C
:10ABF0004EF2C000C2F2000010F0D4FD41F6114345
:10AC0000C2F201034FF2CB081B7803EB830303EB83
:10AC10008303C2F68D089B0088FB0320DB17C3EB80
:10AC2000201069460A2218F057FC054619F088F8EA
:10AC3000C0B20228024628BF0222C2F10200294601
:10AC400043F230070025204406956560A560E56065
:10AC500025612575ADF8187019F0E0F841F68050BF
:10AC600001220521C2F201000FF050FE204619F02A
:10AC700067F8024641F680502146C2F2010010F00A
:10AC80001DFD4EF2C0002B460A220121C2F2000037
:10AC900010F09AFD44F6F8200121C0F2020014F0F1
:10ACA000D1F84EF2C0000A222B460521C2F2000064
:10ACB00010F08AFD44F6E8500321C0F2020014F0BF
:10ACC000C1F8204619F03CF80146204614F0BAF8C5
:10ACD00044F698100121C0F2020014F0B3F84EF2CD
:10ACE000C000C2F2000010F05DFD40F21C03C2F291
:10ACF000010369461B7803EB830303EB83039B008B
:10AD000088FB0320DB17C3EB20100A2218F0E4FBBA
:10AD1000804619F015F8C0B20228024628BF022268
:10AD2000C2F102004146204406956560A560E560D9
:10AD300025612575ADF8187019F070F841F680504E
:10AD400001220D21C2F201000FF0E0FD204618F0B3
:10AD5000F7FF024641F680502146C2F2010010F092
:10AD6000ADFC4EF2C0002B460A220121C2F20000C7
:10AD700010F02AFD44F6F8200121C0F2020014F080
:10AD800061F84EF2C0002B460A220D21C2F20000EB
:10AD900010F01AFD44F6E8500321C0F2020014F04E
:10ADA00051F8204618F0CCFF0146204614F04AF82E
:10ADB00044F698100121C0F202004DF6365714F007
:10ADC00041F8C2F200074EF2C000C2F2000010F0DB
:10ADD000E9FC97F8008041F68050B8F1040FC2F208
:10ADE000010000F04881012204214FF0200806955F
:10ADF0006560A560E560256125758DF818800FF008
:10AE000085FD204618F09CFF024641F68050214601
:10AE1000C2F2010010F052FC4EF2C0002B460A2292
:10AE20000121C2F2000010F0CFFC44F6F82001210D
:10AE3000C0F2020014F006F84EF2C0000A222B46BF
:10AE40000421C2F2000010F0BFFC44F6E8500321D8
:10AE5000C0F2020013F0F6FF204618F071FF014621
:10AE6000204613F0EFFF44F698100121C0F20200D3
:10AE700013F0E8FF4EF2C000C2F2000010F092FCA6
:10AE800041F680500695C2F201006560A560E5605C
:10AE900025612575012207218DF818800FF036FDF8
:10AEA000204618F04DFF024641F680502146C2F27E
:10AEB000010010F003FC4EF2C0002B460A220121D3
:10AEC000C2F2000010F080FC44F6F8200121C0F22C
:10AED000020013F0B7FF4EF2C0002B460A220721F2
:10AEE000C2F2000010F070FC44F6E8500321C0F2FA
:10AEF000020013F0A7FF204618F022FF014620466B
:10AF000013F0A0FF44F698100121C0F2020013F0E4
:10AF100099FF4EF2C000C2F2000010F043FC3B78F3
:10AF200041F68050052B4FF00005C2F2010000F001
:10AF3000FE8001220C21202706956560A560E56052
:10AF4000256125758DF818700FF0E0FC204618F08B
:10AF5000F7FE024641F680502146C2F2010010F091
:10AF6000ADFB4EF2C0002B460A220121C2F20000C6
:10AF700010F02AFC44F6F8200121C0F2020013F080
:10AF800061FF4EF2C0000A222B460C21C2F20000E3
:10AF900010F01AFC44F6E8500321C0F2020013F04E
:10AFA00051FF204618F0CCFE0146204613F04AFF20
:10AFB00044F698100121C0F2020013F043FF4EF254
:10AFC000C000C2F2000010F0EDFB41F68050069583
:10AFD000C2F201006560A560E5602561257501226A
:10AFE0000F218DF818700FF091FC204618F0A8FE84
:10AFF000024641F680502146C2F2010010F05EFB8D
:10B000004EF2C0002B460A220121C2F2000010F0CD
:10B01000DBFB44F6F8200121C0F2020013F012FF1E
:10B020004EF2C0002B460A220F21C2F2000010F09F
:10B03000CBFB44F6E8500321C0F2020013F002FFFC
:10B04000204618F07DFE0146204613F0FBFE44F634
:10B0500098100121C0F2020013F0F4FE4EF2C0007D
:10B06000C2F2000010F09EFB032333700CB0BDE869
:10B07000F08106ACC2E55B2301224146069565607E
:10B08000A560E560256125758DF818300FF03EFC50
:10B09000204618F055FE024641F680502146C2F285
:10B0A000010010F00BFB4EF2C0002B460A220121DA
:10B0B000C2F2000010F088FB44F6F8200121C0F233
:10B0C000020013F0BFFE4EF2C0002B460A2241469A
:10B0D000C2F2000010F078FB44F6E8500321C0F201
:10B0E000020013F0AFFE204618F02AFE014620466B
:10B0F00013F0A8FE44F698100121C0F2020013F0EC
:10B10000A1FE4EF2C000C2F2000010F04BFB41F66F
:10B1100080505D230695C2F201006560A560E56080
:10B1200025612575012207218DF81830B6E65B23CD
:10B1300001220C2106956560A560E56025612575F5
:10B140008DF818300FF0E2FB204618F0F9FD0246AA
:10B1500041F680502146C2F2010010F0AFFA4EF2E3
:10B16000C0002B460A220121C2F2000010F02CFB85
:10B1700044F6F8200121C0F2020013F063FE4EF203
:10B18000C0002B460A220C21C2F2000010F01CFB6A
:10B1900044F6E8500321C0F2020013F053FE2046AB
:10B1A00018F0CEFD0146204613F04CFE44F69810F0
:10B1B0000121C0F2020013F045FE4EF2C000C2F2BF
:10B1C000000010F0EFFA41F680505D230695C2F2C0
:10B1D00001006560A560E5602561257501220F21EC
:10B1E0008DF81830FFE600BFF0B54AF23473C2F2B2
:10B1F000010340F21D068FB0C2F201061B680193E5
:10B200003278019941F68463C2F20103022A19607F
:10B2100000F0D18041F68050C2F201000FF06AFBCD
:10B2200044F67473C0F2020393E8070008AC0025EB
:10B230004FF02033E560C4F80B3084E8070041F696
:10B2400080502A462946C2F20100256125750FF07B
:10B250005DFB204618F074FD024641F68050214601
:10B26000C2F2010010F02AFA4EF2C0002B46294625
:10B270000A22C2F2000010F0A7FA44F6F8200121D9
:10B28000C0F2020013F0DEFD4EF2C0002B460A228F
:10B290002946C2F2000010F097FA44F6E850032164
:10B2A000C0F2020013F0CEFD204618F049FD014621
:10B2B000204613F0C7FD44F698100121C0F20200A9
:10B2C0004DF6385713F0BEFDC2F200074EF2C00033
:10B2D000C2F2000010F066FA3D7C002D73D00A2205
:10B2E00002A9284618F0F8F8054618F029FDC0B262
:10B2F0000228024628BF0222C2F1020043F23003B4
:10B3000029462044002508956560A560E560256113
:10B310002575ADF8203018F081FD41F680502946A2
:10B320000122C2F201000FF0F1FA204618F008FDE8
:10B33000024641F680502146C2F2010010F0BEF9EB
:10B340004EF2C0002B460A220121C2F2000010F08A
:10B350003BFA44F6F8200121C0F2020013F072FD1E
:10B360004EF2C0002B460A222946C2F2000010F01D
:10B370002BFA44F6E8500321C0F2020013F062FDFC
:10B38000204618F0DDFC0146204613F05BFD44F634
:10B3900098100121C0F2020013F054FD4EF2C000DB
:10B3A000C2F2000010F0FEF93F7C012F60D00223B2
:10B3B00033700FB0F0BD4DF63857C2F2000708AC3D
:10B3C0003D7C002D8BD144F64F5341F68050C4F69E
:10B3D0004E1329460122C2F201006560A560E560B6
:10B3E0002561257508930FF091FA204618F0A8FC06
:10B3F000024641F680502146C2F2010010F05EF98B
:10B400004EF2C0002B460A220121C2F2000010F0C9
:10B41000DBF944F6F8200121C0F2020013F012FD1E
:10B420004EF2C0002B460A222946C2F2000010F05C
:10B43000CBF944F6E8500321C0F2020013F002FDFC
:10B44000204618F07DFC0146204613F0FBFC44F634
:10B4500098100121C0F2020013F0F4FC4EF2C0007B
:10B46000C2F2000010F09EF9022333700FB0F0BD5D
:10B4700041F6805042F220033A460221C2F2010016
:10B4800008956560A560E56025612575ADF82030FB
:10B490000FF03CFA204618F053FC024641F680506B
:10B4A0002146C2F2010010F009F94EF2C0002B460D
:10B4B0000A223946C2F2000010F086F944F6F8205C
:10B4C0003946C0F2020013F0BDFC4EF2C0002B461C
:10B4D0000A220221C2F2000010F076F944F6E85088
:10B4E0000321C0F2020013F0ADFC204618F028FC46
:10B4F0000146204613F0A6FC44F698103946C0F2E7
:10B50000020013F09FFC4EF2C000C2F2000010F0E7
:10B5100049F9022333700FB0F0BD00BF2DE9F041AF
:10B5200040F21D06C2F201068CB03378042B00F005
:10B53000F88441F68050C2F201000FF0DBF944F6C6
:10B540008473C0F2020393E8030006AC0025656033
:10B55000A560E56025612575069041F680502A4674
:10B560008DF81C10C2F2010029460FF0CFF92046D9
:10B5700018F0E6FB024641F680502146C2F2010077
:10B5800010F09CF84EF2C0002B460A222946C2F267
:10B59000000010F019F944F6F8200121C0F2020071
:10B5A00013F050FC4EF2C0002B460A222946C2F28C
:10B5B000000010F009F944F6E8500321C0F202003F
:10B5C00013F040FC204618F0BBFB0146204613F068
:10B5D00039FC44F698100121C0F2020013F032FC4D
:10B5E0004EF2C000C2F2000010F0DCF841F68050CC
:10B5F00043F654232A460621C2F2010006956560EF
:10B60000A560E56025612575ADF818300FF07EF96D
:10B61000204618F095FB024641F680502146C2F2C2
:10B62000010010F04BF84EF2C0002B460A222946CA
:10B63000C2F2000010F0C8F844F6F8200121C0F270
:10B64000020013F0FFFB4EF2C0002B460A22062137
:10B65000C2F2000010F0B8F844F6E8500321C0F23E
:10B66000020013F0EFFB204618F06AFB014620466B
:10B6700013F0E8FB44F698100121C0F2020013F029
:10B68000E1FB4EF2C000C2F2000010F08BF841F670
:10B69000805047F26D332A460E21C2F20100069512
:10B6A0006560A560E56025612575ADF818300FF07F
:10B6B0002DF9204618F044FB024641F68050214601
:10B6C000C2F201000FF0FAFF4EF2C0002B460A2230
:10B6D0002946C2F2000010F077F844F6F820012164
:10B6E000C0F2020013F0AEFB4EF2C0002B460A225D
:10B6F0000E21C2F2000010F067F844F6E850032172
:10B70000C0F2020013F09EFB204618F019FB014620
:10B71000204613F097FB44F698100121C0F2020076
:10B7200013F090FB4EF2C000C2F2000010F03AF8A5
:10B7300044F68C73C0F2020341F680501B680695F4
:10B740001F0C29460122C2F201006560A560E56078
:10B7500025612575ADF818308DF81A700FF0D6F800
:10B76000204618F0EDFA024641F680502146C2F21A
:10B7700001000FF0A3FF4EF2C0002B460A22012168
:10B78000C2F2000010F020F844F6F8200121C0F2C7
:10B79000020013F057FB4EF2C0002B460A22294646
:10B7A000C2F2000010F010F844F6E8500321C0F295
:10B7B000020013F047FB204618F0C2FA014620466B
:10B7C00013F040FB44F698100121C0F2020013F080
:10B7D00039FB4EF2C000C2F200000FF0E3FF46F664
:10B7E000567341F68050C3F66C2301220821C2F241
:10B7F00001006560A560E5602561257506930FF081
:10B8000085F8204618F09CFA024641F68050214601
:10B81000C2F201000FF052FF4EF2C0002B460A2286
:10B820000121C2F200000FF0CFFF44F6F820012101
:10B83000C0F2020013F006FB4EF2C0002B460A22B3
:10B840000821C2F200000FF0BFFF44F6E8500321C8
:10B85000C0F2020013F0F6FA204618F071FA014621
:10B86000204613F0EFFA44F69810C0F202000121CE
:10B8700013F0E8FA4EF2C000C2F200000FF092FF9F
:10B8800040F24452C2F201024FF49663107848F23B
:10B890001F57C5F2EB1703FB00F387FB0320DB17F1
:10B8A000C3EB201069460A2217F016FE054618F071
:10B8B00047FAC0B20428024628BF0422C2F104009D
:10B8C0004FF030332946204400256560A560E560CF
:10B8D00025612575069318F0A1FA41F680502A4695
:10B8E0000921C2F201000FF011F8204618F028FAE1
:10B8F000024641F680502146C2F201000FF0DEFE02
:10B900004EF2C0002B460A222946C2F200000FF078
:10B910005BFF44F6F8200121C0F2020013F092FA16
:10B920004EF2C0000A222B460921C2F200000FF09D
:10B930004BFF44F6E8500321C0F2020013F082FAF4
:10B94000204618F0FDF90146204613F07BFA44F634
:10B9500098100121C0F2020013F074FA4EF2C000F8
:10B96000C2F200000FF01EFF41F61043C2F20103C5
:10B970004AF2EB001B7803EB430303EB4313CEF6D1
:10B980000E2080FB03201844DB17C3EB60106946D0
:10B990000A2217F0A1FD804618F0D2F9C0B20228A1
:10B9A000024628BF0222C2F102004146204443F26F
:10B9B000300806956560A560E56025612575ADF8E0
:10B9C000188018F02BFA41F6805001220421C2F2AF
:10B9D00001000EF09BFF204618F0B2F9024641F636
:10B9E00080502146C2F201000FF068FE4EF2C00006
:10B9F0002B460A220121C2F200000FF0E5FE44F6B8
:10BA0000F8200121C0F2020013F01CFA4EF2C0002F
:10BA10000A222B460421C2F200000FF0D5FE44F6A4
:10BA2000E8500321C0F2020013F00CFA204618F08F
:10BA300087F90146204613F005FA44F698100121D3
:10BA4000C0F2020013F0FEF94EF2C000C2F2000094
:10BA50000FF0A8FE41F69453C2F2010369461B7829
:10BA600003EB430303EB431387FB0320DB17C3EB19
:10BA700020100A2217F030FD074618F061F9C0B215
:10BA80000228024628BF0222C2F1020039462044A1
:10BA900006956560A560E56025612575ADF818809F
:10BAA00018F0BCF941F6805001220D21C2F20100CC
:10BAB0000EF02CFF204618F043F9024641F6805064
:10BAC0002146C2F201000FF0F9FD4EF2C0002B46F4
:10BAD0000A220121C2F200000FF076FE44F6F8209F
:10BAE0000121C0F2020013F0ADF94EF2C0002B4666
:10BAF0000A220D21C2F200000FF066FE44F6E85063
:10BB00000321C0F2020013F09DF9204618F018F945
:10BB10000146204613F096F944F698100121C0F230
:10BB200002004DF6365713F08DF9C2F200074EF2BF
:10BB3000C000C2F200000FF035FE3B7841F68050A5
:10BB4000062BC2F2010000F04A822A4608214FF07B
:10BB5000200806956560A560E560256125758DF86E
:10BB600018800EF0D3FE204618F0EAF8024641F69F
:10BB700080502146C2F201000FF0A0FD4EF2C0003D
:10BB80002B460A222946C2F200000FF01DFE44F6A1
:10BB9000F8200121C0F2020013F054F94EF2C00067
:10BBA0000A222B460821C2F200000FF00DFE44F6D7
:10BBB000E8500321C0F2020013F044F9204618F0C7
:10BBC000BFF80146204613F03DF944F698100121D4
:10BBD000C0F2020013F036F94EF2C000C2F20000CB
:10BBE0000FF0E0FD41F680500695C2F2010065605D
:10BBF000A560E560256125752A460D218DF8188020
:10BC00000EF084FE204618F09BF8024641F6805064
:10BC10002146C2F201000FF051FD4EF2C0002B464A
:10BC20000A222946C2F200000FF0CEFD44F6F820A9
:10BC30000121C0F2020013F005F94EF2C0002B46BC
:10BC40000A220D21C2F200000FF0BEFD44F6E850BA
:10BC50000321C0F2020013F0F5F8204618F070F846
:10BC60000146204613F0EEF844F698100121C0F288
:10BC7000020013F0E7F84EF2C000C2F200000FF02D
:10BC800091FD3B7841F68050072B4FF00005C2F242
:10BC9000010000F04881012203214FF020080695A1
:10BCA0006560A560E560256125758DF818800EF04A
:10BCB0002DFE204618F044F8024641F680502146F9
:10BCC000C2F201000FF0FAFC4EF2C0002B460A222D
:10BCD0000121C2F200000FF077FD44F6F8200121A7
:10BCE000C0F2020013F0AEF84EF2C0000A222B465A
:10BCF0000321C2F200000FF067FD44F6E850032173
:10BD0000C0F2020013F09EF8204618F019F8014620
:10BD1000204613F097F844F698100121C0F2020073
:10BD200013F090F84EF2C000C2F200000FF03AFD9E
:10BD300041F680500695C2F201006560A560E5609D
:10BD400025612575012206218DF818800EF0DEFD93
:10BD5000204617F0F5FF024641F680502146C2F218
:10BD600001000FF0ABFC4EF2C0002B460A2201216D
:10BD7000C2F200000FF028FD44F6F8200121C0F2C5
:10BD8000020013F05FF84EF2C0002B460A22062193
:10BD9000C2F200000FF018FD44F6E8500321C0F293
:10BDA000020013F04FF8204617F0CAFF0146204664
:10BDB00013F048F844F698100121C0F2020013F085
:10BDC00041F84EF2C000C2F200000FF0EBFC3B78ED
:10BDD00041F68050082B4FF00005C2F2010000F040
:10BDE0005A8101220C21202706956560A560E56037
:10BDF000256125758DF818700EF088FD204617F026
:10BE00009FFF024641F680502146C2F201000FF02A
:10BE100055FC4EF2C0002B460A220121C2F200005E
:10BE20000FF0D2FC44F6F8200121C0F2020013F01A
:10BE300009F84EF2C0000A222B460C21C2F2000083
:10BE40000FF0C2FC44F6E8500321C0F2020012F0E9
:10BE5000F9FF204617F074FF0146204612F0F2FF6A
:10BE600044F698100121C0F2020012F0EBFF4EF2EE
:10BE7000C000C2F200000FF095FC41F6805006951C
:10BE8000C2F201006560A560E560256125750122AB
:10BE90000F218DF818700EF039FD204617F050FF75
:10BEA000024641F680502146C2F201000FF006FC26
:10BEB0004EF2C0002B460A220121C2F200000FF010
:10BEC00083FC44F6F8200121C0F2020012F0BAFF10
:10BED0004EF2C0002B460A220F21C2F200000FF0E2
:10BEE00073FC44F6E8500321C0F2020012F0AAFFEE
:10BEF000204617F025FF0146204612F0A3FF44F626
:10BF000098100121C0F2020012F09CFF4EF2C00016
:10BF1000C2F200000FF046FC042333700CB0BDE801
:10BF2000F08106ACACE45B23012203210695656039
:10BF3000A560E560256125758DF818300EF0E6FCEA
:10BF4000204617F0FDFE024641F680502146C2F21F
:10BF500001000FF0B3FB4EF2C0002B460A22012174
:10BF6000C2F200000FF030FC44F6F8200121C0F2CC
:10BF7000020012F067FF4EF2C0002B460A22032196
:10BF8000C2F200000FF020FC44F6E8500321C0F29A
:10BF9000020012F057FF204617F0D2FE014620465D
:10BFA00012F050FF44F698100121C0F2020012F086
:10BFB00049FF4EF2C000C2F200000FF0F3FB41F661
:10BFC00080505D230695C2F201006560A560E560C2
:10BFD00025612575012206218DF81830B6E65B2310
:10BFE0002A46082106956560A560E56025612575EE
:10BFF0008DF818300EF08AFC204617F0A1FE02469C
:10C0000041F680502146C2F201000FF057FB4EF27C
:10C01000C0002B460A222946C2F200000FF0D4FBD2
:10C0200044F6F8200121C0F2020012F00BFF4EF29C
:10C03000C0002B460A220821C2F200000FF0C4FB08
:10C0400044F6E8500321C0F2020012F0FBFE204645
:10C0500017F076FE0146204612F0F4FE44F69810E2
:10C060000121C0F2020012F0EDFE4EF2C000C2F259
:10C0700000000FF097FB41F680505D230695C2F259
:10C0800001006560A560E560256125752A460D21E2
:10C090008DF81830B4E55B2301220C21069565600C
:10C0A000A560E560256125758DF818300EF02EFC31
:10C0B000204617F045FE024641F680502146C2F266
:10C0C00001000FF0FBFA4EF2C0002B460A220121BC
:10C0D000C2F200000FF078FB44F6F8200121C0F214
:10C0E000020012F0AFFE4EF2C0002B460A220C21D5
:10C0F000C2F200000FF068FB44F6E8500321C0F2E2
:10C10000020012F09FFE204617F01AFE014620465C
:10C1100012F098FE44F698100121C0F2020012F0CD
:10C1200091FE4EF2C000C2F200000FF03BFB41F660
:10C1300080505D230695C2F201006560A560E56050
:10C140002561257501220F218DF81830A3E600BF67
:10C150002DE9F04F2DED068B4AF23477C2F201073C
:10C1600089B041F684623B680493C2F20102049BE9
:10C17000116840F6B7325B1A934207D940F21D03AB
:10C18000C2F201031B78002B40F0428141F27C484F
:10C19000C2F2010841F690533A680592C2F20103D7
:10C1A00041F287321968059B5B1A934208D94DF614
:10C1B0003654C2F200042378023B012B40F2628124
:10C1C00041F27C44C2F2010441F6F03340F224060D
:10C1D0004BF6836A04F10C02C2F201039FEDAF8AB1
:10C1E0009FEDAF9ADFEDAF8A9FEDAFAADFEDAF9A7B
:10C1F000CDF80480C2F201060093C2F6A07A0025B1
:10C200009046009B03EB051B58460EF0DFF958469D
:10C210005FFA85F90EF020FA38B13B68069341F6D3
:10C22000E833C2F20103069A1A6058460EF00AFA81
:10C23000A0B341F6E8333A680792C2F201031A68E4
:10C24000079B9B1AB3F5FA7F00F2328140F21D037F
:10C25000C2F20103B9F1010F1B7800F0CE80012B6F
:10C2600000F0D083C0F08682022B00F0E483AB465E
:10C2700044F6BC700721C0F2020012F0E3FD4EF25A
:10C28000C0005946C2F2000000230A220FF09CFAB7
:10C290004EF2C000C2F200000FF084FA237C012BA2
:10C2A00040F24D8172B6E36862B6002B56F8042B5B
:10C2B000B8BF0333B2EBA30F5CD0B9F1010F66D165
:10C2C00040F21D02C2F201021378012B00F0B88186
:10C2D000C0F0C982032B00F0CB81042B0FD14DF6A7
:10C2E0003653C2F200031B78072B00F02186082B7F
:10C2F00000F02384062B00F08B86FFF70FF945F240
:10C3000050000821C0F2020012F09CFD4EF2C00065
:10C3100000230A222946C2F200000FF055FA44F623
:10C32000A850C0F20200022112F08CFD237C012BE8
:10C3300040F2468272B6E16862B60029B8BF0331A6
:10C340004EF2C0008910C2F200000FF0CDF94EF29B
:10C35000C000C2F200000FF025FA237C012B40F24E
:10C360005A8272B6E36862B6002BB8BF03339B10E3
:10C3700046F8043C0135022D04F1140408F11408B8
:10C380007FF43FAF09B0BDEC068BBDE8F08F40F203
:10C390001D03C2F201031B78012B40F2F880022B2F
:10C3A000ADD1237C012B40F2B98672B6E36862B648
:10C3B000032B40F3BB84237C012B40F28F8772B6A2
:10C3C000E36862B63F2B03DD72B64023E36062B6DA
:10C3D000237C012B40F2CE8672B6E36862B64DF63E
:10C3E0003852002BC2F20002B8BF03339B10137403
:10C3F000FAF7D4F9FEF7F8FE81E7002B00F0A581EB
:10C40000033B012B4FF0040140F29F82CB462FE704
:10C41000033B012B7FF6BAAE4DF63853C2F2000350
:10C4200093ED027ADFED1D6ADFED1D7A9FED1D6A47
:10C4300027EE267A27EE277AC7EE267A77EE867AD7
:10C44000FDEEE77A17EE903A9B0072B641F27C4817
:10C45000C2F20108C8F80C3062B698F81030012B0F
:10C4600040F29E8272B6D8F80C3062B640F22402D6
:10C47000002BC2F20102B8BF03339B101360FDF71B
:10C48000BFFA87E6FDF7BCFA2378022B00F0D580CF
:10C49000032B7FF495AE0123237091E60000C84280
:10C4A00000002C420000000000000C4200FEFF468D
:10C4B00044F690702921C0F2020012F0C3FC4EF243
:10C4C000C00000230A222946C2F200000FF07CF9C6
:10C4D0004EF2C000C2F200000FF064F9B9F1010F92
:10C4E000AB467FF4C5AE40F21D03C2F201031B78D8
:10C4F000032B00F04A84042B00F02884002B7FF4E7
:10C50000B7AE4DF6365241F61143C2F20002C2F206
:10C510000103042111701B7872B69B00E36062B6C0
:10C52000237C012B41F29D8172B6E36862B6002B39
:10C53000B8BF03339B103360FEF752FA98E672B629
:10C5400094E80C0010781978637A227A194202EA8A
:10C55000000259D0A37A03F00303002A42F04E8070
:10C5600043F008039A10082BA27258D8072B80F0CA
:10C570009382032B00F0868240F2CB83042B58D0A9
:10C58000062B7FF490AEE368023BE3608CE6237CED
:10C59000012B40F2478672B6E36862B6032B40F384
:10C5A000C083237C012B40F26D8672B6E36862B6CD
:10C5B000AB2B03DD72B6AC23E36062B6237C012BA8
:10C5C00040F2048672B6E26862B64DF63853002A2D
:10C5D000B8BF0332C2F20003D3ED030A9210642302
:10C5E00003FB02F38AFB0312DB17C3EBE20307EE44
:10C5F000903AB8EEE70A80EE080AF9F7F5FBFAF789
:10C60000CDF8FDF7A5FF7AE6A37A03F00303002A2D
:10C61000A8D043F004039A10082BA272A6D90C2BC1
:10C6200000F0308200F23282092BACD00B2B7FF469
:10C630003AAEE368013BE36036E600232370BFE5D2
:10C640004DF6385341F68050C2F200030021C2F289
:10C6500001000293039311700EF04CF9029B5B7979
:10C6600072B6019A9B00136262B6FDF7C9F946E6FD
:10C670004DF63653C2F200031B78042B00F0A4835E
:10C68000052B5FD1237C012B41F2148272B6E36843
:10C6900062B6032B40F30987237C012B41F29C8374
:10C6A00072B6E36862B6B3F5CA7F04DB72B64FF4C4
:10C6B000C873E36062B6237C012B41F2C48172B679
:10C6C000E36862B6002BB8BF0333C3F3870307EEFA
:10C6D000903AB8EE677A41F2D442C7EE087AC2F2D5
:10C6E000010240F21C091268C2F2010944F6E4702A
:10C6F000C0F2020089F800301A21F7EE00AA7AEEA3
:10C70000E77AC2ED587A12F09DFB99F8003007EEF7
:10C71000903AF8EE677A87EE887A7AEEC77A17EE63
:10C72000900A16F0EBFA41EC100B4EF2C000C2F288
:10C73000000005210FF088F84EF2C000C2F20000A0
:10C740000FF030F8FEF74CF9D9E54DF63652C2F24B
:10C7500000021378012B00F0B083C0F0C282022BDC
:10C7600000F0BF82032B00F0A883FDF749F94FF0DA
:10C77000010B7DE54DF63853C2F2000393ED027ACA
:10C7800027EE087A27EE097AC7EE087A77EEA87ABC
:10C79000FDEEE77A17EE903A9B0072B6E36062B660
:10C7A000237C012B40F2CB8672B6E36862B6002B85
:10C7B000B8BF03339B103360AB46FDF7C9FE57E5A6
:10C7C00072B694E80C0010781978637A227A1942CC
:10C7D00002EA000200F08B80A37A03F003030AB19F
:10C7E00043F0040343F008039A10082BA27200F2EE
:10C7F0008F80072B80F09C81032B00F0A28240F2F7
:10C800005581042B00F08F80062B7FF494ADE168F6
:10C810000239E16090E572B694E80C00107819785E
:10C82000637A227A194202EA000269D0A37A03F0FD
:10C8300003030AB143F0040343F008039A10082BE2
:10C84000A27274D8072B80F06981032B00F07482E8
:10C8500040F22681042B74D0062B7FF483ADE3686D
:10C86000023BE3607FE54DF63653C2F200031A78CF
:10C87000012A00F00385C0F0F381022A00F0F28162
:10C88000032A31D1237C012B40F2428772B6E36840
:10C8900062B6032B40F39385237C012B41F2D281B6
:10C8A00072B6E36862B67F2B4DF63853C2F20003CE
:10C8B00007DD1A79622A41F2918072B67C22E26029
:10C8C00062B6227C012A40F24D8772B6E26862B6F7
:10C8D000002AB8BF0332C2F38702114618795A7191
:10C8E00003F070FEF9F75AFFFDF78AF807E5A37A1F
:10C8F00003F00303002A3FF477AF43F0040373E728
:10C90000A37A03F00303002A98D043F0040395E7C9
:10C910000C2B00F0168200F20581092B3FF477AF53
:10C920000B2B7FF408ADE1680139E16004E50C2BC5
:10C9300000F0028200F2EC80092B90D00B2B7FF4E8
:10C9400011ADE368013BE3600DE54DF63653C2F2ED
:10C9500000031A78062A00F0FF8400F2B680042A49
:10C9600000F0EF84052A40F0A48241F61142C2F2A1
:10C9700001021970137872B69B00E36062B6237CE3
:10C98000012B41F2518172B6E36862B6002BB8BF49
:10C9900003339B1033604FF0010BFEF721F867E47F
:10C9A00072B6D8F80030D8F804101A78087898F8D9
:10C9B000091098F80830084202EA03027CD098F87F
:10C9C0000A3003F003030AB143F0040343F0080301
:10C9D0009A10082B88F80A2000F23882072B80F082
:10C9E000C884032B00F0A68440F2E284042B00F0FC
:10C9F0003882062B7FF437ADD8F80C30023BC8F8EC
:10CA00000C3032E54DF63853C2F200031B7C72B68F
:10CA10009B00E36062B6237C012B40F2518572B625
:10CA2000E36862B6002BB8BF03339B103360AB469C
:10CA3000FEF7DAFB1CE44DF63853C2F2000393ED27
:10CA4000027A27EE087A27EE097AC7EE087A77EE9F
:10CA5000A87AFDEEE77A17EE903A9B0072B6E36093
:10CA600062B6237C012B40F2978572B6E36862B60A
:10CA7000002BB8BF03339B103360AB46FCF7C0FFFD
:10CA8000FFF7F6BBE3680233E3600DE40D2B3FF4E0
:10CA9000D0AD0E2B7FF407ACE3680133E36003E411
:10CAA000012B3BD0022B3FF44CAF5BE4012B3FD07A
:10CAB000022B3FF438AF3EE498F80A3003F003034A
:10CAC000002A85D043F0040382E7072A00F0D881CA
:10CAD000082A40F0EE8140F24452C2F201020621DF
:10CAE0001278197072B69300E36062B6237C012B52
:10CAF00041F2058172B6E36862B6002BB8BF03331A
:10CB00009B1033604FF0010BFEF708FDFFF7B0BB41
:10CB10000D2B3FF416AF0E2B7FF424ACE3680133EA
:10CB2000E36020E40D2B3FF4FEAE0E2B7FF403AC4C
:10CB3000E1680131E160FFF7FFBB237C012B41F28B
:10CB4000968172B6E36862B6032B40F37685237C48
:10CB5000012B41F2328272B6E36862B6CB2B03DD61
:10CB600072B6C823E36062B6237C012B41F2408198
:10CB700072B6E36862B6002BB8BF0333C3F3870312
:10CB800007EE903A9FEDBC7AF8EE676A41F6945949
:10CB9000C6EE877AC2F2010989F80030B7EE007A52
:10CBA00077EEA87A37EE677AB4EEE97AF1EE10FA0A
:10CBB00000F3FA83DFEDAE6AB4EEE67AF1EE10FA36
:10CBC00000F14F85F0EE476AFEEEC86A16EE903A25
:10CBD00041F24442C2F20102F4EEE97AF1EE10FAB7
:10CBE000936100F3DC839FEDA27AF4EEC77AF1EE55
:10CBF00010FA00F18385B0EE677ABEEEC87A17EEC0
:10CC0000103AF4EEE97AF1EE10FAD36101F30685F9
:10CC10009FED977AF4EEC77AF1EE10FA00F169858C
:10CC2000B0EE677ABEEEC87A17EE103A45F23400DD
:10CC30001921C0F20200136212F004F94EF2C00092
:10CC400099F8001000230A22C2F200000EF0BCFD89
:10CC50004EF2C000C2F200000EF0A4FDFFF74DBB83
:10CC600002221A70237C012B40F2D18572B6E36850
:10CC700062B6032B40F3B08341F6EC32237CC2F260
:10CC80000102012B117841F2098072B6E36862B6A5
:10CC9000002BB8BF0333B1EBA30F05DC1378013BC6
:10CCA0009B0072B6E36062B6237C012B40F285855F
:10CCB00072B6E36862B61A1EB8BF03324DF6385337
:10CCC000C2F38702C2F2000310461A71029303F006
:10CCD00091F9029B5979187903F074FCF9F75EFD1C
:10CCE00002E64DF63853C2F2000301215B79117060
:10CCF00072B69B00E36062B6237C8B4240F2EC800C
:10CD000072B6E36862B6002BB8BF03339B10336082
:10CD10002BE5012B3FF4C0AE022B3FF48AACFFF7AA
:10CD2000C2BA72B60023E36062B647E472B600236B
:10CD3000E36062B6FFF74CBBE3680233E360FFF7E2
:10CD400012BBE1680231E160FFF7F6BA4DF63652E8
:10CD50004DF63853C2F20002C2F2000382F800908E
:10CD60005B7972B69B00E36062B6237C012B40F2D4
:10CD7000D28572B6E36862B6002BB8BF03339B104E
:10CD80003360FCF73DFEFFF773BA4DF6365240F2C2
:10CD90004453C2F20002C2F20103062111701B7853
:10CDA00072B69B00E36062B6237C012B40F286855D
:10CDB00072B6E36862B6002BB8BF03339B103360D2
:10CDC000FEF7ACFBFFF754BA237C012B40F2DA8567
:10CDD00072B6E36862B6032B40F36D83237C012BAC
:10CDE00041F2008072B6E36862B6B3F5CA7F04DB35
:10CDF00072B64FF4C873E36062B6237C012B40F235
:10CE0000858672B6E36862B6002BB8BF0333C3F3FE
:10CE1000870307EE903AB8EE677A41F2D442C7EE44
:10CE2000087AC2F2010241F611491268C2F2010900
:10CE300044F6C470C0F2020089F800301D21F7EEFC
:10CE400000AA7AEEE77AC2ED597A5CE40C2B00F086
:10CE5000718200F28882092B3FF4CEAD0B2B7FF458
:10CE600002ABD8F80C30013BC8F80C30FFF7FDBA24
:10CE700000FEFFC600009644000048427978304228
:10CE800041F69452C2F2010208211278197072B66A
:10CE90009300E36062B6237C012B41F2648172B699
:10CEA000E36862B6002BB8BF03339B103360FEF714
:10CEB00035FB4FF0010BFFF7DBB94DF63853C2F2EB
:10CEC000000300211B79117072B69B00E36062B60B
:10CED000237C012B3FF614AF72B658F80C2C636814
:10CEE00010781978637A227A194202EA000200F077
:10CEF0007186A37A03F003030AB143F0040343F0FD
:10CF000008039A10082BA27200F21A87072B81F0EF
:10CF1000D081032B01F0F28141F2E981042B00F072
:10CF20001A87062B7FF4EDAEE368023BE360E9E687
:10CF3000237C012B40F2248772B6E36862B6032B90
:10CF400040F38183237C012B41F23D8072B6E3687C
:10CF500062B68F2B03DD72B68C23E36062B6237C4E
:10CF6000012B40F2588772B6E36862B6002BB8BF57
:10CF70000333C3F3870307EE903AB8EE677A41F6BE
:10CF80001049C7EE0A7AC2F2010989F8003077EE3B
:10CF9000A87AF4EEE97AF1EE10FA00F3F1811FEDD0
:10CFA0004C7AF4EEC77AF1EE10FA00F15683B0EE47
:10CFB000677ABEEEC87A17EE103A41F20C42C2F21E
:10CFC000010245F218001B21C0F20200D36111F0EA
:10CFD00039FF99F8003007EE903AF8EE677A87EE5D
:10CFE0008A7A77EE287A17EE900A15F087FE41ECE0
:10CFF000100B4EF2C0000221C2F200000EF024FC21
:10D000004EF2C000C2F200000EF0CCFBFFF775B983
:10D01000237C012B40F2F98672B6E36862B6032BDB
:10D0200040F31683237C012B40F2C18772B6E3687C
:10D0300062B6CB2B03DD72B6C823E36062B6237CF5
:10D04000012B40F21F8772B6E36862B6002BB8BFAF
:10D050000333C3F3870307EE903AB8EE677A5FEDC8
:10D060007B7A5FED7B6A67EE277A40F2445987EE60
:10D07000A67AC2F2010989F8003077EE287AF5EE37
:10D08000C07AF1EE10FA00F1D4825FED846AB6EE58
:10D09000007AA7EEA67A49F68073C0F20103FCEE8F
:10D0A000C77A17EE90EA9E4540F22D839E464FF4D4
:10D0B000507040F2C863C2F201031A7ED10700F13A
:10D0C0006381D98BC3F820E0814242F0010238BF6E
:10D0D000D8831A7645F200001721C0F2020011F041
:10D0E000B1FE99F800104FF4966348F21F5203FB0B
:10D0F00001F3C5F2EB1282FB03124EF2C000D91706
:10D10000C1EB2211C2F200000EF0EEFA4EF2C000A6
:10D11000C2F200000EF046FBFFF7EFB872B694E8DB
:10D120000C0010781978637A227A194202EA000218
:10D1300000F06081A37A03F003030AB143F0040313
:10D1400043F008039A10082BA27200F26E81072B9D
:10D1500080F06984032B00F00B8440F2D685042B09
:10D1600000F06E81062B7FF421A9E368023BE360A7
:10D17000FFF71DB972B694E80C0010781978637A3D
:10D18000227A194202EA000200F04681A37A03F0F3
:10D1900003030AB143F0040343F008039A10082B79
:10D1A000A27200F27281072B80F02D84032B00F015
:10D1B0002F8440F2B285042B00F07281062B7FF49D
:10D1C0000CA9E368023BE360FFF708B972B694E884
:10D1D0000C0010781978637A227A194202EA000268
:10D1E00000F01181A37A03F003030AB143F00403B2
:10D1F00043F008039A10082BA27200F23681072B25
:10D2000080F05384032B00F0AD8440F2DB84042BC8
:10D2100000F03681062B7FF4D6A9E268023AE2607C
:10D22000FFF7D2B972B694E80C0010781978637AD7
:10D23000227A194202EA000200F0D380A37A03F0B6
:10D2400003030AB143F0040343F008039A10082BC8
:10D25000A27200F2FA80072B80F0F083032B00F01B
:10D260008C8340F2E784042B00F0FA80062B7FF4D5
:10D2700093A9E368023BE360FFF78FB903221A70BA
:10D28000FFF700BB72B694E80C0010781978637A47
:10D29000227A194202EA000200F03F81A37A03F0E9
:10D2A0000303002A41F0AE8143F008039A10082BD3
:10D2B000A27200F29E81072B80F03D85032B00F0C7
:10D2C000DC8540F2E585042B00F09E81062B7FF47F
:10D2D0006DA9E368023BE360FFF769B972B694E8B1
:10D2E0000C0010781978637A227A194202EA000257
:10D2F00000F01C81A37A03F003030AB143F0040396
:10D3000043F008039A10082BA27200F28281072BC7
:10D3100080F02C85032B00F02E8540F2C185042B74
:10D3200000F08281062B7FF44BA8E368023BE360A8
:10D33000FFF747B8D8F80C300233C8F80C30FFF7C5
:10D3400094B840F21C02C2F2010205211278197051
:10D3500072B69300FFF711BB41F61042C2F2010210
:10D360000721FFF7BDBB0D2B3FF47BAD0E2B7FF4E8
:10D370007AA8D8F80C300133C8F80C30FFF775B82C
:10D380000023C7F6FF7318E6196A8E4540F26E81D6
:10D39000DA8BC3F820E0824238BFD8839AE60023B4
:10D3A000C7F6FF73D36141E40023C7F6FF730FE4B0
:10D3B000012BDED0022B3FF454ADFFF754B84DF6ED
:10D3C0003853C2F200031A79002A40F0178572B66A
:10D3D000E26062B6FFF775BA72B60023E36062B628
:10D3E00062E4A37A03F00303002A3FF42FAF43F073
:10D3F00004032BE7A37A03F00303002A3FF4A2AE51
:10D4000043F004039EE6A37A03F00303002A3FF4EB
:10D41000F1AE43F00403EDE6A37A03F00303002A20
:10D420003FF4BCAE43F00403B8E60C2B00F0A0823E
:10D4300000F2F382092B3FF498AE0B2B7EF4B6AFCB
:10D44000E368013BE360FEF7B2BF0C2B00F095826E
:10D4500000F2EE82092B3FF40CAF0B2B7FF49CA85B
:10D46000E368013BE360FFF798B80C2B00F07A8388
:10D4700000F21583092B3FF4D0AE0B2B7FF4A3A849
:10D48000E268013AE260FFF79FB80C2B00F0C0821F
:10D4900000F2B382092B3FF494AE0B2B7EF49DAFC8
:10D4A000E368013BE360FEF799BF72B60023E360D7
:10D4B00062B6FFF700B972B60023E36062B69CE47F
:10D4C00072B658F80C2C636810781978637A227A4F
:10D4D000194202EA000200F04A83A37A03F0030330
:10D4E0000AB143F0040343F008039A10082BA27218
:10D4F00000F27A83072B80F0AA86032B00F09C862B
:10D5000040F29386042B00F07A83062B7FF488AADE
:10D51000E368023BE360FFF784BAA37A03F00303F6
:10D52000002A3FF4C3AE43F00403BFE6A37A03F03E
:10D530000303002A3FF4E6AE43F00403E2E672B6CA
:10D5400058F80C2C636810781978637A227A19429B
:10D5500002EA000200F01D83A37A03F00303002A0D
:10D5600041F0588043F008039A10082BA27200F291
:10D570001983072B80F05486032B00F02D8640F290
:10D580002486042B00F01983062B7FF40EA9E36890
:10D59000023BE360FFF70AB972B658F80C2C6368D7
:10D5A00010781978637A227A194202EA000200F0B0
:10D5B000E782A37A03F003030AB143F0040343F0C4
:10D5C00008039A10082BA27200F21E83072B80F02A
:10D5D0006586032B00F0478640F23E86042B00F060
:10D5E0001E83062B7FF442AAE368023BE360FFF749
:10D5F0003EBA0C2B00F0418400F29783092B3FF4D4
:10D6000068AE0B2B7EF4D2AFE368013BE360FEF71C
:10D61000CEBF0C2B00F0AF8300F2A283092B3FF4A6
:10D6200084AE0B2B7EF4CCAEE368013BE360FEF7E7
:10D63000C8BE01204FF0000E3BE572B60023E36048
:10D6400062B6FFF791BA72B60023E36062B686E471
:10D6500072B60023E36062B6F1E40023C8F201036E
:10D66000ABE40023C8F20103FFF7B2BA9107C3F895
:10D6700020E006D5596A7F31C9090131884238BF97
:10D680000846510706D5996A7F31C9090131884298
:10D6900038BF0846110706D5D96A7F31C90901315B
:10D6A000884238BF0846D10606D5196B7F31C909B3
:10D6B0000131884238BF0846910606D5596B7F3143
:10D6C000C9090131884238BF0846510606D5996B11
:10D6D0007F31C9090131884238BF0846D20906D0D6
:10D6E000DA6B7F32D2090132904238BF1046D883BC
:10D6F000F0E40023C8F20103FFF798BA0023C8F250
:10D700000103FFF77EBA0EF17F00C0090130D0E4BB
:10D7100072B694E80C0010781978637A227A19426C
:10D7200002EA000240F0D683A37A03F00303002A42
:10D7300040F060879A10082BA27200F21684072B23
:10D7400080F00E86032B00F0178640F20E86042B25
:10D7500000F01684062B7FF49AA8E368023BE3608E
:10D76000FFF796B872B694E8060091F800E01078DA
:10D77000627A217A10420EEA010140F09983A27A7E
:10D7800002F00302002940F04E879110082AA1728E
:10D7900000F2B283072A80F00686032A00F0F8859B
:10D7A00040F2EF85042A00F0B283062A7FF48EA8A7
:10D7B000E268023AE260FFF78AB872B694E80C00B9
:10D7C00010781978637A227A194202EA000240F04E
:10D7D0007883A37A03F00303002A40F007879A10A6
:10D7E000082BA27200F29883072B80F05886032B37
:10D7F00000F01F8640F21686042B00F09883062B5B
:10D800007FF457AAE368023BE360FFF753BA72B6AE
:10D8100094E80C0010781978637A227A194202EAA7
:10D82000000240F06083A37A03F00303002A40F073
:10D83000ED869A10082BA27200F27E83072B80F0EF
:10D840007885032B00F0818540F27885042B00F069
:10D850007E83062B7FF40BAAE368023BE360FFF7AD
:10D8600007BA72B658F80C2C636810781978637A86
:10D87000227A194202EA000200F09083A37A03F0B0
:10D8800003030AB143F0040343F008039A10082B82
:10D89000A27200F2CD83072B80F0B385032B00F03A
:10D8A000A58540F29C85042B00F0CD83062B7EF4E9
:10D8B0003CAEE368023BE360FEF738BE72B658F850
:10D8C0000C2C636810781978637A227A194202EA7C
:10D8D000000200F05A83A37A03F003030AB143F075
:10D8E000040343F008039A10082BA27200F202848A
:10D8F000072B80F06385032B00F06C8540F2638575
:10D90000042B00F00284062B7FF453AAE368023B49
:10D91000E360FFF74FBA72B658F80C2C63681078C2
:10D920001978637A227A194202EA000200F014831D
:10D93000A37A03F003030AB143F0040343F008039E
:10D940009A10082BA27200F28383072B80F0E184E7
:10D95000032B00F0628540F25985042B00F083838D
:10D96000062B7FF407AAE368023BE360FFF703BAE4
:10D97000E3680233E360FEF71ABDE3680233E36055
:10D98000FEF70BBE72B694E80C0010781978637A33
:10D99000227A194202EA000200F08A83A37A03F095
:10D9A00003030AB143F0040343F008039A10082B61
:10D9B000A27200F2B883072B80F06185032B00F080
:10D9C000638540F2A285042B00F0B883062B7FF418
:10D9D00000AAE368023BE360FFF7FCB972B60022DD
:10D9E000E26062B61A790132D2B210461A7102931D
:10D9F00002F000FB029BFEF764BF0D2B3FF450AD1D
:10DA00000E2B7EF4EAACE3680133E360FEF7E6BC7C
:10DA1000E3680233E360FEF7E1BC0D2B3FF410AD89
:10DA20000E2B7EF4C3ACE3680133E360FEF7BFBCAA
:10DA30000D2B3FF415AD0E2B7EF4AEADE368013334
:10DA4000E360FEF7AABD72B694E80C00107819786E
:10DA5000637A227A194202EA000200F05B83A37A19
:10DA600003F003030AB143F0040343F008039A10E0
:10DA7000082BA27200F20C83072B80F0E584032BA5
:10DA800000F0E78440F23A85042B00F00C83062B6B
:10DA90007EF416AEE368023BE360FEF712BE0D2B88
:10DAA0003FF4EEAC0E2B7EF48EADE2680132E26004
:10DAB000FEF78ABD72B694E80C0010781978637A84
:10DAC000227A194202EA000200F0FB82A37A03F0F4
:10DAD00003030AB143F0040343F008039A10082B30
:10DAE000A27200F2C582072B80F0E484032B00F0C1
:10DAF000158440F2FC84042B00F0C582062B7EF4D2
:10DB0000C6ADE368023BE360FEF7C2BD72B694E8BF
:10DB10000C0010781978637A227A194202EA00021E
:10DB200000F07D82A37A03F003030AB143F00403FB
:10DB300043F008039A10082BA27200F2CB82072B45
:10DB400080F09284032B00F0BA8440F2BD84042B51
:10DB500000F0CB82062B7FF455A9E368023BE3601B
:10DB6000FFF751B9E2680232E260FEF72DBDA37AF9
:10DB700003F00303002A3FF4B8AC43F00403B4E419
:10DB8000A37A03F00303002A3FF41BAD43F0040320
:10DB900017E5A37A03F00303002A3FF4E5AC43F052
:10DBA0000403E1E40C2B00F0178300F23383092B0C
:10DBB0003FF4EDAC0B2B7EF4F8ADE368013BE36082
:10DBC000FEF7F4BD012B3FF470AF022B3FF458ACCD
:10DBD000FEF7F9BCA37A03F00303002A3FF491A9EE
:10DBE00043F00403FFF78DB90C2B00F0258300F2FE
:10DBF0002883092B3FF48CAC0B2B7EF411AFE36828
:10DC0000013BE360FEF70DBF0C2B00F02C8300F20C
:10DC10003F83092B3FF4E8AC0B2B7EF427AFE3687E
:10DC2000013BE360FEF723BF72B62046F7F7F4F935
:10DC3000FEF7AABE012B3FF401AF022B3FF410AC5C
:10DC4000FEF7AABC72B694E80C0010781978637AD3
:10DC5000227A194202EA000200F09582A37A03F0C8
:10DC600003030AB143F0040343F008039A10082B9E
:10DC7000A27200F29182072B80F05484032B00F0F3
:10DC80005D8440F25484042B00F09182062B7EF4D4
:10DC900008AEE368023BE360FEF703BE72B623689A
:10DCA000606893F800E090F800C0607A237A1CEA7C
:10DCB000000F0EEA030E00F05C82A37A03F0030368
:10DCC000BEF1000F01D043F0040343F008039810A5
:10DCD000082BA07200F23782072B80F04584032BBB
:10DCE00000F0008440F2F783042B00F03782062B0B
:10DCF0007EF4CCAFE368023BE360FEF7C7BF72B6C9
:10DD00002046F7F789F9FEF7F6BE012B3FF48BAEFC
:10DD1000022B3FF495ABFEF749BB012B3FF473AEEA
:10DD2000022B3FF4BDABFEF758BB0D2B3FF46CACA0
:10DD30000E2B7EF43BACE3680133E360FEF737BCA7
:10DD40000C2B00F0DB8200F2AE82092B3FF4ECA832
:10DD50000B2B7EF4D6AFE368013BE360FEF7D2BF46
:10DD60000D2B3FF461AC0E2B7EF42AABE36801333C
:10DD7000E360FEF726BBE3680233E360FEF721BBF6
:10DD800072B694E80C0010781978637A227A1942F6
:10DD900002EA000200F01082A37A03F003030AB142
:10DDA00043F0040343F008039A10082BA27200F218
:10DDB0005F82072B80F0F483032B00F0FD8340F299
:10DDC000F483042B00F05F82062B7FF4B6A8E3688F
:10DDD000023BE360FFF7B1B872B62046F7F71CF9D3
:10DDE000FEF75FBC72B62046F7F716F9FEF7FBBFE9
:10DDF00072B62046F7F710F9FEF7BBBE72B67C226A
:10DE0000E26062B61A79013AEEE572B62046F7F79B
:10DE100003F9FFF702B972B694E80C00107819788C
:10DE2000637A227A194202EA000200F0EA81A37AB8
:10DE300003F00303002A40F0D68343F008039A104E
:10DE4000082BA27200F2CD81072B80F08283032B76
:10DE500000F09B8340F29283042B00F0CD81062BCF
:10DE60007FF482A8E368023BE360FFF77DB872B6F7
:10DE70002046F7F7D1F8FEF765BEE3680233E360AA
:10DE8000FEF795BB72B62046F7F7C6F8FFF7DCB889
:10DE9000012B3FF450AF022B3FF4B6ABFEF786BB2D
:10DEA000012B3FF463AF022B3FF4BEABFEF788BA01
:10DEB000A27A02F0030209B142F0040242F0080221
:10DEC00063E4A37A03F003030AB143F0040343F0CD
:10DED000080384E4A37A03F003030AB143F00403C4
:10DEE00043F0080326E4A37A03F003030AB143F0E6
:10DEF000040343F008039CE40C2A00F0498200F27A
:10DF00004C82092A3FF454AC0B2A7EF4DFACE26861
:10DF1000013AE260FEF7DBBC0C2B00F08A8200F2D3
:10DF2000B882092B3FF46EAC0B2B7EF4C2AEE368D3
:10DF3000013BE360FEF7BEBE0C2B00F0068200F250
:10DF4000F281092B3FF488AC0B2B7EF490AEE36892
:10DF5000013BE360FEF78CBEA37A03F00303002AC3
:10DF60003FF4EEAC43F00403EAE40C2B00F004822F
:10DF700000F2F081092B3FF4F0AB0B2B7EF487AC61
:10DF8000E368013BE360FEF783BCA37A03F003037D
:10DF9000002A3FF4A8AC43F00403A4E4A37A03F0FE
:10DFA0000303002A3FF472AC43F004036EE472B63C
:10DFB0002046F7F731F8FFF73AB872B62046F7F780
:10DFC0002BF8FEF7C9BD72B694E80C0010781978EA
:10DFD000637A227A194202EA000200F06F81A37A82
:10DFE00003F003030AB143F0040343F008039A105B
:10DFF000082BA27200F26B81072B80F0E882032BC2
:10E0000000F0B78240F2E882042B00F06B81062B0F
:10E010007EF49DAFE368023BE360FEF798BFA37A0E
:10E0200003F00303002A3FF485AD43F0040381E5C8
:10E030000C2B00F0DB8100F2DE81092B3FF439ACC0
:10E040000B2B7EF472AAE368013BE360FEF76EBA25
:10E050000C2B00F0E28100F25681092B3FF483ACD7
:10E060000B2B7EF487AEE368013BE360FEF783BED3
:10E070000C2B00F0538100F21782092B3FF441ADC5
:10E080000B2B7EF404ABE368013BE360FEF700BBBF
:10E090000C2B00F0DE8100F2D181092B3FF4FAACA9
:10E0A0000B2B7EF40DABE368013BE360FEF709BB8D
:10E0B000A37A03F00303002A3FF478AC43F004038F
:10E0C00074E4A37A03F00303002A3FF407AD43F09E
:10E0D000040303E50C2B00F0F28100F2BF81092B51
:10E0E0003FF43BAD0B2B7EF48DAEE368013BE36068
:10E0F000FEF789BE0C2B00F06D8100F25981092BCF
:10E100003FF404AC0B2B7EF454AEE368013BE360B8
:10E11000FEF750BEA37A03F00303002A3FF4A7AC36
:10E1200043F00403A3E40C2B00F0AE8100F2A181C4
:10E13000092B3FF44EAC0B2B7EF44BAEE368013B56
:10E14000E360FEF747BE0C2B00F0CC8100F20682A4
:10E15000092B3FF4CFAD0B2B7EF498ADE368013B68
:10E16000E360FEF793BD72B62046F6F755FFFEF763
:10E1700097BEA37A03F00303BEF1000F3FF4A7ADEF
:10E1800043F00403A3E5A37A03F00303002A3FF45A
:10E190006DAD43F0040369E50C2B00F0CF8100F274
:10E1A000BB81092B3FF475AD0B2B7EF47AABE36892
:10E1B000013BE360FEF775BBA37A03F00303002A7B
:10E1C0003FF4F2AD43F00403EEE5012B28D0022B1F
:10E1D0003FF4F3ACFEF7E9BAE3680233E360FEF71D
:10E1E000E5BA0C2B00F0D18100F2AD81092B3FF490
:10E1F00039AE0B2B7EF4B8AEE368013BE360FEF76B
:10E20000B3BEA37A03F00303002A3FF418AE43F031
:10E21000040314E60D2B3FF4D0AC0E2B7EF4C5AAFC
:10E22000E3680133E360FEF7C1BA012B0FD0022B84
:10E230003FF4E5ACFEF7F4BBE3680233E360FEF7BE
:10E24000F0BB0D2B3FF4DBAC0E2B7EF4E9ABE368A7
:10E250000133E360FEF7E5BB012B1FD0022B3FF437
:10E26000DEACFEF703BCE3680233E360FEF7FFBBFE
:10E270000C2B00F0A18100F28D81092B3FF4A7AD9A
:10E280000B2B7EF45AAEE368013BE360FEF755BE0C
:10E290000D2B3FF4C4AC0E2B7EF4E8ABE3680133E6
:10E2A000E360FEF7E4BB0D2B3FF455AD0E2B7EF47F
:10E2B00028ADE3680133E360FEF724BDA37A03F0E1
:10E2C0000303002A3FF493AE43F004038FE60C2BC4
:10E2D00000F04F8100F27581092B3FF49BAE0B2BB0
:10E2E0007EF435AEE368013BE360FEF730BE012B00
:10E2F000DFD0022B3FF42FADFEF703BDE3680233FE
:10E30000E360FEF7FFBC0D2B3FF4ADAE0E2B7EF4A9
:10E3100031ADE3680133E360FEF72DBDE3680233FE
:10E32000E360FEF7B5B90D2B3FF411AE0E2B7EF472
:10E330009EACE3680133E360FEF79ABC012BF8D092
:10E34000022B3FF404AEFEF792BCE3680233E360B5
:10E35000FEF78EBC0D2B3FF413AE0E2B7EF497AA66
:10E36000E3680133E360FEF793BA012BF8D0022B88
:10E370003FF406AEFEF78BBAE3680233E360FEF7C4
:10E3800087BA012A0FD0022A3FF4C1ADFEF79EBA28
:10E39000E2680232E260FEF79ABA0D2A3FF4B7ADA6
:10E3A0000E2A7EF493AAE2680132E260FEF78FBA89
:10E3B0000D2B3FF4AAAE0E2B7EF4FBACE3680133C9
:10E3C000E360FEF7F7BC012BF8D0022B3FF49DAEC3
:10E3D000FEF7EFBCE3680233E360FEF7EBBC012B12
:10E3E0000FD0022B3FF42FAEFEF79FB8E368023345
:10E3F000E360FEF79BB80D2B3FF425AE0E2B7EF4A9
:10E4000094A8E3680133E360FEF790B8012B80D055
:10E41000022B3FF428AEFEF7ADBCE3680233E360A5
:10E42000FEF7A9BC012B3AD0022B3FF480ADFEF7DA
:10E4300040BCE3680233E360FEF73CBC0D2B3FF4C5
:10E4400032AE0E2B7EF43CA9E3680133E360FEF7A5
:10E4500038B9E3680233E360FEF733B90D2B3FF4BC
:10E4600044AE0E2B7EF4CEACE3680133E360FEF7DE
:10E47000CABC0D2B3FF462AE0E2B7EF4AAACE3684F
:10E480000133E360FEF7A6BCE3680233E360FEF706
:10E49000A1BC0D2B3FF44BAD0E2B7EF40AACE36810
:10E4A0000133E360FEF706BC0D2B3FF4ECAD0E2B01
:10E4B0007EF4EDA8E3680133E360FEF7E9B8E368B2
:10E4C0000233E360FEF79FBC012BCDD0022B3FF45B
:10E4D0000CAEFEF797BC012B46D0022B3FF43EAEAC
:10E4E000FEF7D4BBE3680233E360FEF7CFBB012B3A
:10E4F000E0D0022B3FF4C7ADFEF7C9B8012BA3D083
:10E50000022B3FF4D0ADFEF7DBB8012BB7D0022BC6
:10E510003FF414AEFEF75DBC0D2B3FF448AE0E2B5E
:10E520007EF4BFA9E3680133E360FEF7BAB9012BBB
:10E53000F8D0022B3FF43BAEFEF7B3B9E3680233E9
:10E54000E360FEF7AEB90D2B3FF456AE0E2B7EF412
:10E550000BADE3680133E360FEF706BD0D2B3FF41E
:10E56000FDAD0E2B7EF492ABE3680133E360FEF762
:10E570008DBBE3680233E360FEF7E9BC012BE8D012
:10E58000022B3FF439AEFEF7EFBCE3680233E360E1
:10E59000FEF7EABC0D2B3FF476AE0E2B7EF4CDAC2D
:10E5A000E3680133E360FEF7C8BC012BF8D0022B0F
:10E5B0003FF469AEFEF7C1BCE3680233E360FEF7E7
:10E5C000BCBC0D2B3FF48EAE0E2B7EF4C0ACE368CA
:10E5D0000133E360FEF7BBBC012BF8D0022B3FF404
:10E5E00081AEFEF7B4BC43F0040326E443F0040319
:10E5F000FFF7F5B843F00403FFF79CB843F00403BA
:10E60000FDF7AEBF43F00403FEF74EBE43F0040334
:10E61000FFF70FB943F00403FEF7A4BF0023C7F6CA
:10E62000FF73FEF703BB42F00402FFF7AEB800BF72
:10E630002DE9F0432DED028B0546002783B000F154
:10E64000F004204685F8D97085F8DA7085F8DB701B
:10E6500085F8DC7085F8DD7085F8DE7085F8DF7090
:10E6600085F8E07085F8E17085F8E27085F8E37070
:10E6700085F8E47085F8E57085F8E67085F8E77050
:10E6800085F8E87085F8CC7085F8CD7085F8CE7087
:10E690000191FAF72DFF45F25C01AD22C0F20201B3
:10E6A00005F5B6700DF024FB102385F8193202F041
:10E6B000F7FF03F045F803F00BFDDDED017AB8EE4E
:10E6C000E78A2E46B0EE480A03F002FBB0EE480A95
:10E6D00003F04AFBB0EE480A03F026FCB0EE480A0D
:10E6E00002F0E0FD01992046FAF70AFF4FF40970A5
:10E6F0000DF08CFD0446F1F7C3FEC5F85C424FF403
:10E7000009700DF083FD44F2F833C0F20203036098
:10E71000C5F860024FF409700DF078FD45F2304302
:10E72000C0F20203C5F85802036005F1C0092C4687
:10E730004FF425700DF06AFD80460C3402F03EF86F
:10E7400044F8048C04F80A7C04F8097C04F8087C7A
:10E75000A1454FF00003EBD195F8D9209FEDD06A89
:10E76000DFEDCE6A85F81A3207EE902AB8EEE77A26
:10E7700095F8DB20C5F8C43067EE067A102067EE06
:10E78000A67A4FF40051FCEEE77AC5F8C830CDED1B
:10E79000017A85F8D23085F8D13085F8D03085F807
:10E7A000CF3085F8CE3085F8CD3085F8CC3085F87F
:10E7B00019029DF80430C5F8C0100AB185F8CC30B4
:10E7C00095F8DA200AB185F8CD3095F8DC200AB149
:10E7D00085F8CE3095F8E1309FEDB16ADFEDAF6A94
:10E7E00095F8E31007EE903AB8EEE77A67EE067A0E
:10E7F00067EEA67AFCEEE77ACDED017A9DF804305B
:10E8000031B195F8CC10994238BF194685F8CC1033
:10E8100095F8E21031B195F8CD10994238BF1946FC
:10E8200085F8CD1095F8E40030B195F8CE108B4204
:10E8300038BF0B4685F8CE3095F8DD309FED986AED
:10E84000DFED966A95F8DF1007EE903AB8EEE77ABA
:10E8500067EE067A67EEA67AFCEEE77ACDED017AEE
:10E860009DF8043031B195F8CC10994238BF194663
:10E8700085F8CC1095F8DE1031B195F8CD1099429D
:10E8800038BF194685F8CD1095F8E01031B195F8EC
:10E89000CE40A34238BF234685F8CE3095F8E53008
:10E8A0009FED7F6ADFED7D6A95F8E74007EE903ACD
:10E8B000B8EEE77A67EE067A67EEA67AFCEEE77ABC
:10E8C000CDED017A9DF8043034B195F8CC409C42EE
:10E8D00038BF1C4685F8CC4095F8E64034B195F831
:10E8E000CD409C4238BF1C4685F8CD4095F8E840A5
:10E8F00034B195F8CE70BB4238BF3B4685F8CE3078
:10E900002AB921B918B914B97F2385F8CE303F232D
:10E91000002485F8D830C5F8D44005F2F51105F586
:10E92000107003F037FA95F81C320BB185F81C42D1
:10E9300095F81E32002485F81B42002B00F0EF8072
:10E94000D5F8583285F81E42C5F8EC3033793BB122
:10E95000B368B47018463471F4700BB102F088FCDF
:10E960000C36B145F2D195F8D9309FED4D6A95F846
:10E97000DB1007EE903A95F8D230B8EEE77A06EE63
:10E98000903A67EE067AF8EEE66A002267EEA67A1B
:10E9900085F8CE20FCEEE77A85F8CD20CDED017A22
:10E9A0009DF8043085F8CC2009B185F8CC3095F875
:10E9B000DA200AB185F8CD3095F8DC200AB185F867
:10E9C000CE3095F8E1309FED366A95F8E31007EE0A
:10E9D000903A95F8D030B8EEE77A06EE903A67EEC6
:10E9E000067AF8EEE66A67EEA67AFCEEE77ACDEDF7
:10E9F000017A9DF8043031B195F8CC10994238BFB6
:10EA0000194685F8CC1095F8E21031B195F8CD1083
:10EA1000994238BF194685F8CD1095F8E40030B119
:10EA200095F8CE108B4238BF0B4685F8CE3095F85E
:10EA3000DD309FED1B6A95F8DF1007EE903A95F8F0
:10EA4000D130B8EEE77A06EE903A67EE067AF8EE45
:10EA5000E66A67EEA67AFCEEE77ACDED017A9DF8DC
:10EA6000043031B195F8CC10994238BF194685F879
:10EA7000CC1095F8DE1031B195F8CD10994238BF21
:10EA8000194685F8CD1095F8E01059B195F8CE40AB
:10EA9000A34238BF234685F8CE3003E000000000D3
:10EAA0000AD7233C95F8E5301FED036A95F8E74057
:10EAB00007EE903A95F8CF30B8EEE77A06EE903A46
:10EAC00067EE067AF8EEE66A67EEA67AFCEEE77A7B
:10EAD000CDED017A9DF8043034B195F8CC409C42DC
:10EAE00038BF1C4685F8CC4095F8E64034B195F81F
:10EAF000CD409C4238BF1C4685F8CD4095F8E84093
:10EB000034B195F8CE60B34238BF334685F8CE3085
:10EB10002AB921B918B914B97F2385F8CE3028460F
:10EB200003B0BDEC028BBDE8F08300BF2DE9F04FD0
:10EB30002DED028B8B00CDB00A3302AF23F007031B
:10EB40007961ADEB030D90F81D127A6002AB0646B9
:10EB50003B6139B390F81932DBB1002400F5B6758A
:10EB600003E00134A4B2A34213D904EB440206EB40
:10EB7000820108790028F4D04B78886816F82220A2
:10EB8000294602F03BF9013496F81932A4B2A342A7
:10EB9000EBD806F2F51106F5107003F0FBF8002330
:10EBA00086F81D327B69002B00F0AB8007F1270847
:10EBB00040F2200406F510739FED588ABB6028F0E0
:10EBC0000F08C2F201044FF0000A3B694FF4807253
:10EBD00003EB8A090021404614F07AFF00214FF42C
:10EBE0008072484614F074FFBD68284603F014F99B
:10EBF0008346284603F06AF996F81912002955D081
:10EC0000C7F80CA00025824603E00135EDB28D4225
:10EC10004AD205EB450306EB83031A79002AF4D0A8
:10EC2000986806F1C00300935A465346414601F0E6
:10EC30009DFFA8F1040308F1FC0E4A46F7EE006AB6
:10EC4000BFEE006A00200DE0216801312160B7EEBF
:10EC5000007AD2ED007A186037EE877A7345A2EC1D
:10EC6000017A1BD053F8041F091121F357214910D1
:10EC700007EE901AF8EEE77A87EE887AB4EEE67A35
:10EC8000F1EE10FAE0DCB4EEC67AF1EE10FAE0D55F
:10EC9000216801312160BFEE007ADAE796F8191297
:10ECA0000135EDB28D42B4D3D7F80CA07B690AF1DF
:10ECB000400A1FFA8AFA534587D83C691D4606F177
:10ECC000F0001A462146FAF79DFC7A689FED137A08
:10ECD000681E80B202EB40002146023AF1EC017A54
:10ECE00067EE877AFDEEE77A17EE903A22F8023F58
:10ECF0008242F3D107F59677BD46BDEC028BBDE8A5
:10ED0000F08F39691A4606F1F000FAF77BFC07F537
:10ED10009677BD46BDEC028BBDE8F08F00FEFF4646
:10ED20002DE9F843054690F8FC3190F81962002A65
:10ED300000F0D680183BCF1890F81A82FFB2002E50
:10ED400000F0C5804FEA480909EB080300EB830394
:10ED500041469C78CE46002C00F09380002403E0CE
:10ED60008378002B00F08D800131013491FBF6F3A4
:10ED700006FB1311E4B24FEA410E0EEB0100B44260
:10ED800005EB80005FFA81F8EAD195F81C32002B80
:10ED90006ED095F81932002B6AD02A79002A40F0FB
:10EDA000CF81012B64D92A7C002A40F0D781022B25
:10EDB0005ED02A7F002A40F0CD81032B58D095F8F1
:10EDC0002820002A40F0C881042B51D095F8342027
:10EDD000002A40F0B781052B4AD095F84020002A40
:10EDE00040F0B281062B43D095F84C20002A40F029
:10EDF000AD81072B3CD095F85820002A40F0A8811F
:10EE0000082B35D095F86420002A40F0AB81092BFF
:10EE10002ED095F87020002A40F0A6810A2B27D02A
:10EE200095F87C20002A40F0A1810B2B20D095F88A
:10EE30008820002A40F09C810C2B19D095F8942052
:10EE4000002A40F097810D2B12D095F8A020002ABF
:10EE500040F092810E2B0BD095F8AC20002A40F0A8
:10EE60007F810F2B04D095F8B830002B40F0328111
:10EE70004FEA4809C84405EB880501232B71BDE81A
:10EE8000F8838E444FEA8E0E013105EB0E0991FB9B
:10EE9000F6F306FB131685F81A6205F80E7089F86A
:10EEA000012095F81B3289F803300121134689F8B7
:10EEB0000210D9F808003A4605F5B67101F098FC41
:10EEC00095F8F431002B78D1002C7FF45EAF05F576
:10EED000107003F021F895F81C32002BC8D058E7C9
:10EEE000183BCF18FBB2002E65D00178994200F094
:10EEF000BB80012E5FD92A7B9A4200F0AF80022EA0
:10EF000059D02A7E9A4200F0A380032E53D095F860
:10EF100024209A4200F09580042E4CD095F83020A1
:10EF20009A4200F08780052E45D095F83C209A4201
:10EF30007AD0062E3FD095F848209A426ED0072E00
:10EF400039D095F854209A4262D0082E33D095F8E3
:10EF500060209A4256D0092E2DD095F86C209A4206
:10EF60004AD00A2E27D095F878209A423ED00B2E10
:10EF700021D095F884209A4232D00C2E1BD095F8DF
:10EF800090209A4226D00D2E15D095F89C209A42BA
:10EF90001AD00E2E0FD095F8A8209A4200F0938038
:10EFA0000F2E08D095F8B4209A4204D195F8B630C7
:10EFB000002B40F0A780BDE8F883D9F8080002F0E4
:10EFC00057F9002C83D0E0E695F89E20002AE0D087
:10EFD0000D2798E095F89220002AD4D00C2792E0D3
:10EFE00095F88620002AC8D00B278CE095F87A2067
:10EFF000002ABCD00A2786E095F86E20002AB0D0FF
:10F00000092780E095F86220002AA4D008277AE03A
:10F0100095F85620002A98D0072774E095F84A20E2
:10F02000002A8CD006276EE095F83E20002A80D07A
:10F03000052768E095F83220002A3FF474AF0427D2
:10F0400061E095F82620002A3FF466AF03275AE0D6
:10F05000AA7E002A3FF459AF022754E0AA7B002A77
:10F060003FF44DAF01274EE0817800293FF441AFD6
:10F0700082701746804695F81C32E3B14FF0000EBF
:10F08000734671464FF0FF3203EB430305EB8304F5
:10F09000481CA4782CB115F823309342C4BF5AB24F
:10F0A0008E4641B2B1420B46EEDB013203D098F8F6
:10F0B0000430002B62D195F81B32C3B3012388F8CA
:10F0C0000330BDE8F88395F8AA20002A3FF468AF22
:10F0D0000E2718E00F2303EB43039B00EA189178F7
:10F0E000C9B1EB5CBB42BFF466AF4FEA480909EB1C
:10F0F000080305EB8303002111719868916802F001
:10F1000063F8B7E60F2707EB470805EB88080023ED
:10F1100088F80230AFE74FEA480909EB080305EB2E
:10F12000830311719868916802F06EF8A2E607EB0C
:10F13000470205EB8205A868BDE8F84301F04ABE26
:10F140000023C8E70423C6E70523C4E70623C2E774
:10F150000723C0E70223BEE70323BCE70123BAE786
:10F160000E23B8E70823B6E70923B4E70A23B2E77A
:10F170000B23B0E70C23AEE70D23ACE70EEB4E0EEE
:10F1800007EB470205EB8E03002105EB820288F8AE
:10F190000410012119719868916802F015F88AE746
:10F1A000F8B590F8FC3190F81972183B1944002F0B
:10F1B00063D00378C9B28B4260D0012F5DD9037B45
:10F1C0008B4200F0EA80022F57D0037E8B4200F082
:10F1D000DE80032F51D090F824308B4200F0D08095
:10F1E000042F4AD090F830308B4200F0C280052FB7
:10F1F00043D090F83C308B4200F0B480062F3CD0D6
:10F2000090F848308B4200F0A680072F35D090F858
:10F2100054308B4200F09880082F2ED090F8603048
:10F220008B4200F08A80092F27D090F86C308B42F7
:10F230007CD00A2F21D090F878308B4270D00B2FE1
:10F240001BD090F884308B4264D00C2F15D090F8EE
:10F2500090308B4258D00D2F0FD090F89C308B42BD
:10F260004CD00E2F09D090F8A8308B4240D00F2FF1
:10F2700003D090F8B4308B422ED0F8BD8378002BA9
:10F280009BD000258570064690F81C320446E3B1F9
:10F2900000231A469C464FF0FF3E03EB430304EB6A
:10F2A0008300511C807830B114F823307345C4BFFB
:10F2B0004FFA83FE94464AB2BA421346EDDBBEF1E2
:10F2C000FF3F02D03379002B76D194F81B32002B0C
:10F2D00069D00123F370F8BD90F8B630002BCCD084
:10F2E0000F2505EB450600EB86060023B370CBE740
:10F2F00090F8AA30002BBAD00E25F2E790F89E3095
:10F30000002BAED00D25ECE790F89230002BA2D068
:10F310000C25E6E790F88630002B96D00B25E0E729
:10F3200090F87A30002B8AD00A25DAE790F86E3010
:10F33000002B3FF47EAF0925D3E790F86230002B15
:10F340003FF471AF0825CCE790F85630002B3FF41E
:10F3500063AF0725C5E790F84A30002B3FF455AF5F
:10F360000625BEE790F83E30002B3FF447AF052559
:10F37000B7E790F83230002B3FF439AF0425B0E7FF
:10F3800090F82630002B3FF42BAF0325A9E7837EAE
:10F39000002B3FF41EAF0225A3E7837B002B3FF435
:10F3A00012AF01259DE705EB450504EB8500BDE89F
:10F3B000F840806801F00EBD0CEB4C0C05EB4502EB
:10F3C00004EB8C03002104EB8202317101211971DD
:10F3D0009868916801F0F8FE77E700BF012380F894
:10F3E0001D32704790F81C328B4218BF80F81C12F7
:10F3F000704700BF90F81B328B4218BF80F81B1279
:10F40000704700BF90F81B02704700BF70B50446FC
:10F4100000F1C006002523793BB1A368A57018460A
:10F420002571E5700BB101F023FF0C34B442F2D129
:10F4300070BD00BF90F8D9309FED6C6ADFED6C6A4B
:10F4400090F8DB1007EE903AB8EEE77A70B467EE0A
:10F45000067A83B067EEA67A0023FCEEE77A4FF4D3
:10F460000052CDED017AC0F8C020C0F8C4309DF83C
:10F470000420C0F8C83080F8D23080F8D13080F84D
:10F48000D03080F8CF3080F8CE3080F8CD3080F8A2
:10F49000CC3009B180F8CC2090F8DA300BB180F88C
:10F4A000CD2090F8DC1009B180F8CE2090F8E13042
:10F4B0009FED4E6ADFED4E6A90F8E32007EE903A3A
:10F4C000B8EEE77A67EE067A67EEA67AFCEEE77AA0
:10F4D000CDED017A9DF8043032B190F8CC209A42FB
:10F4E00038BF1A4680F8CC2090F8E22032B190F86C
:10F4F000CD209A4238BF1A4680F8CD2090F8E440DB
:10F5000034B190F8CE20934238BF134680F8CE3005
:10F5100090F8DD309FED356ADFED356A90F8DF2039
:10F5200007EE903AB8EEE77A67EE067A67EEA67ACB
:10F53000FCEEE77ACDED017A9DF8043032B190F817
:10F54000CC209A4238BF1A4680F8CC2090F8DE20B2
:10F5500032B190F8CD209A4238BF1A4680F8CD20BB
:10F5600090F8E02032B190F8CE50AB4238BF2B4635
:10F5700080F8CE3090F8E5309FED1C6ADFED1C6A14
:10F5800090F8E75007EE903AB8EEE77A67EE067A21
:10F5900067EEA67AFCEEE77ACDED017A9DF80430AD
:10F5A00035B190F8CC509D4238BF1D4680F8CC5004
:10F5B00090F8E65035B190F8CD509D4238BF1D46C9
:10F5C00080F8CD5090F8E85035B190F8CE60B34255
:10F5D00038BF334680F8CE3029B922B91CB915B9E5
:10F5E0007F2380F8CE3003B070BC70470AD7233C2D
:10F5F0000000000003791BB18378002B40F09A8053
:10F60000037C1BB1837B002B40F09180037F1BB1F7
:10F61000837E002B40F0888090F828301BB190F852
:10F620002630002B7CD190F834301BB190F832306A
:10F63000002B71D190F840301BB190F83E30002B78
:10F6400066D190F84C301BB190F84A30002B5BD15A
:10F6500090F858301BB190F85630002B50D190F8EC
:10F6600064301BB190F86230002B45D190F87030B7
:10F6700013B190F86E30DBBB90F87C3013B190F88A
:10F680007A308BBB90F8883013B190F886303BBB52
:10F6900090F8943013B190F89230EBB990F8A03014
:10F6A00013B190F89E309BB990F8AC3013B190F83C
:10F6B000AA304BB990F8B8302BB190F8B63013B1EE
:10F6C000002380F8B6307047002380F8AA30F1E7B5
:10F6D000002380F89E30E7E7002380F89230DDE7D2
:10F6E000002380F88630D3E7002380F87A30C9E71A
:10F6F000002380F86E30BFE7002380F86230B5E762
:10F70000002380F85630AAE7002380F84A309FE7AC
:10F71000002380F83E3094E7002380F8323089E7F8
:10F72000002380F826307EE70023837674E70023E9
:10F7300083736BE70023837062E700BF90F81902C0
:10F74000704700BF2DE9F04F054690F8F211D0F850
:10F75000EC0085B002F030F995F81912002900F09C
:10F76000C780C0F3C0030093C0F3001300260193C9
:10F77000C0F34013344600F00108C0F3400BC0F35F
:10F78000800A029305F5087703E00134E4B2A14250
:10F790007CD904EB440305EB830999F80420002A83
:10F7A000F3D000212022384614F092F93946D9F8D6
:10F7B000080001F0CBFCB8F1000F6BD0D5F8201297
:10F7C00040F22D42914269D895F83812A1F1040116
:10F7D000B1FA81F1022049090122BBF1000F0AD0E0
:10F7E000D5F8242240F22D4E724503D895F83922DF
:10F7F000042A57D00246BAF1000F0DD0D5F82802DE
:10F8000040F22D4E01327045D2B205D895F83A0239
:10F81000042804BF0131C9B2009B6BB1D5F82C029A
:10F8200040F22D4E01327045D2B205D895F83B0218
:10F83000042804BF0131C9B2019B6BB1D5F8300275
:10F8400040F22D4E01327045D2B205D895F83C02F7
:10F85000042804BF0131C9B2029B6BB1D5F8340250
:10F8600040F22D4E01327045D2B205D895F83D02D6
:10F87000042804BF0131C9B2914217D095F819127A
:10F880000134E4B20136A142F6B282D8304605B066
:10F89000BDE8F08F0120424641469EE7022001224A
:10F8A00000219AE70131C9B20246A4E7002245F2DD
:10F8B0000C1089F8042089F8032089F8022010210F
:10F8C000C0F2020003920FF0BDFA039A4EF2C0009C
:10F8D000134621460A22C2F200000BF075FF4EF2D9
:10F8E000C000C2F200000BF05DFF95F819124CE762
:10F8F0000E46CBE72DE9F04100F5B67384B004461F
:10F900000A4600F5F575106856685E601860108943
:10F91000967A9E721881D07A00F00306C0F38100B7
:10F92000DE721873107BC0F3C30600F007001E756B
:10F930005873507BC0F3820600F00300DE739873A7
:10F94000907B1874D07BC0F3440600F001009E74D5
:10F950005874107CD87415339D4202F11102D2D133
:10F960000B460A4653F8660FDFEDD25A5B68C4F8BF
:10F97000EA016B6091F86E3003F01F0384F8F231F6
:10F9800091F86F30C3F3C00003F0070384F8F4016B
:10F9900084F8F3310B6FC4F8F53191F87430C3F388
:10F9A0000115C3F3420003F0010384F8FB5184F80E
:10F9B000FA0184F8F93191F8753084F8FC3152F885
:10F9C000761F04F2FD175368C4F8FD117B6013899C
:10F9D0003B8163220123072184F8073284F808322F
:10F9E00084F8092284F80B2284F80D2284F80F226F
:10F9F00084F80A1284F80C1284F80E1284F810129B
:10FA000094F8D01084F8123206EE101A94F8D2103E
:10FA100084F8133206EE901A94F8D11084F8143258
:10FA2000B8EEC66AF8EEE66A07EE101A26EE256A08
:10FA300094F8CF1084F8153266EEA56AB8EEC77A4E
:10FA400007EE901ABCEEC66AFCEEE66A27EE257A4F
:10FA50008DED016ACDED026AF8EEE77A9DF80400BB
:10FA60009DF8081084F81632BCEEC77A67EEA57AC6
:10FA700088428DED037A38BF0846FCEEE77A9DF8A0
:10FA80000C10CDED017A884238BF08469DF804106D
:10FA900084F817328842C4F8C430C4F8C83084F8F7
:10FAA000D92084F8DA3084F8DB3084F8DC3084F84C
:10FAB000DD2084F8DE3084F8DF3084F8E03084F82C
:10FAC000E12084F8E23084F8E33084F8E43084F80C
:10FAD000E52084F8E63084F8E73084F8E8302379CC
:10FAE00038BF0846102500213F2284F8CC0084F856
:10FAF0001112C4F8D41084F8185284F8CD0084F898
:10FB0000CE0084F8D8201BB1A378002B40F0A3814D
:10FB1000237C1BB1A37B002B40F09A81237F1BB178
:10FB2000A37E002B40F0918194F8283023B194F803
:10FB30002630002B40F0858194F8343023B194F8BE
:10FB40003230002B40F0798194F8403023B194F8A2
:10FB50003E30002B40F06D8194F84C3023B194F886
:10FB60004A30002B40F0618194F8583023B194F86A
:10FB70005630002B40F0558194F8643023B194F84E
:10FB80006230002B40F0758194F8703023B194F806
:10FB90006E30002B40F0698194F87C3023B194F8EA
:10FBA0007A30002B40F05D8194F8883023B194F8CE
:10FBB0008630002B40F0518194F8943023B194F8B2
:10FBC0009230002B40F05D8194F8A03023B194F87E
:10FBD0009E30002B40F0518194F8AC3023B194F862
:10FBE000AA30002B40F0518194F8B83023B194F83A
:10FBF000B630002B40F01181102384F819322546CD
:10FC000004F1C00800262B793BB1AB68AE701846F2
:10FC10002E71EE700BB101F02BFB0C354545F2D186
:10FC200094F8D9309FED246A94F8DB1007EE903AEF
:10FC300094F8D230B8EEE77A06EE903A67EE067A9C
:10FC4000F8EEE66A002267EEA67A84F8CE20FCEE93
:10FC5000E77A84F8CD20CDED017A9DF8043084F860
:10FC6000CC2009B184F8CC3094F8DA20002A40F096
:10FC7000288194F8DC200AB184F8CE3094F8E13081
:10FC80009FED0D6A94F8E31007EE903A94F8D030A7
:10FC9000B8EEE77A06EE903A67EE067AF8EEE66A94
:10FCA00067EEA67AFCEEE77ACDED017A9DF8043096
:10FCB00004E000BFA3707D3F0AD7233C31B194F824
:10FCC000CC10994238BF194684F8CC1094F8E21051
:10FCD000002940F0EE8094F8E41031B194F8CE00A1
:10FCE000834238BF034684F8CE3094F8DD301FEDF0
:10FCF0000E6A94F8DF0007EE903A94F8D130B8EE2F
:10FD0000E77A06EE903A67EE067AF8EEE66A67EE74
:10FD1000A67AFCEEE77ACDED017A9DF8043030B199
:10FD200094F8CC00984238BF184684F8CC0094F878
:10FD3000DE00002840F0B58094F8E00030B194F87F
:10FD4000CE50AB4238BF2B4684F8CE3094F8E53025
:10FD50001FED276A94F8E75007EE903A94F8CF30F9
:10FD6000B8EEE77A06EE903A67EE067AF8EEE66AC3
:10FD700067EEA67AFCEEE77ACDED017A9DF80430C5
:10FD800035B194F8CC509D4238BF1D4684F8CC5014
:10FD900094F8E650002D7CD194F8E85035B194F8F1
:10FDA000CE60B34238BF334684F8CE302AB920B98A
:10FDB00019B915B97F2384F8CE30012541F6745066
:10FDC0000A22394684F81D52C2F2010014F026F8C6
:10FDD00045F220100721C0F202000FF033F841F67F
:10FDE0007450C2F2010013F0ABFF014641F67450AB
:10FDF000C2F201000FF026F845F228100921C0F2E6
:10FE000002000FF01FF84EF2C000C2F200000BF02B
:10FE1000C9FC284604B0BDE8F081002384F8B63060
:10FE2000EAE6002384F85630A6E6002384F84A3038
:10FE30009AE6002384F83E308EE6002384F83230C0
:10FE400082E6002384F8263076E60023A3766BE66C
:10FE50000023A37362E6A1705AE6002384F886307B
:10FE6000AAE6002384F87A309EE6002384F86E30F8
:10FE700092E6002384F8623086E6002384F89E3000
:10FE8000AAE6002384F892309EE6002384F8AA3084
:10FE9000AAE694F8CD509D4238BF1D4684F8CD5057
:10FEA0007AE794F8CD00984238BF184684F8CD0020
:10FEB00042E794F8CD10994238BF194684F8CD1026
:10FEC00009E784F8CD30D4E610B5044613F038FFC6
:10FED00001462046BDE810400EF0B4BF10B5044600
:10FEE00013F02EFF014620460EF0ACFF04464EF202
:10FEF000C000C2F200000BF055FC204410BD00BF52
:10FF00002DE9F04100262F270C468E600E604E60D2
:10FF1000C1F80B600A2201F8017B804613F0DCFA7D
:10FF2000204613F00DFF08EB480540F23002C2F204
:10FF3000010208EB85051544431C27542946E018A7
:10FF400013F092FE4EF2C00745F23410C2F20007E1
:10FF50002121C0F202000EF075FF33460A2241460D
:10FF600038460BF031FC45F258100A21C0F202006D
:10FF70000EF068FF284613F0E3FE014628460EF017
:10FF800061FF44F6E8500321C0F202000EF05AFF70
:10FF9000204613F0D5FE014620460EF053FF44F6EE
:10FFA0009810C0F2020001210EF04CFF3846BDE867
:10FFB000F0410BF0F7BB00BF10B584B00C46014612
:10FFC000684613F051FE45F230116846C0F2020156
:10FFD00013F058FF28B10146204613F045FE04B047
:10FFE00010BD45F26413C0F2020303CB20606160D0
:10FFF00004B010BD2DE9F04194B0044604A804F00B
:020000021000EC
:1000000023FA41F61440C2F201004FF4B07200210D
:1000100013F05EFD41F2AD43C2F201031B7833B928
:1000200004A804F01FFA002014B0BDE8F08148F2E3
:100030001F53C5F2EB13A3FB04235B09642000FBF1
:100040001340C0B26946FFF75BFF45F26C101E21FA
:10005000C0F202000EF0F6FE684613F071FE014693
:1000600068460EF0EFFE44F698100121C0F202003F
:100070000EF0E8FE4EF2C000C2F200000BF092FB60
:1000800048F6307101236A460CA8C2F2010104F05F
:10009000B7FA14AB9DF8344053F8131DCDF81D107A
:1000A0005A689E681D7B0E99CDF82120139B9DF800
:1000B0003C20CDF825600CA88DF829508DF814400F
:1000C00006918DF81C200B9304F0CCF904A804F0E1
:1000D000E3F90028A4D004A804F0DAF941F20803F7
:1000E00098420DD045F28C101A21C0F202000EF099
:1000F000A9FE4EF2C000C2F200000BF053FB8FE7E6
:1001000004A804F011F9F0280DD045F2A8101F2121
:10011000C0F202000EF096FE4EF2C000C2F20000E5
:100120000BF040FB7CE704A804F0FEF843280DD058
:1001300045F2C8101C21C0F202000EF083FE4EF200
:10014000C000C2F200000BF02DFB69E741F207018D
:1001500004A804F093F904A804F0E6F8F72806D000
:1001600045F2E810C0F20200FFF7B8FE58E703219D
:1001700004A804F083F904A804F0D6F8092806D0EE
:1001800045F20820C0F20200FFF7A8FE48E741F25E
:10019000060104A804F072F904A804F0C5F80621C9
:1001A00046B204A804F06AF904A804F0BDF80027D8
:1001B00041F6144502463C46B846C2F2010516E037
:1001C00004F0B2F804F07F0108EB880308EB430366
:1001D0000246A1F1760009282B449CBF5B1803F866
:1001E000762C7F2904BF08F101085FFA88F80134F2
:1001F000A4B2D2B2B4F5805F04A8A7EB0207DFD1A6
:1002000045F22820C0F20200FFF75EFE07F07F07EC
:100210004EF2C000394600231022C2F200000BF05B
:10022000D3FA45F23C20C0F20200FFF74DFE4EF239
:10023000C000002310223146C2F200000BF0C4FAC5
:1002400044F69810C0F20200FFF748FEB7423FF4B0
:10025000E7AE45F24420C0F20200FFF735FE4EF251
:10026000C000394600231022C2F200000BF0ACFAA5
:1002700045F26420C0F20200FFF726FE4EF2C000F5
:10028000314600231022C2F200000BF09DFA4EF21C
:10029000C000C2F200000BF085FAC1E62DE9F04182
:1002A00092B002A804F0D0F840F23000C2F201008F
:1002B00040F21452002113F00BFC41F2AD43C2F2A4
:1002C00001031C78002C00F09E8040F23006C2F240
:1002D0000106002408E00AA804F0C4F802A804F00B
:1002E000DBF8002800F08F802F2300250A220DF173
:1002F0000501204601958DF8043013F0EDF848F61D
:100300003071C2F20101012301AA0AA804F078F9B0
:100310009DF82CE00C9D9DF834709DF836009DF8FA
:1003200037109DF838209DF839309DF83AC09DF877
:1003300035808DF80CE004959DF83BE08DF8147045
:100340009DF83D509DF83C708DF816008DF8171003
:100350009DF83E009DF83F108DF818208DF819305B
:100360009DF840209DF841308DF81F108DF8202019
:100370008DF81AC08DF81BE08DF81E008DF81580E1
:100380008DF81C708DF81D508DF821300AA8119B36
:10039000099304F067F802A804F07EF8012202A98C
:1003A00088B30AA804F0A4F90AA804F05FF80028AA
:1003B00091D10AA804F058F804EB440504EB850534
:1003C00035440146284613F04FFC45F26C200C21C1
:1003D000C0F202000EF036FD284613F0B1FC0146D3
:1003E00028460EF02FFD44F698100121C0F20200BD
:1003F0000EF028FD4EF2C000C2F2000001340BF0F6
:10040000D1F9E4B267E702A804F02CF8204612B054
:10041000BDE8F0812DE9F0470E469046054604F010
:1004200037F841F2080398420FD045F28C10C0F221
:1004300002001A210EF006FD4EF2C000C2F20000CA
:100440000BF0B0F90020BDE8F087284603F06CFF00
:10045000F02805D045F2A810C0F202001F21E9E7FC
:10046000284603F061FF432805D045F2C810C0F2CA
:1004700002001C21DEE741F20701284603F0FEFFDF
:10048000284603F051FFF72805D045F2E810C0F2E6
:1004900002001D21CEE70321284603F0EFFF284686
:1004A00003F042FF092804D045F20820C0F2020000
:1004B000EFE741F20601284603F0E0FF284603F08B
:1004C00033FF06214FFA80F9284603F0D7FF06F1E3
:1004D000010A00244FEACA1AF6012746284603F00B
:1004E00023FFB442C3B2A7EB030704DBA31B5445AD
:1004F000B8BF08F803000134B4F5805FEED145F2CF
:1005000028201221C0F202000EF09CFC07F07F07A9
:100510004EF2C000002310223946C2F200000BF058
:1005200053F945F23C200421C0F202000EF08AFC8F
:100530004EF2C000002310224946C2F200000BF028
:1005400043F944F698100121C0F202000EF07AFC43
:100550004EF2C000C2F200000BF024F94F4508D162
:1005600040F22C03C2F2010300221A800120BDE8F0
:10057000F08745F244201F21C0F202000EF062FC19
:100580004EF2C000394600231022C2F200000BF0E8
:100590001BF945F264200621C0F202000EF052FC65
:1005A0004EF2C000494600231022C2F200000BF0B8
:1005B0000BF94EF2C000C2F200000BF0F3F800207D
:1005C000BDE8F08730B541F2AD42C2F20102B5B0EC
:1005D0001378002B00F09C80044604A80D4603F01D
:1005E00033FF48F21F53C5F2EB13A3FB04235B094F
:1005F000642000FB1340C0B26946FFF781FC48F657
:10060000307101236A4614A8C2F2010103F0F8FF19
:1006100034AB9DF8544053F8732DCDF81D20596824
:100620009A681B7BCDF82110CDF8252016999DF8EE
:100630005C208DF8293014A81B9B8DF8144006917E
:100640008DF81C200B9303F00DFF04A803F024FF8A
:10065000044600BB45F27C201021C0F202000EF0DF
:10066000F1FB684613F06CFB014668460EF0EAFBAE
:1006700045F29020C0F2020008210EF0E3FB4EF29A
:10068000C000C2F200000BF08DF804A803F0EAFEEF
:10069000204635B030BDDDF82130DDF81D20CDF825
:1006A0004130DDF82530CDF84530CDF83D209DF8BE
:1006B0002930069A8DF849300E929DF814308DF845
:1006C000343045F6F8029DF81C308DF83C30C0F20D
:1006D000020205F01F050B9B0C9229460CA814AAD8
:1006E0001393FFF797FE04460CA803F0BBFE04BB70
:1006F00045F2AC201A21C0F202000EF0A3FB4EF22C
:10070000C000C2F200000BF04DF804A803F0AAFEEE
:1007100045F2C8201321C0F202000EF093FB4EF206
:10072000C000C2F200000BF03DF80024204635B0B6
:1007300030BD0A220DF1C6010CA813F06FFB45F283
:100740009C200E21C0F202000EF07CFB684613F0E4
:10075000F7FA014668460EF075FB44F60470022174
:10076000C0F202000EF06EFB05EB850341F614406B
:1007700005EB4305C2F201000544284613F0E0FAF8
:10078000014628460EF05EFB44F698100121C0F2A7
:1007900002000EF057FB4EF2C000C2F200000BF058
:1007A00001F841F2D443C2F2010314A91868FFF71B
:1007B000A1F8044669E700BF0BF0F6B90022C0F8C3
:1007C000A421C0F89C21C0F8B421C0F8AC21C0F825
:1007D000C421C0F8BC21C0F8D421C0F8CC21C0F895
:1007E000E421C0F8DC21C0F8F421C0F8EC21704706
:1007F0002DE9F04F45F255541646C0F2150404FB9E
:1008000006F49A4604F142732DED088B08EE903AF7
:100810004FF04E530AEE103A4CF28303CBF6CA6304
:1008200009EE903A43F27A63C3F6AB4309EE103A0D
:100830004DF20A73C3F623430BEE103A4AF63B23FC
:10084000C4F6B83345F256550AEE903A18EE903A8F
:10085000C5F2555593B085FB022703F2317332463A
:10086000A7EBE67745F2243B08EE903A4FEA6A039D
:1008700003958146073F08930C460546C0F2020BDC
:100880000026099190464EE0BAF1000F00F30F8167
:100890006FF0EE0101FB02F20732D21000EB0213FF
:1008A000002F23EAE373627B40F3FF801F2FCCBF4E
:1008B000C2EB42127A43D21000920AA90EAA09EBA7
:1008C000060000F007FD627CA37CE17C207D002A0D
:1008D0007AD003F0030C4FF0640E40F678031EFB51
:1008E0000C11C0F2440303FB01F307284FEAE301B4
:1008F000C3BF073843F29143434300230B44C5F879
:100900006C22C5F83032A37B03F0030344365BF856
:100910002330C5F85432B6F5CC7F04F1150405F147
:10092000040500F0D48020782179627863790A90F8
:10093000A0780E910B92A179E2780F930C90E37955
:10094000207C0D921193109100F01EFE237AC3EBD0
:100950000803B3F1110200F18680039A217B94F819
:100960000AE0103B82FB03C2A2EBE37301B303294D
:100970001ED01F2BDBBF45F2B432C0F20202FA23B5
:10098000D35C03FB0EFE40F2491303FB0EF3012977
:100990004FEAE33316DD18447F28A8BF7F20BAF161
:1009A0007F0F4FEA4010E27B7FF76EAF0F2171E7B8
:1009B00003FB0EF340F2491202FB03F301294FEA55
:1009C0002333E8DC5B42E6E7B8EEE88A079028EEDE
:1009D0000A0A069120EE290A059304920FF0C8FC3A
:1009E00020EE090AF1EE0C7A80EE277A0798059B33
:1009F0000699073845F2343E03F01F03C0F2020E99
:100A00005EF8233007EE900A27EE087AF8EEE77AD0
:100A1000A7EE278ABDEEC88A18EE102A1A4413469C
:100A2000049A00293FF46BAF07EE901AF8EEE77ACC
:100A3000B7EE000AA7EE8B0A05930FF01BFDF6EE4A
:100A4000007AE0EE2A7A17EE900A12F057F941EC9C
:100A5000100B0EF069FF51EC100B12F053FC059BCC
:100A6000049A03444BE7039B94F809C0C2F10101C7
:100A7000E27A83FB013EAEEBE17102B3032A1ED0A2
:100A80001F29DBBF45F2B43EC0F2020EFA211EF868
:100A9000011040F2491301FB0CF103FB01F3DB13DE
:100AA000012A3FF778AF5B4275E7002204E745F281
:100AB000DC23C0F202030899595CEF39EAE601FB36
:100AC0000CF140F2491303FB01F31B13E8E7DDF8D7
:100AD000248098F87E5098F8824098F87F3098F8F3
:100AE000830098F880600A950E9498F8845098F8DE
:100AF00081400B930F9098F8853011930EAA0AA9A4
:100B000009F5FC700C9610950D9401F029FA98F8EF
:100B10008630C9F8883298F887302BB3C3F10803C0
:100B2000C9F8503298F88B3003EB830303EB43137F
:100B30009B11C9F88C3298F88F3045F21C32C0F204
:100B4000020203F00703D35CC9F8903298F88C30A6
:100B500003EB830303EB43139B11C9F8843213B0F7
:100B6000BDEC088BBDE8F08F1023D9E72DE9F04FDD
:100B70002DED048B89B0D0F89052DDF858800791A4
:100B80008146D0F88C0298F80DE09B46A2F5000350
:100B900005FB03F500FB0BF0A0FB0567EB1700FB63
:100BA000037714468EFB0523900B40EA8340FE1129
:100BB00086EAE67380EAE072A2EBE072A3EBE673EA
:100BC0009342B8BF134609F5FC701E4601F000FAC7
:100BD000D8F80030002DB4BF4FF0FF320122B3F53A
:100BE000005A06FB02001AD0D8F80820002A40F06C
:100BF000D980D8F804304FEACA2A07EE90AA07EE47
:100C0000103AF8EEE77AB8EEC77AF2EE086A67EEC5
:100C1000877A87EEA67AFDEEC77A17EE90AA4FF094
:100C20005A5309EE103A45F62943C3F68F53D9F8C3
:100C3000842298F80C1008EE903A43F23333C4F251
:100C4000431308EE103A82FB0B23C4F180744FEA81
:100C5000122B4BEA036BE3170BFB03F298F80E30F1
:100C6000002704FB07225B04ABFB046781FB044500
:100C7000C3F57E0BE30943EA45635B4517444FEA3E
:100C8000166138BF5B4641EA0721D8F814208B4231
:100C900038BF0B4692449B4600EB0A0305934E4631
:100CA00009F50C744F46002514E0504401F040F85B
:100CB000C6F8A001384600F065FB626A02BBC6F8C0
:100CC00098010135062D07F1440706F1100604F1DD
:100CD000040452D098F818302B4113F0010344D08B
:100CE000E36B2068002BE0D1059B184401F020F84D
:100CF000C6F8A001384600F045FB626A002ADED043
:100D0000D117ABFB0223CDE90223039A06900BFB1C
:100D100001230393DDE90201020E42EA012207EEFC
:100D2000902AF8EE677AB0EE480A67EE897AA7EE65
:100D3000A80A0FF01DFBFCEEC07A069817EE901A79
:100D4000C3174FEA011E0EFB03F3090F00FB01312D
:100D5000AEFB0023CDE902230B440393029B1A0F41
:100D6000039B42EA0312801AA9E73846029300F077
:100D700009FB029BC6F89831A3E7D8F82C00D9F8F4
:100D800050120268D9F88832019109F51271009168
:100D90009468079909F5CC72A04709B0BDEC048BA3
:100DA000BDE8F08F21230C21C8F2040391FBF2F27D
:100DB00002FB0AFA83FB0A1353444FEAEA7ACAEBAE
:100DC000233A41F6FF7393FBF2F303FB0AFA4FEA6F
:100DD000CA2A24E770B50646044600F5CC752046BD
:100DE0000021443400F080FBAC42F8D106F5FC70E1
:100DF0000021BDE8704001F039B900BF2DE9F04F86
:100E000045F255549246C0F2150404FB0AF4994683
:100E100004F142732DED088B08EE903A4FF04E53DB
:100E20000AEE103A4CF28303CBF6CA6309EE903A0D
:100E300043F27A63C3F6AB4309EE103A4DF20A73FC
:100E4000C3F623430BEE103A4AF63B23C4F6B833FD
:100E500045F256550AEE903A18EE903AC5F25555BD
:100E600093B085FB0A2803F23173A8EBEA7845F2C8
:100E7000243B08EE903A4FEA690302950746079033
:100E80000891A8F1070809930C460546C0F2020B29
:100E900000262AE0B9F1000F00F312816FF0EE0195
:100EA00001FB02F20732D21000EB0213B8F1000F7F
:100EB00023EAE373627B40F30181B8F11F0FCCBFDB
:100EC000C2EB421208FB02F2D21000923846013601
:100ED0000EAA0AA900F062FB062E04F1150405F122
:100EE000040507F1440700F0FB80627CA37CE17CF1
:100EF000207D002A71D003F0030C4FF0640E40F601
:100F000078031EFB0C11C0F2440303FB01F3072816
:100F10004FEAE301C3BF073843F291434343002341
:100F20000B44C5F83032A37BC5F86C2203F00303F1
:100F30005BF82330C5F854322078217962786379E0
:100F40000A90A0780E910B92A179E2780F930C9001
:100F5000E379207C0D921193109100F015FB237A18
:100F6000C3EB0A03B3F1110200F18680029A217BE0
:100F700094F80AE0103B82FB03C2A2EBE37301B3D7
:100F800003291ED01F2BDBBF45F2B432C0F2020290
:100F9000FA23D35C03FB0EFE40F2491303FB0EF36E
:100FA00001294FEAE33316DD18447F28A8BF7F20CC
:100FB000B9F17F0F4FEA4010E27B7FF76BAF0F2153
:100FC0006EE703FB0EF340F2491202FB03F3012923
:100FD0004FEA2333E8DC5B42E6E7B8EEE88A0690A6
:100FE00028EE0A0A059120EE290A049303920FF0D5
:100FF000BFF920EE090AF1EE0C7A80EE277A069806
:10100000049B0599073845F2343E03F01F03C0F2F4
:10101000020E5EF8233007EE900A27EE087AF8EE0B
:10102000E77AA7EE278ABDEEC88A18EE102A1A447E
:101030001346039A00293FF474AF07EE901AF8EEB6
:10104000E77AB7EE000AA7EE8B0A04930FF012FAC4
:10105000F6EE007AE0EE2A7A17EE900A11F04EFED4
:1010600041EC100B0EF060FC51EC100B12F04AF941
:10107000049B039A034454E7029B94F809C0C2F10D
:101080000101E27A83FB013EAEEBE17102B3032A78
:101090001ED01F29DBBF45F2B43EC0F2020EFA217A
:1010A0001EF8011040F2491301FB0CF103FB01F3A0
:1010B000DB13012A3FF778AF5B4275E7002204E7B4
:1010C00045F2DC23C0F202030999595CEF39E7E6E7
:1010D00001FB0CF140F2491303FB01F31B13E8E79A
:1010E000089A079992F88630C1F8883292F88730CA
:1010F0003BB3C3F1080308461446C0F8503294F8D5
:101100008B3003EB830303EB43139B11C0F88C324A
:1011100094F88F3045F21C32C0F2020203F007034C
:10112000D35CC0F8903294F88C3003EB830303EB6C
:1011300043139B11C0F8843213B0BDEC088BBDE89B
:10114000F08F102308461446D7E700BF2DE9F84F6B
:1011500043F6886A804689460646A1F1040B01F1F0
:10116000180500F160070446C2F2010AD4F898118C
:1011700001F172414A1340F2FE731340581C5AF8B1
:1011800023205AF82000C1F30D0382FB0323920BA6
:1011900042EA83420916C1F1060102440A4130467F
:1011A000294610344BF8042F00F050FAA74205F1FD
:1011B000010506F14406D9D109F11E0108F5FC70BC
:1011C000BDE8F84F00F080BF2DE9F04104460F461E
:1011D00000F5CC7806460D463946204600F03AFA2E
:1011E000D5F89C31C6F89C314434D5F8A431C6F802
:1011F000A431444507F1440705F1100506F1100636
:10120000EAD1BDE8F08100BFD1F8AC31D1F8A4211A
:1012100010B4D1F89C41C0F89C41C0F8A421C0F89A
:10122000AC31D1F8B431C0F8B431D1F8BC31C0F828
:10123000BC31D1F8C431C0F8C431D1F8CC31C0F8D8
:10124000CC31D1F8D431C0F8D431D1F8DC31C0F888
:10125000DC31D1F8E431C0F8E431D1F8EC31C0F838
:10126000EC31D1F8F431C0F8F4315DF8044B70473B
:101270000023C0F89C31C0F8A431C0F8AC31C0F8EC
:10128000B431C0F8BC31C0F8C431C0F8CC31C0F8BA
:10129000D431C0F8DC31C0F8E431C0F8EC31C0F82A
:1012A000F43170474FF48843C4F22C7307EE103AC0
:1012B00087EE000A4FF0974307EE903A20EE270A98
:1012C0004DF64C53BCEEC00AC2F2000383ED000A97
:1012D000704700BF30B40C680460146804614D6846
:1012E0004560556845618D68856095688561C96808
:1012F000C160D268C261132C4FF000028262426367
:10130000DBBF45F2D832C0F202021C3452F824404E
:101310000362641003EB8413A3F5855302680299FA
:101320004162102B02EB8204B8BF102302EBC4020F
:101330001B04002B01EBA212D4BF002401240125C1
:101340003E2A80F84050C36280F8304016DC02F03C
:10135000030392100433083203FA02F2D3174DF656
:101360004C51C2F200010968A1FB024501FB035583
:10137000230E43EA0523836330BC70474FF060724D
:101380000023ECE7426B022AF0B4034605DD032A92
:1013900066D190F84010002962D193F8301071B9ED
:1013A000986A996BDC6A401AA042986259DC511C19
:1013B00003299C6259635BDD2046F0BC70474FF601
:1013C000FF70996AC0F2B36081424CDDC1F1885070
:1013D00000169D6BDC6A05FB0010A042986240DBA2
:1013E000511C03299C625963E6DC03EB82025169BC
:1013F0001329DBBF45F2D830C0F2020001F11C0511
:1014000050F82150196A586A6D1001EB8511A1F549
:1014100085511029B8BF102109048C42ACBF0025AA
:101420000125D96283F83050526802EB820102EB49
:10143000C10200EBA2123E2A4CDD4FF0607600277D
:101440004DF64C52C2F2000220461268A2FB06453D
:1014500002FB0755220E42EA05229A63F0BC704750
:10146000986AF0BC70470021C0F2B4610A20B0E76E
:1014700003EB820251691329DBBF45F2D830C0F279
:10148000020001F11C0550F82150196A586A6D10CC
:1014900001EB8511A1F585511029B8BF1021090470
:1014A0008C42ACBF00250125D96283F830505268C8
:1014B00002EB820102EBC10200EBA2103E28BCDC71
:1014C00000F0030680100436083006FA00F00646E5
:1014D000C717B5E702F0030692100436083206FA81
:1014E00002F21646D717ABE790F840308B4241D056
:1014F00000290CBF0323002330B49D00421980F85B
:10150000401043631369816A132BDBBF45F2D83265
:10151000C0F2020203F11C0452F82340036A426A3B
:10152000641003EB8413A3F58553102BB8BF10236D
:101530001B048B42D4BF0021012180F83010C3620C
:10154000435903EB830103EBC10302EBA3123E2AD1
:1015500011DD4FF0607200234DF64C51C2F20001D4
:101560000968A1FB024501FB0355230E43EA05234D
:1015700030BC8363704702F00303921004330832D7
:1015800003FA02F2D317E7E71328DBBF45F2D8339B
:10159000C0F202031C3053F82000704730B40C68CE
:1015A0000460146804614C684460546844618C6849
:1015B000846094688461C968C16090F84010D568FF
:1015C000029AC56103624262002934D0132CDBBF4A
:1015D00045F2D831C0F202011C3451F8244085682C
:1015E000816A641003EB8413A3F58553102BB8BFF5
:1015F000102305EB85041B0405EBC4058B4202EBAD
:10160000A512D4BF0021012102243E2AC36280F822
:101610003010446311DD4FF0607200234DF64C51E1
:10162000C2F200010968A1FB024501FB0355230E2C
:1016300043EA0523836330BC704702F00303224171
:101640000433083203FA02F2D317E7E7436B0B7057
:10165000704700BF0A680B69036102604B68436012
:101660004B6943618B6883608B698361CB68C3601E
:10167000F0B5CB69C3610B6A4F6A8E6ACD6A91F887
:1016800030E04C6B8A6B036291F8403047628662AF
:10169000C56280F830E04463826380F84030F0BD7A
:1016A00070B54FF09D432DED048B08EE103A41F2DA
:1016B0003063002143F68864C3F680730020C4F2CF
:1016C000D01108EE903AC2F201040025B6EE009A5D
:1016D0000BE078EE097A17EE900A11F00FFB41EC5F
:1016E000100B0EF021F951EC100B6E0011F00AFEF8
:1016F00001360135B5F5806F28EE288A44F82600BA
:10170000E7D1002340F2FF355A00D11C501C54F899
:10171000211054F820000133091AAB4243F68860C7
:1017200044F82210C2F20100EED141F6FC73BDEC88
:10173000048BC35841F6F872C3F10043835070BD67
:10174000002207EE902A4FF0974202EE102A4FF047
:101750006C5204EE902A4FF06E5202EE902A4AF636
:10176000AB22C3F62A2241F6886303EE102AC2F2A6
:1017700001030022F6EE003AB7EE006AB0EE004A2E
:10178000F0EE465AE7EEE75A03EBC2010132B0EE43
:10179000677AA5EEA47AB2F5806FB0EE465AA7EE4E
:1017A000475AF0EE636AE7EE826AB0EE677AA5EE1A
:1017B000247AFDEEE66AC1ED016AF0EE466AE7EED4
:1017C000476AB0EE677AA6EEA27A76EE856AB0EE48
:1017D000465AA7EE475A35EE257AA6EE847AE7EE0A
:1017E000037ACDD130B4002240F2FF355100C81C3D
:1017F0004C1C53F8200053F824400132001BAA422D
:1018000041F6886443F82100C2F20104EED14FF0A2
:10181000974306EE903AB6EE007AA7EEA67A41F626
:10182000FC7341F6F872E358FDEEC77A17EE901A92
:10183000CB1AA35030BC7047704700BF2DE9F04F62
:1018400045F23C4491B003EB4303C0F2020404EBC5
:10185000C3041546069007910FCC0AAE0FC694E854
:101860000300002386E803004FF0010843F6886672
:101870000AAF05F160098DF824808DF825308DF8C8
:101880002630C2F2010605973BE00AF1FF30069BC5
:1018900000EB001003EB0010133020F00F0095E870
:1018A000084003F1724B4FEA6B3340F2FE721A406C
:1018B000531C56F8222056F82340CBF30D0382FB2D
:1018C0000323920B4FEA2B6B42EA8342CBF1060BC8
:1018D000144444FA0BF4BEF58C6F6C601CDAB4F55A
:1018E0008C6F19DABCF1000F03D110AB9A440AF8DF
:1018F0001CCCEB68AA6803EB8213EB601035A9459A
:101900002FD0059B53F8041B059311F0030A01F037
:10191000040CBAD10798C2E710AB9A441AF81C3CE1
:101920001BB11CF1000318BF0123C1F301123AB12E
:1019300010AF07EB020C1CF81CCCBCF1000F13D14C
:1019400001F0C001C02902D11B9A0F2A20DDAA682C
:10195000E96801930094734600F0D6F80AF81C8CED
:10196000C7E711B0BDE8F08F0699D5F808C0013A75
:1019700002EB021201EB02111331EA68029321F02B
:101980000F0163460194CDF800E000F051F8E5E75F
:101990001746E968AA6802971A9F03938DE890009A
:1019A000734600F00FF9D9E710B54FF409710446FA
:1019B0000AF02EFC204610BD45F23C43F0B401EB8A
:1019C0004101C0F2020303EBC1040FCC86B06D46A7
:1019D0000FC507460B4694E80300C7F3800485E86B
:1019E000030013F0040F44F0020314BF184620460E
:1019F000164640F00403039A049916F0040F18BF2A
:101A0000184640F0080312F0040F059A18BF184654
:101A100011F0040F40F0100308BF034612F0040F4A
:101A200043F0200008BF184606B0F0BC704700BF66
:101A30002DE9F04F099E0A9C9DF82C50C6EB040C32
:101A40000CF1200C9E464FEAAC1C46F6946785B319
:101A5000C2F201074FF0400B4FF0000A51F82A4044
:101A600014444FEA643840F2FE7508EA0505C4F3F1
:101A70000D0457F82530013583FB048957F82550AC
:101A800050F82A304FEA983444EA89442C4466449A
:101A900084FB06894FEA186444EA09242344BBF115
:101AA000010B40F82A3072440AF1010AD6D1BDE890
:101AB000F08FAA46C2F201074FF0400B51F82A30CE
:101AC00013445D1340F2FE742C40C3F30D0357F82A
:101AD0002450013485FB038957F824404FEA98339A
:101AE00043EA89431C44664484FB0645230E43EACB
:101AF0000523BBF1010B40F82A3072440AF1010AB8
:101B0000DCD1BDE8F08F00BF2DE9F043079C9DF8C4
:101B10002050C3EB040C0CF1200C4FEAAC1C46F631
:101B2000946E4DB3C2F2010E4FF040094FF0000821
:101B30004D1340F2FE742C40651C5EF824605EF884
:101B40002550C1F30D0486FB0467B40B44EA8744B7
:101B50002C44634484FB03562C0E50F8285044EA6E
:101B600006242C44B9F1010940F82840114408F139
:101B70000108DDD1BDE8F083A846C2F2010E4FF0A6
:101B800040094D1340F2FE742C40651C5EF8246041
:101B90005EF82550C1F30D0486FB0467B40B44EADC
:101BA00087442C44634484FB03562C0E44EA0624E9
:101BB000B9F1010940F82840114408F10108E0D1C9
:101BC000BDE8F0832DE9F04F099F0A9C9DF8308015
:101BD000D4F800C065680B9EC3EB070A0AF1200A1F
:101BE0001C4696464FEAAA1A46F69467B8F1000FCB
:101BF00039D0C2F20107624606F1010BD4464FF01C
:101C000040094FF00008BA4600E03546561946FA3A
:101C10000BF60E44721340F2FE731340C6F30D022E
:101C20005AF82360013386FB02675AF82330B20B5F
:101C300042EA874264441A4482FB0423160E46EAB1
:101C4000032650F82830B9F10109334440F8283010
:101C50007144334608F101082A46D6D10A9A156024
:101C60005360BDE8F08F864601366046C2F2010738
:101C70004FF040098B46944600E00D462844304121
:101C80005844421340F2FE731340C0F30D0057F85E
:101C90002320013382FB000157F82320830B43EA02
:101CA000814354441A4482FB0423110E41EA032168
:101CB000B9F101094EF82810E3440B4608F1010878
:101CC0002846DAD10A9A15605360BDE8F08F00BF4C
:101CD00038B54FF0AB4307EE903A2DED048B87EE0D
:101CE000808A41F23063C3F6807345F6846446F619
:101CF0008865C2F20104C2F2010509EE103AF6EE5F
:101D0000008A78EE287A28EE098A17EE900A10F0F9
:101D1000F5FF41EC100B0DF007FE51EC100B11F02C
:101D2000F1FA44F8040FA542EBD1BDEC048B38BDA9
:101D300010B445F68861C0F38934631CC2F2010116
:101D4000C0F30D0251F8233051F824105DF8044B14
:101D50005B1A83FB0223920B001642EA8342C0F116
:101D6000140388181841704743F20C03C4F6C0638B
:101D700007EE903A87EE800A46F68C63C2F20103C2
:101D8000F6EE007A30EE270ABDEEC00A83ED000AB7
:101D9000704700BF0B7810B4002B35D003EB8303E2
:101DA00003EB43139A119F2AC5BFA2F1A0031B1195
:101DB0000B230B3302FB03F346F68C62C2F20102E3
:101DC000146803FB04F343604A78C2F16303EAB189
:101DD00003F00F021B11013310329A404FF680734B
:101DE0001340802BB8BF802304FB03F304FB02F2F3
:101DF000436102614B7903720B795DF8044B003348
:101E000018BF0123837270470B23D5E74FF0FF33D0
:101E100003614361EEE700BF03684168027A0B4447
:101E2000022A03603BD00CD9042A14D032D3052AED
